:1000000000000320D5010000550200003D3B010027
:10001000590200005B0200005D02000000000000C9
:100020000000000000000000000000005F0200006F
:100030006102000000000000630200006502000091
:10004000251A01002D1A0100958D0000351A0100B6
:100050003D1A0100451A01004D1A0100551A010010
:100060005D1A0100651A01006D1A0100751A010080
:100070007D1A0100851A01008D1A0100951A0100F0
:100080009D1A0100A51A0100AD1A0100B51A010060
:10009000BD1A0100C51A0100CD1A0100D51A0100D0
:1000A000DD1A0100C5900000E51A0100ED1A0100FB
:1000B000F51A0100FD1A0100051B01000D1B0100CE
:1000C000151B01001D1B0100251B01002D1B01003C
:1000D000351B01003D1B0100451B01004D1B0100AC
:1000E000551B01005D1B0100651B01006D1B01001C
:1000F000751B01007D1B0100851B01008D1B01008C
:10010000ED80000051800000C5800000951B0100BB
:100110009D1B0100A51B0100AD1B0100B51B0100CB
:10012000BD1B0100C51B0100CD1B0100917F00001C
:10013000D51B0100DD1B0100E51B0100ED1B0100CB
:10014000F51B0100FD1B0100051C01000D1C010039
:10015000151C01001D1C0100251C01002D1C0100A7
:10016000351C01003D1C0100451C01004D1C010017
:10017000551C01005D1C0100651C01006D1C010087
:10018000751C01007D1C010079CB000001CB000033
:1001900029CB000051CB0000D867010000000020EF
:1001A000A0010000D86701000000FF1F0000000050
:1001B000D86701000000001400000000A00100202A
:1001C000002B00000000FF1F0000000000000014D2
:1001D0000000000010B572B60EF076F90E4B0F4A13
:1001E000934208D203F10C049A685968186800F029
:1001F00019F82346F3E70A4A934207D21C46596886
:1002000054F8080B00F01DF82346F4E70FF084FDC6
:1002100062B607F009FAFEE798010000BC01000091
:10022000D4010000002393420AD210B450F8044BCA
:1002300041F8044B04339342F8D35DF8044B704704
:10024000704700238B4204D2002240F8042B043371
:10025000F8E77047FEE7FEE7FEE7FEE7FEE7FEE7AA
:10026000FEE7FEE7FEE7FEE7FFFFFFFFFFFFFFFF02
:10027000FFFFFFFFFFFFFFFFFFFFFFFFFFFFFFFF8E
:10028000FFFFFFFFFFFFFFFFFFFFFFFFFFFFFFFF7E
:10029000FFFFFFFFFFFFFFFFFFFFFFFFFFFFFFFF6E
:1002A000FFFFFFFFFFFFFFFFFFFFFFFFFFFFFFFF5E
:1002B000FFFFFFFFFFFFFFFFFFFFFFFFFFFFFFFF4E
:1002C000FFFFFFFFFFFFFFFFFFFFFFFFFFFFFFFF3E
:1002D000FFFFFFFFFFFFFFFFFFFFFFFFFFFFFFFF2E
:1002E000FFFFFFFFFFFFFFFFFFFFFFFFFFFFFFFF1E
:1002F000FFFFFFFFFFFFFFFFFFFFFFFFFFFFFFFF0E
:10030000FFFFFFFFFFFFFFFFFFFFFFFFFFFFFFFFFD
:10031000FFFFFFFFFFFFFFFFFFFFFFFFFFFFFFFFED
:10032000FFFFFFFFFFFFFFFFFFFFFFFFFFFFFFFFDD
:10033000FFFFFFFFFFFFFFFFFFFFFFFFFFFFFFFFCD
:10034000FFFFFFFFFFFFFFFFFFFFFFFFFFFFFFFFBD
:10035000FFFFFFFFFFFFFFFFFFFFFFFFFFFFFFFFAD
:10036000FFFFFFFFFFFFFFFFFFFFFFFFFFFFFFFF9D
:10037000FFFFFFFFFFFFFFFFFFFFFFFFFFFFFFFF8D
:10038000FFFFFFFFFFFFFFFFFFFFFFFFFFFFFFFF7D
:10039000FFFFFFFFFFFFFFFFFFFFFFFFFFFFFFFF6D
:1003A000FFFFFFFFFFFFFFFFFFFFFFFFFFFFFFFF5D
:1003B000FFFFFFFFFFFFFFFFFFFFFFFFFFFFFFFF4D
:1003C000FFFFFFFFFFFFFFFFFFFFFFFFFFFFFFFF3D
:1003D000FFFFFFFFFFFFFFFFFFFFFFFFFFFFFFFF2D
:1003E000FFFFFFFFFFFFFFFFFFFFFFFFFFFFFFFF1D
:1003F000FFFFFFFFFFFFFFFFFFFFFFFFFFFFFFFF0D
:10040000FFFFFFFFFFFFFFFFFFFFFFFFFEFFFFFFFD
:1004100001F0FF01102A2BDB10F0070F08D010F8B5
:10042000013B013A8B422DD010F0070F42B3F6D1B9
:10043000F0B441EA012141EA014122F007047FF0D2
:1004400000070023F0E80256083C85EA010586EA29
:10045000010685FA47F5A3FA87F586FA47F6A5FA65
:1004600087F68EB9EED1F0BC01F0FF0102F0070271
:1004700032B110F8013B013A83EA010313B1F8D11C
:100480000020704701387047002D06BF35460338FD
:10049000073815F0010F07D1013015F4807F02BF36
:1004A000013015F4C03F0130F0BC0138704700BF87
:1004B000B0B586B000AF87ED030AC7ED020A87ED3D
:1004C000011AB8680EF0C2FF02460B4620A1D1E91E
:1004D00000010FF03DF902460B4614461D4697ED0C
:1004E000037AD7ED017A37EE677AD7ED036AD7ED55
:1004F000017A76EEE77A67EE277AB1EE677AD7ED82
:10050000027A77EEA76AD7ED027A66EEA77AC7EE8F
:10051000276AB0EE660A12F015F910EE103A184686
:100520000EF094FF02460B46204629460EF0E6FFE9
:1005300002460B46104619460FF0F2F903467B615E
:100540007B6907EE903AB0EE670A1837BD46B0BD3A
:100550002BF697DD9387D93F80B483B000AF7860E6
:100560001A4BD3F81031C3F38063DBB2002B17D0E2
:100570007B68DB889BB201339AB27B68DA807B6848
:10058000DB889BB24EF6602293428CBF012300238E
:10059000DBB2002B14D07B684FF47A72DA800FE064
:1005A0007B68DB889BB2142B8CBF01230023DBB25A
:1005B000002B02D07B6801229A727B680022DA80CD
:1005C00000BF0C37BD465DF8047B704700F00F405C
:1005D00080B582B000AF78607B68DB78DBB2002B3F
:1005E0000CBF01230023DBB2002B00F040817B68AD
:1005F0001B79DBB20133DAB27B681A717B681B7935
:10060000DBB2802B0CBF01230023DBB2002B02D016
:100610007B6800221A717B681B79DBB2002B0CBF50
:1006200001230023DBB2002B18D07B681B7ADBB2DE
:1006300083F00103DAB27B681A727B681B78DBB245
:10064000002B14BF01230023DBB2002B06D07B68F4
:100650001B78DBB2013BDAB27B681A707B681B79CE
:10066000DBB2402B0CBF01230023DBB2002B10D0E8
:100670007B681B78DBB2002B14BF01230023DBB2A5
:10068000002B06D07B681B78DBB2013BDAB27B68BB
:100690001A709C4AB2F8403043F40063A2F840302C
:1006A000984AB2F8403043F48063A2F840307B6847
:1006B0005B79DBB2934A03F00F03D9B2D2F88030F2
:1006C00061F34813C2F880307B685B8A9BB21A469C
:1006D0007B685B79DBB242FA03F303F00103002B82
:1006E00014BF01230023DBB2002B10D07B681B7AE0
:1006F000DBB283F00103DBB2824A03F00103D9B21B
:10070000B2F8403061F38A23A2F8403018E07B68E9
:100710001B8A9BB21A467B685B79DBB242FA03F311
:1007200003F00103002B14BF01230023DBB2002BD5
:1007300006D0744AB2F840306FF38A23A2F84030F2
:100740007B68DB7ADBB2002B30D07B685B79DBB275
:10075000082B0CBF01230023DBB2002B0FD07B68DA
:100760001B7ADBB283F00103DBB2664A03F00103BC
:10077000D9B2B2F8403061F38A23A2F840307B68E6
:100780005B79DBB20A2B0CBF01230023DBB2002B09
:100790000CD07B681B7ADBB25A4A03F00103D9B252
:1007A000B2F8403061F38A23A2F840307B68DB89DD
:1007B0009AB27B689B8A9BB213439BB21A467B68B2
:1007C0005B79DBB242FA03F303F00103002B14BFA1
:1007D00001230023DBB2002B06D04A4AB2F8403096
:1007E0006FF3CB23A2F840307B68DB8A9BB21A46BA
:1007F0007B685B79DBB242FA03F303F00103002B61
:1008000014BF01230023DBB2002B2DD07B681B7AA1
:10081000DBB283F00103DBB23A4A03F00103D9B241
:10082000B2F8403061F3CB23A2F840307B68DB891B
:100830009AB27B689B8A9BB213439BB21A467B6831
:100840005B79DBB242FA03F303F00103002B14BF20
:1008500001230023DBB2002B06D02A4AB2F8403035
:100860006FF3CB23A2F840307868FFF775FE7B6802
:10087000DB78DBB2022B0CBF01230023DBB2002BA1
:1008800000F08280204B5B68C3F38103DBB2032B53
:100890000CBF01230023DBB2002B1ED07B689B8A98
:1008A0009BB21A467B685B79DBB242FA03F303F032
:1008B0000103002B04D07B689B7EDBB2002B01D1AF
:1008C000012300E00023002B2AD00E4AB2F840306A
:1008D00043F40063A2F8403022E07B68DB899BB2DE
:1008E0001A467B685B79DBB242FA03F303F001033B
:1008F000002B04D17B689B7EDBB2002B06D1012349
:1009000005E000BF00F00F40F40100200023002BA1
:1009100006D08C4AB2F8403043F40063A2F840306D
:100920007B68DB8A9BB21A467B685B79DBB242FA52
:1009300003F303F00103002B13D07B689B8A9AB268
:100940007B68DB899BB213439BB21A467B685B7959
:10095000DBB242FA03F303F00103002B01D00123C1
:1009600000E00023002B0FD07B681B7ADBB283F002
:100970000103DBB2734A03F00103D9B2B2F840308D
:1009800061F3CB23A2F840307B681B78DBB2002BED
:1009900014BF01230023DBB2002B00F0A6807B688C
:1009A0005B79DBB21A467B685B78DBB2013B9A422B
:1009B0000CBF01230023DBB2002B43D07B681B78E4
:1009C000DBB2082B0CBF01230023DBB2002B06D0C7
:1009D0005C4AB2F840306FF38A23A2F840307B685B
:1009E0001B78DBB2062B0CBF01230023DBB2002BEC
:1009F00006D0544AB2F8403043F48063A2F8403045
:100A00007B681B78DBB2042B0CBF01230023DBB215
:100A1000002B06D04B4AB2F840306FF38A23A2F87D
:100A200040307B681B78DBB2022B0CBF0123002314
:100A3000DBB2002B06D0434AB2F8403043F4806367
:100A4000A2F840307B685B79DBB21A467B689B7802
:100A5000DBB2013B9A420CBF01230023DBB2002B27
:100A600043D07B681B78DBB2072B0CBF012300232C
:100A7000DBB2002B06D0334AB2F840306FF3CB2301
:100A8000A2F840307B681B78DBB2052B0CBF01233A
:100A90000023DBB2002B06D02A4AB2F8403043F4E0
:100AA0000063A2F840307B681B78DBB2032B0CBFDD
:100AB00001230023DBB2002B06D0224AB2F84030DB
:100AC0006FF3CB23A2F840307B681B78DBB2012B9D
:100AD0000CBF01230023DBB2002B06D0194AB2F869
:100AE000403043F40063A2F840307B68DB78DBB22F
:100AF000072B0CBF01230023DBB2002B0ED07B6839
:100B00005B79DBB20133DAB27B685A717B685B795F
:100B1000DBB203F00F03DAB27B685A717B68DB78D3
:100B2000DBB20133DAB27B68DA707B68DB78DBB288
:100B300003F00703DAB27B68DA7000BF0837BD46FE
:100B400080BD00BF00F00F4080B485B000AF78607A
:100B5000554AB2F840306FF38A23A2F84030524A27
:100B6000B2F8403043F40063A2F840300023FB8128
:100B7000FB899BB20F2B94BF01230023DBB2002B18
:100B800037D0FB899BB2484A03F00F03D9B2D2F8A1
:100B9000803061F34813C2F880300023BB81BB89E9
:100BA0009BB240F28F12934294BF01230023DBB229
:100BB000002B18D000237B817B899BB240F28F12DF
:100BC000934294BF01230023DBB2002B05D07B8925
:100BD0009BB201339BB27B81EEE7BB899BB20133B1
:100BE0009BB2BB81DBE7FB899BB201339BB2FB81EC
:100BF000BEE72D4AB2F8403043F48063A2F840309B
:100C0000294AB2F840306FF3CB23A2F840300023DA
:100C1000FB81FB899BB20F2B94BF01230023DBB226
:100C2000002B3BD0FB899BB2DBB2C3F10F03DBB2DD
:100C30001D4A03F00F03D9B2D2F8803061F3481394
:100C4000C2F880300023BB81BB899BB240F28F1277
:100C5000934294BF01230023DBB2002B18D0002362
:100C60007B817B899BB240F28F12934294BF012318
:100C70000023DBB2002B05D07B899BB201339BB2F2
:100C80007B81EEE7BB899BB201339BB2BB81DBE783
:100C9000FB899BB201339BB2FB81BAE700BF1437DB
:100CA000BD465DF8047B704700F00F4080B582B010
:100CB00000AF78600A4BB3F840207B685A807B68AD
:100CC0005A887B681B889A4202D0786800F01AF82C
:100CD0007B685A887B681A8000BF0837BD4680BD94
:100CE000A001002080B483B000AF7860044BB3F85B
:100CF000403018460C37BD465DF8047B704700BF96
:100D0000A001002080B586B000AF78607B685B886A
:100D1000BB827B685A887B681B8853409BB27B826E
:100D20000023FB75FB7D0F2B00F2E9817B8A9BB2D0
:100D300003F00103002B14BF01230023DBB2002BBF
:100D400000F0CF81FB7D03F00F03DAB23B7B62F34F
:100D500003033B73BB8A9BB203F00103DAB23B7B14
:100D600062F304133B733B7B6FF345133B733B7B95
:100D70006FF386133B733B7B6FF3C7133B73A14B3E
:100D80001B78DBB20E2B14BF01230023DBB2002B38
:100D900000F097819C4B1B69C3F34333DBB2042BF8
:100DA00000F0E980042B00F38581022B02D0032B95
:100DB0007CD07FE13B7BC3F30303DBB2022B4CD03F
:100DC000022B00F38981002B02D0012B22D083E17A
:100DD0003B7B03F01003DBB2002B61D0894A13790F
:100DE0006FF383031371874B5B68C3F38103DBB23B
:100DF0001A46864B1A70864B0022DA813B7BC3F37E
:100E00000303DBB20133DBB21A460221804811F042
:100E100008FA45E03B7B03F01003DBB2002B41D026
:100E2000784A1379012161F383031371754B5B6871
:100E3000C3F38103DBB21A46744B1A70744B002261
:100E4000DA813B7BC3F30303DBB20133DBB21A4627
:100E500002216F4811F0E5F924E03B7B03F0100319
:100E6000DBB2002B20D0674A1379022161F38303A0
:100E70001371644B5B68C3F38103DBB21A46634BA7
:100E80001A70634B0022DA813B7BC3F30303DBB2AE
:100E90000133DBB21A4602215D4811F0C2F903E0CA
:100EA00000BF19E100BF17E100BF15E13B7BC3F3B1
:100EB0000303DBB2022B40D0022B00F30F81002B87
:100EC00002D0012B1CD009E14E4A13796FF3830342
:100ED00013714C4B5B68C3F38103DBB21A464B4B77
:100EE0005A704B4B0022DA813B7BC3F30303DBB226
:100EF0000133DBB21A460321454811F092F939E07B
:100F0000404A1379012161F3830313713D4B5B6800
:100F1000C3F38103DBB21A463C4B5A703C4B0022B0
:100F2000DA813B7BC3F30303DBB20133DBB21A4646
:100F30000321374811F075F91CE0324A1379022178
:100F400061F3830313712F4B5B68C3F38103DBB23F
:100F50001A462E4B5A702E4B0022DA813B7BC3F38C
:100F60000303DBB20133DBB21A460321284811F038
:100F700058F900BFB2E03B7BC3F30303DBB2022BA3
:100F800048D0022B00F3AC80002B02D0012B1CD0E8
:100F9000A6E01C4A13796FF383031371194B5B6846
:100FA000C3F38103DBB21A46184B9A70184B002228
:100FB000DA813B7BC3F30303DBB20133DBB21A46B6
:100FC0000421134811F02DF973E00E4A1379012121
:100FD00061F3830313710B4B5B68C3F38103DBB2D3
:100FE0001A460A4B9A700A4B0022DA813B7BC3F304
:100FF0000303DBB20133DBB21A460421044811F0CB
:1010000010F956E0F401002000F00F40F405002034
:10101000C01D00203C4B1B78DBB20B2B0CBF012307
:101020000023DBB2002B28D0374A137943F00C039E
:101030001371354B5B68C3F38103DBB21A46334B44
:101040009A70314A13796FF3041313712E4A13798E
:101050006FF3471313712E4B01229A762C4B072204
:10106000DA813B7BC3F30303DBB20133DBB21A4605
:101070000421274811F0D5F81BE0234A13796FF3B8
:1010800083031371204B5B68C3F38103DBB21A4601
:101090001E4B9A701E4B0022DA813B7BC3F3030385
:1010A000DBB20133DBB21A460421194811F0B9F85A
:1010B00000BF15E07B689B68F968184610F00DFECC
:1010C0000FE0144B1B69C3F343337B689B68F968DB
:1010D000184610F002FE04E000BF02E000BF00E08E
:1010E00000BF7B8A9BB25B109BB27B82BB8A9BB2A8
:1010F0005B109BB2BB82FB7D0133FB7512E600BF28
:101100001837BD4680BD00BFF4010020F405002063
:10111000C01D002000F00F4080B483B000AF7860A5
:101120000B46FB701346BB70BB78032B32D801A271
:1011300052F823F045110000591100006D11000014
:1011400081110000FB7803F00F03D9B2144A137821
:1011500061F3030313701DE0FB7803F00F03D9B2B2
:101160000F4A137861F30713137013E0FB7803F051
:101170000F03D9B20A4A537861F30303537009E0AD
:10118000FB7803F00F03D9B2054A537861F30713D4
:10119000537000BF00BF0C37BD465DF8047B70473D
:1011A000E401002080B483B000AF78600B46FB7090
:1011B0001346BB70BB78032B32D801A252F823F040
:1011C000D1110000E5110000F91100000D1200001E
:1011D000FB7803F00103D9B2144A937861F300035A
:1011E00093701DE0FB7803F00103D9B20F4A9378A6
:1011F00061F34103937013E0FB7803F00103D9B26C
:101200000A4A937861F38203937009E0FB7803F054
:101210000103D9B2054A937861F3C303937000BF09
:1012200000BF0C37BD465DF8047B7047E401002029
:1012300080B483B000AF78600B46FB701346BB7080
:101240007B68FA7883F824207B68BA7883F82520B5
:101250007B6893F82430DBB21A467B6893F825301C
:10126000DBB218467B681C499200024451F82220E8
:101270005A617B681B7D03F00703DBB2012B0CD1A5
:101280007B681B7D03F00803DBB2002B05D07B6875
:10129000DB7CDAB27B689A7417E07B681B7DC3F352
:1012A0000203DBB21A467B68DB7CDBB29A4206DAC9
:1012B0007B681B7DC3F30203DBB21A4602E07B6846
:1012C000DB7CDAB27B689A7400BF00BF0C37BD4686
:1012D0005DF8047B704700BF2C53010090B585B0CA
:1012E00000AF78600B46FB707B687A6852699A6140
:1012F000994B1B78DBB2092B08D17B681B7E03F06E
:101300000703DBB2042B01D1012300E00023002BF3
:101310000ED07A68137E43F0080313767A68537E02
:1013200043F0010353767A68137E43F0100313767B
:101330007B685B7E03F00103DBB2002B23D17B686B
:101340005B7CDBB21A467B681B7EC3F30203DBB215
:1013500019467B68DB7CDBB2994205DA7B681B7E31
:10136000C3F30203DBB202E07B68DB7CDBB29342B7
:1013700094BF01230023DBB2002B01D00023FCE14A
:101380007B6800221A747B681B7E03F04003DBB28B
:10139000002B3AD07B681B6A184610F005FE034606
:1013A00003F00F03D9B27A68137861F30303137063
:1013B0007B681B6A184610F0C9FD034603F00F0353
:1013C000D9B27A68137961F3030313717A681378D9
:1013D00043F0100313707A68137943F0100313710C
:1013E00000220021786810F09BFF0122012178681B
:1013F00010F096FF786810F0B9FF7B6802225A74EB
:10140000786800F0BFF90123B7E17B689B7CDAB212
:101410007B681B7CDBB29A4294BF01230023DBB2C2
:10142000002B02D07B6800221A747B685B7CDAB2E6
:101430007B689B7CDBB29A422CBF01230023DBB28A
:10144000002B54D00023FB737B689B7CDBB2FA7BC0
:101450009A4234BF01230023DBB2002B7ED07B688D
:101460001B7CDBB21A467B6853F82230C3F30303BC
:10147000DBB21C467B681A6A7B681B7EC3F30203DF
:10148000DBB219467B68DB7CDBB2994205DA7B680C
:101490001B7EC3F30203DBB202E07B68DB7CDBB2C2
:1014A0001946104610F035FD03469C4214BF012337
:1014B0000023DBB2002B16D07B681B7CDBB2013330
:1014C000DAB27B681A747B689B7CDAB27B681B7C1F
:1014D000DBB29A4294BF01230023DBB2002B02D07F
:1014E0007B6800221A74FB7B0133FB73ACE700239B
:1014F000BB737B689B7CDBB2BA7B9A4234BF01230F
:101500000023DBB2002B29D07B681B7CDBB21A46A0
:101510007B6853F82230C3F30013DBB2002B16D0E4
:101520007B681B7CDBB20133DAB27B681A747B68A0
:101530009B7CDAB27B681B7CDBB29A4294BF0123AE
:101540000023DBB2002B02D07B6800221A74BB7B25
:101550000133BB73CDE700BFF40100207B681B7E25
:1015600003F01003DBB2002B23D000237B737B68D6
:101570009B7CDBB27A7B9A4234BF01230023DBB22F
:10158000002B16D07A7B7B6853F82230C3F3030319
:10159000DBB21A46FB789A420CBF01230023DBB270
:1015A000002B02D07B687A7B1A747B7B01337B73C0
:1015B000DDE77B681B7EC3F30203DBB21A467B6860
:1015C000DB7CDBB29A4206DA7B681B7EC3F3020344
:1015D000DBB21A4603E07B68DB7CDBB21A467B6831
:1015E0009B7CDBB29A4214BF01230023DBB2002BA9
:1015F00029D000233B737B689B7CDBB23A7B9A4209
:1016000034BF01230023DBB2002B1CD07B681B7C82
:10161000DBB23A7B9A4214BF01230023DBB2002BDA
:101620000DD0397B7A6812F821306FF3041302F879
:1016300021303B7B1A4600217868FFF7B3FD3B7BE6
:1016400001333B73D7E77B685B7E03F00203DBB2B9
:10165000002B0FD07B68FA781A747B681B7CDBB296
:10166000032B8CBF01230023DBB2002B02D07B684D
:1016700003221A747B681B7CDBB21946FB7803F0EB
:101680000F03D8B27A6812F8213060F3030302F82E
:1016900021307B681B7CDBB219467A6812F8213056
:1016A00043F0100302F821307B681B7CD9B27B68C1
:1016B0001B7CDBB21A46786810F032FE786810F0B6
:1016C00055FE7B681B7E03F00803DBB2002B16D0AF
:1016D0007B681B7CDBB20133DAB27B681A747B68EF
:1016E0009B7CDAB27B681B7CDBB29A4294BF0123FD
:1016F0000023DBB2002B02D07B6800221A747B68C7
:101700005B7CDBB20133DAB27B68114659747B68CB
:101710001B7EC3F30203DBB219467B68DB7CDBB2C2
:10172000994205DA7B681B7EC3F30203DBB202E059
:101730007B68DB7CDBB2934234BF01230023DBB246
:10174000002B16D07B681B7EC3F30203DBB21A4664
:101750007B68DB7CDBB29A4206DA7B681B7EC3F3D4
:101760000203DBB21A4602E07B68DB7CDAB27B68FC
:101770005A74786800F006F8012318461437BD46FD
:1017800090BD00BF80B485B000AF7860814B1B78FE
:10179000DBB20B2B0CBF01230023DBB2002B3ED0AE
:1017A0007B681B7F002B02D07B4B00229A82002398
:1017B000FB737B68DB7CDBB2FA7B9A4234BF01238C
:1017C0000023DBB2002B69D0FA7B7B6853F8223010
:1017D000C3F30013DBB2012B05D17B681B7F002B09
:1017E00001D0012300E00023002B14D0FA7B7B689A
:1017F00053F82230C3F30303DBB21A46012303FA82
:1018000002F1654B9B8A9BB21AB20BB213431BB217
:101810009AB2614B9A82FB7B0133FB73C9E77B6809
:101820001B7F002B02D05C4B0022DA810023BB73AC
:101830007B68DB7CDBB2BA7B9A4234BF0123002396
:10184000DBB2002B2AD0BA7B7B6853F82230C3F37B
:101850000013DBB2012B05D17B681B7F002B01D06D
:10186000012300E00023002B14D0BA7B7B6853F8DF
:101870002230C3F30303DBB21A46012303FA02F159
:10188000454BDB899BB21AB20BB213431BB29AB21F
:10189000414BDA81BB7B0133BB73C9E73D4B5B68CE
:1018A000C3F38103DBB2032B0CBF01230023DBB2A4
:1018B000002B68D07B681B7F002B02D0364B0722A1
:1018C000DA817B681B7F002B02D0334B00229A8287
:1018D00000237B737B68DB7CDBB27A7B9A4234BF6C
:1018E00001230023DBB2002B4DD07A7B7B6853F8B9
:1018F0002230C3F30013DBB2002B40D07A7B7B682D
:1019000053F82230C3F30303DBB2022B05D97B6803
:101910001B7F002B01D0012300E00023002B15D0FA
:101920007A7B7B6853F82230C3F30303DBB21A4699
:10193000012303FA02F1184BDB899BB21AB20BB2F6
:1019400013431BB29AB2144BDA8118E07B681B7FF9
:10195000002B14D07A7B7B6853F82230C3F3030347
:10196000DBB21A46012303FA02F10B4B9B8A9BB2AE
:101970001AB20BB213431BB29AB2074B9A827B7B0B
:1019800001337B73A6E700BF1437BD465DF8047BC7
:10199000704700BFF4010020C01D002080B483B058
:1019A00000AF78607A6892F82420D2B202F0030285
:1019B000D2B262F301037A6892F82520D2B202F023
:1019C0000302D2B262F38303094A5268C2F30012DF
:1019D000D2B262F30413064A5268C2F34212D2B280
:1019E00062F3471318460C37BD465DF8047B704719
:1019F000F401002080B584B000AF7860396007F151
:101A00000C03042219460A4812F0EBFDFB68396802
:101A10007A688A1AB3FBF2F102FB01F29A1A7B6828
:101A20001344FB60FB6818461037BD4680BD00BFFD
:101A30000090024080B598B000AF0346FB800023C1
:101A400087F85F300023BB6407F14C0300221A6063
:101A50005A609A60002387F85E30002387F85D3073
:101A60004FF00003BB6507F1080340220021184630
:101A700013F0DDF9FB88002B00F0BF80FB88002B02
:101A80001ED0FB8803F00103002B10D097F85F30C5
:101A9000013387F85F3097F85D305A1C87F85D2076
:101AA00007F16002134497F85E2003F8182CFB88B6
:101AB0005B10FB8097F85E30013387F85E30DDE71E
:101AC000002387F85E3097F85E2097F85F309A42DF
:101AD0004ED2002387F85D3097F85D300F2B41D848
:101AE00097F85D3007EE903AB8EE677A97F85F3076
:101AF000C3F110034D4A9B001344D3ED007AB0EEBE
:101B0000006AC7EE866A97F85E3007F160021344F8
:101B100013F8183C07EE903AF8EE677AB0EE671AC1
:101B2000F0EE660AB0EE470AFEF7C2FCB0EE407A6D
:101B300097F85D309B0007F160021344583BD3EDEA
:101B4000007A97F85D3077EE277A9B0007F1600204
:101B50001344583BC3ED007A97F85D30013387F8A2
:101B60005D30B9E797F85E30013387F85E30AAE759
:101B7000002387F85D3097F85D300F2B14D897F865
:101B80005D309B0007F160021344583BD3ED007AAF
:101B900097ED167A77EE277AC7ED167A97F85D30CB
:101BA000013387F85D30E6E7DFED216A97ED167ABD
:101BB000C6EE877AC7ED167A002387F85D3097F86E
:101BC0005D300F2B2DD897F85D309B0007F1600238
:101BD0001344583B93ED007A97F85D30D7ED167AB1
:101BE00067EE277A134A9B001344C3ED007A97F8F7
:101BF0005D30013387F85D30E1E7002387F85D3021
:101C000097F85D300F2B0CD897F85D30094A9B0090
:101C10001344094A1A6097F85D30013387F85D3044
:101C2000EEE700BF6037BD4680BD00BFA0000020CA
:101C30000000C642600000200000C84080B588B0A7
:101C400000AFF860B9601346FB710023FB764FF0DC
:101C500000037B61FB79002B34D064210020FFF767
:101C6000C9FE03463B613B6907EE903AF8EE677A9E
:101C700097ED057AB4EEE77AF1EE10FA12D5FB7E15
:101C80005A1CFA76154A9B001344D3ED007A97ED5F
:101C9000057A77EE277AC7ED057AFB7E0F2B00D801
:101CA000E1E700BFFB7E013BB968FA688A1A02FBD4
:101CB00003F3002B00DA0F331B111A46FB681344A1
:101CC000FB6105E0B968F868FFF794FE0346FB6125
:101CD000FB6918462037BD4680BD00BF600000206C
:101CE00080B485B000AF78600B46FB707B689B7C4E
:101CF000DAB27B6893F86630DBB29A4234BF0123D4
:101D00000023DBB2002B36D07B689B7CDBB2013337
:101D1000DAB27B689A747B689B7CFB73FB7B002B3D
:101D20000BD0FB7B5A1EFB7B79688A5CD1B27A6848
:101D3000D154FB7B013BFB73F0E77B68FA781A70A8
:101D40007B68B3F864309BB21AB2FB78012101FAC8
:101D500003F31BB213431BB29AB27B68A3F864204F
:101D60007B6893F86830002B05D07B68B3F864304B
:101D70009AB2044B9A8200BF1437BD465DF8047BCB
:101D8000704700BFC01D002080B485B000AF7860F0
:101D90000B46FB700023FB737B689B7CDBB2FA7BFA
:101DA0009A4234BF01230023DBB2002B41D0FB7BDE
:101DB0007A68D35CDBB2FA789A420CBF0123002325
:101DC000DBB2002B31D0FB7BBB737B689B7CDBB22F
:101DD000BA7B9A4234BF01230023DBB2002B0BD025
:101DE000BB7B5A1CBB7B79688A5CD1B27A68D154C0
:101DF000BB7B0133BB73E8E77B689B7CDBB2013BB9
:101E0000DAB27B689A747B68B3F864309BB21AB21A
:101E1000FB78012101FA03F31BB2DB431BB2134031
:101E20001BB29AB27B68A3F86420FB7B0133FB737F
:101E3000B2E77B6893F86830002B05D07B68B3F875
:101E400064309AB2034B9A8200BF1437BD465DF8E6
:101E5000047B7047C01D002080B584B000AF78605F
:101E60000B46FB707B68DB7CDBB283F00103DBB2EB
:101E7000002B05D0FB7819467868FFF731FF01E1A8
:101E8000FB781946786810F037FF0346002B0CBF2B
:101E900001230023DBB2002B00F0B3807B6893F8B2
:101EA00069301A461346DB0013445B0013441833B1
:101EB0007A6813440633FA78114618460FF08FFFFC
:101EC0007B6893F869301A461346DB0013445B00C5
:101ED000134418337A681344063318460FF0FDFF95
:101EE00003461A467B6893F86630DBB29A428CBF91
:101EF00001230023DBB2002B7DD07B6893F8663092
:101F0000FB737B6893F869301A461346DB00134471
:101F10005B00134418337A681344063318460FF0F5
:101F2000DCFF03461A46FB7B934234BF01230023A8
:101F3000DBB2002B4AD07B6893F869301A4613460F
:101F4000DB0013445B00134418337A6813440633F0
:101F5000FA7B114618460FF0DCFF034619467868F5
:101F6000FFF712FF7B6893F869301A461346DB00CF
:101F700013445B00134418337A6813440633FA7B26
:101F8000114618460FF0C5FF03461A460123934039
:101F900083F47F4383F0FF037A6892F86920114647
:101FA0007A680C3132F8112092B212B21BB213408F
:101FB00019B27B6893F869301A4689B27B680C3293
:101FC00023F81210FB7B0133FB739AE77B6893F8CD
:101FD00069301A461346DB0013445B001344183380
:101FE0007A6813449A1D7B6893F86630DBB2194611
:101FF00010460FF07FFFFB7819467868FFF770FEF8
:1020000016E07B6893F869301A461346DB001344E8
:102010005B00134418337A6813440633FA78114688
:1020200018460FF011FFFB7819467868FFF7ACFEF1
:102030007B6893F869301A467B680C3233F81230AB
:102040009BB21AB2FB78012101FA03F31BB2534091
:1020500019B27B6893F869301A4689B27B680C32F2
:1020600023F812107B6893F86830002B0AD07B6845
:1020700093F869301A467B680C3233F812309AB202
:10208000024B9A8200BF1037BD4680BDC01D0020A4
:1020900090B587B002AF78600B46FB701346BB70FB
:1020A0007B689B7CDBB2002B0CBF01230023DBB2DF
:1020B000002B0CD0BB78052B00F0ED81F978BB78B4
:1020C00000930F230022786810F072FCE3E1BB78E4
:1020D000013B042B00F2DF8101A252F823F000BF84
:1020E000F52000001F2100008722000029230000A6
:1020F000C92300007B689B7CDBB2002219460020CC
:10210000FFF79CFD0346DBB21946FB787A68525C08
:10211000D1B27A6813440A4683F85720BBE17B6842
:102120009B7CDBB2012B8CBF01230023DBB2002B95
:1021300072D00023FB73FB7B0F2B78D87B68B3F83E
:1021400064309BB21946FB787A68134493F8573091
:10215000DBB21A4601239340013B0B40002B0CBF1E
:1021600001230023DBB2002B05D0FB787A681344EF
:10217000012283F85F207B68B3F864309BB2194674
:10218000FB787A68134493F85730DBB201330122AD
:1021900002FA03F3013B83F47F4383F0FF030B4018
:1021A000002B0CBF01230023DBB2002B05D0FB78F2
:1021B0007A681344FF2283F85F20FB787A6813441F
:1021C00093F85F3058B2FB787A68134493F857302D
:1021D000D9B2C2B2FB780A44D1B27A6813440A4633
:1021E00083F857207B68B3F864309BB21946FB78BC
:1021F0007A68134493F85730DBB241FA03F303F0E3
:102200000103002B14BF01230023DBB2002B0DD1EF
:10221000FB7B0133FB738EE7FB787A681278D1B2CF
:102220007A6813440A4683F8572000E000BF7B68B1
:1022300093F86730DBB2002B00F02681FB787A68D8
:10224000134493F85F305BB2012B0CBF01230023D2
:10225000DBB2002B0BD07B68FC7818460FF0A4FE95
:1022600003461A467B68234483F857200CE17B68B9
:10227000FC7818460FF06AFE03461A467B68234432
:1022800083F8572000E1FB787A681344FF2283F833
:102290005F200023BB73BB7B0F2B32D8FB787A689F
:1022A0001A4492F85720D2B2013AD1B27A68134454
:1022B0000A4683F85720FB7850337A681344073373
:1022C0001A78D2B202F00F02D2B21A707B68B3F859
:1022D00064309BB21946FB787A68134493F8573000
:1022E000DBB241FA03F303F00103002B14BF012317
:1022F0000023DBB2002B03D1BB7B0133BB73CAE7E6
:1023000000BF7B6893F86730DBB2002B00F0BE8023
:102310007B68FC7818460FF019FE03461A467B6866
:10232000234483F85720B1E0FB787A6813440122F4
:1023300083F85F2000237B737B7B0F2B32D8FB78E5
:102340007A681A4492F85720D2B20132D1B27A6830
:1023500013440A4683F85720FB7850337A681344B5
:1023600007331A78D2B202F00F02D2B21A707B6829
:10237000B3F864309BB21946FB787A68134493F83B
:102380005730DBB241FA03F303F00103002B14BF13
:1023900001230023DBB2002B03D17B7B01337B7352
:1023A000CAE700BF7B6893F86730DBB2002B6FD0C1
:1023B0007B68FC7818460FF0F7FD03461A467B68E9
:1023C000234483F8572063E0FB787A68134493F83A
:1023D0005B30DBB2002B0AD0FB787A68134493F8A9
:1023E0005B30DAB27B689B7CDBB29A4201D301237B
:1023F00000E00023002B08D0FB787A68927CD1B2F1
:102400007A6813440A4683F85B20FB787A681A449A
:1024100092F85B20D2B2013AD1B27A6813440A46EC
:1024200083F85B20FB787A68134493F85B30DBB267
:102430001946FB787A68525CD1B27A6813440A462E
:1024400083F857207B6893F86730DBB2002B21D0EC
:102450007B689B7CDAB2FB78013AD1B27A6813448C
:102460000A4683F85B20FB787A68134493F85B3064
:10247000DBB21946FB787A68525CD1B27A681344B1
:102480000A4683F8572005E000BF04E000BF02E0E1
:1024900000BF00E000BF00BF1437BD4690BD00BFC5
:1024A00090B587B002AF78600B46FB701346BB70E7
:1024B0007B689B7CDBB2032B00F2418101A252F8C6
:1024C00023F000BFD524000031250000B325000013
:1024D00027260000B978FB7800930F230022786844
:1024E00010F066FA0023FB73FB7B032B00F22281C2
:1024F000FA7BBB789A4217D0BA78FB7B79680A449A
:1025000092F85720D1B27A6813440A4683F85720CC
:10251000BA78FB7B79680A4492F85F2051B27A68F6
:1025200013440A4683F85F20FB7B0133FB73DBE730
:10253000BB7803F00103002B0ED17B6818460FF027
:1025400005FD03461A46B978FB780093134600222E
:10255000786810F02DFA0DE07B6818460FF0F6FC55
:1025600003460133DAB2B978FB7800930F23786819
:1025700010F01EFABB78BA7882F00202D2B211468D
:102580007A68134493F85730DAB27B680B4483F8C7
:102590005720BB78BA7882F00202D2B211467A682C
:1025A000134493F85F305AB27B680B4483F85F2082
:1025B000C5E07B6818460FF0F7FC03461C467B68B5
:1025C00018460FF0C3FC03461A46B978FB7800930F
:1025D00013462246786810F0EBF90023BB73BB7BEF
:1025E000032B00F2A980BA7BBB789A4217D0BA7845
:1025F000BB7B79680A4492F85720D1B27A681344B9
:102600000A4683F85720BA78BB7B79680A4492F867
:102610005F2051B27A6813440A4683F85F20BB7B7F
:102620000133BB73DBE7BB78032B00F2878001A289
:1026300052F823F045260000632600008D26000096
:10264000EB2600007B6818460FF0AEFC03461A46E6
:10265000B978FB78009313460022786810F0A8F947
:1026600067E07B6818460FF09FFC03460133DCB23D
:10267000786810F050F903461A46B978FB78009351
:1026800013462246786810F093F952E07B681846AA
:102690000FF05CFC03460E2B94BF01230023DBB23A
:1026A000002B14D0786810F036F903460133DCB201
:1026B0007B6818460FF04AFC03461A46B978FB7847
:1026C000009313462246786810F072F931E078687A
:1026D00010F021F903460133DAB2B978FB780093A0
:1026E0000E23786810F064F923E07B6818460FF039
:1026F0002DFC03460E2B94BF01230023DBB2002BDD
:102700000ED07B6818460FF021FC03460133DAB285
:10271000B978FB7800930F23786810F049F90DE041
:10272000B978FB7800930F230F22786810F040F9F6
:1027300004E003E000BF02E000BF00E000BF7B68F0
:1027400093F86730DBB2002B03D07B68002283F85C
:10275000672000BF1437BD4690BD00BF90B585B05F
:1027600002AF78600B46FB707B6893F86930012BF1
:1027700040F024817B689B7CDBB2032B00F2248138
:1027800001A252F823F000BF99270000FF270000A4
:1027900071280000EF280000FB7800930F2300222F
:1027A0000021786810F004F97B6893F85730DAB2AA
:1027B0007B6883F858207B6893F85730DAB27B68DF
:1027C00083F859207B6893F85730DAB27B6883F836
:1027D0005A207B6893F85F305AB27B6883F8602098
:1027E0007B6893F85F305AB27B6883F861207B681E
:1027F00093F85F305AB27B6883F86220E4E07B682C
:1028000018460FF0A3FB03461A46FB7800931346C5
:1028100000220021786810F0CBF87B6818460FF092
:1028200095FB03460133DAB2FB7800930F230121B5
:10283000786810F0BDF87B6893F85730DAB27B689F
:1028400083F859207B6893F85830DAB27B6883F8B4
:102850005A207B6893F85F305AB27B6883F8612016
:102860007B6893F860305AB27B6883F86220ABE0F3
:102870007B6818460FF098FB03461C467B68184699
:102880000FF064FB03461A46FB780093134622467A
:102890000021786810F08CF87B6893F85730DAB232
:1028A0007B6883F858207B6893F85730DAB27B68EE
:1028B00083F859207B6893F85730DAB27B6883F845
:1028C0005A207B6893F85F305AB27B6883F86020A7
:1028D0007B6893F85F305AB27B6883F861207B682D
:1028E00093F85F305AB27B6883F862206CE07B68B3
:1028F00018460FF059FB03461A46FB78009313461F
:1029000000220021786810F053F87B6818460FF019
:102910004BFB03460133DCB278680FF0FCFF034643
:102920001A46FB780093134622460121786810F07E
:102930003FF87B6818460FF009FB03460E2B94BF47
:1029400001230023DBB2002B22D078680FF0E3FFD5
:1029500003460133DCB27B6818460FF0F7FA0346F2
:102960001A46FB780093134622460221786810F03D
:102970001FF87B6818460FF0E9FA03460133DAB214
:10298000FB7800930F230321786810F011F81BE007
:1029900078680FF0C0FF03460133DAB2FB7800938A
:1029A0000E230221786810F003F8FB7800930F23C0
:1029B0000F22032178680FF0FBFF05E0FB781A4631
:1029C00000217868FFF764FB7B6893F86730DBB21F
:1029D000002B03D07B68002283F8672000BF0C37F0
:1029E000BD4690BD90B585B000AF78607B68DB7C5C
:1029F000DBB2002B0CBF01230023DBB2002B00F065
:102A0000A2807B680122DA747B689B7CDBB2002B9E
:102A100014BF01230023DBB2002B4AD0786810F0EA
:102A20004AF97B689B7CFB73FB7B002B00F08B805F
:102A30007B6893F869301A461346DB0013445B0049
:102A4000134418337A6813449C1D7A68FB7B013B5E
:102A5000DBB2194610460FF05CFA034619462046D1
:102A60000FF0BDF97A68FB7B013BDBB219461046DB
:102A70000FF04FFA03461A46012303FA02F17B686E
:102A800093F869301A467B680C3233F812309BB2E7
:102A90001AB20BB2134319B27B6893F869301A4625
:102AA00089B27B680C3223F81210FB7B013BFB736D
:102AB000BAE77B6893F869301A461346DB00134483
:102AC0005B00134418337A681344063318460FF03A
:102AD00004FA0346002B14BF01230023DBB2002BB2
:102AE00031D07B6893F869301A461346DB001344F3
:102AF0005B00134418337A681344063318460FF00A
:102B0000ECF90346BB73BB7B002B1CD07B6893F8AE
:102B100069301A461346DB0013445B001344183334
:102B20007A6813449A1DBB7B013BDBB21946104601
:102B30000FF0EFF9034619467868FFF7D1F8BB7B31
:102B4000013BBB73DFE77B6893F86830002B0AD04A
:102B50007B6893F869301A467B680C3233F8123080
:102B60009AB2034B9A8200BF1437BD4690BD00BF96
:102B7000C01D002090B585B000AF78607B68DB7C1D
:102B8000DBB2012B0CBF01230023DBB2002B59D099
:102B90007B6893F869301A461346DB0013445B00E8
:102BA000134418337A681344063318460FF095F926
:102BB0000346FB73FB7B002B41D02848FEF792F8BD
:102BC00003461C467B6893F869301A461346DB00BF
:102BD00013445B00134418337A6813449A1DFB7B3B
:102BE000013BDBB2194610460FF093F9034644FA55
:102BF00003F303F00103002B0CBF01230023DBB21E
:102C0000002B18D07B6893F869301A461346DB0016
:102C100013445B00134418337A6813449A1DFB7BFA
:102C2000013BDBB2194610460FF073F90346194613
:102C30007868FFF7A9F8FB7B013BFB73BAE77B6879
:102C40000022DA747B6893F86830002B02D0044BC2
:102C500000229A8200BF1437BD4690BD601E00203E
:102C6000C01D0020B0B584B000AF78607B681E3313
:102C700018460FF032F903463B733B7B002B46D0DE
:102C80000023FB73FA7B3B7B9A4240D2FB7B03F031
:102C90000103002B1BD17B6803F11E003A7BFB7BF9
:102CA000D31ADBB2013BDBB219460FF032F903460F
:102CB0001A46FB7B5B1002F00F02D1B2584A023376
:102CC0009B0013441A7961F303021A711BE07B68BD
:102CD00003F11E003A7BFB7BD31ADBB2013BDBB274
:102CE00019460FF016F903461A46FB7B013B5B10B1
:102CF00002F00F02D1B24A4A02339B0013441A7900
:102D000061F307121A71FB7B0133FB73BAE7444A84
:102D10003B7B82F82C307B6893F869309AB2404B49
:102D20001A867B68DB7CDAB23D4B83F854230023A0
:102D3000BB73BB7B022B6ED8BA7BBB7B79680A4422
:102D4000127DD1B2364A13440A4683F85523B97B23
:102D5000BB7B7A680C3132F8112091B2304A03F50E
:102D6000D4735B0013440A461A8100237B737B7B78
:102D7000102B1ED8B97B7C7BBA7B787B7D680B4699
:102D8000DB000B445B000B442B4423441E331B78B5
:102D9000DCB223491346DB0013445B0013440B44AD
:102DA000034403F25E3322461A707B7B01337B734C
:102DB000DDE7B97BBA7B78680B46DB000B445B0030
:102DC0000B4403442F331B78D8B215491346DB005C
:102DD00013445B0013440B4403F26F3302461A7032
:102DE000B97BBA7B78680B46DB000B445B000B4475
:102DF000034430331B78D8B209491346DB0013442F
:102E00005B0013440B4403F55C7302461A70BB7BF2
:102E10000133BB738DE700BF1037BD46B0BD00BFA7
:102E2000F4010020B0B584B000AF78604F4B93F848
:102E30002C307B7378680FF0B1FC4C4B1B8E9BB22F
:102E4000DAB27B6883F869207B7B002B03D00021FA
:102E500078680FF000FF454B1B8E9BB2002B14BF10
:102E600001230023DBB2002B03D0012178680FF08F
:102E7000F2FE3E4B93F85433DAB27B68DA740023E7
:102E8000FB73FB7B022B6DD8FA7BFB7B37490A4433
:102E900092F85523D1B27A6813440A461A75FB7B1F
:102EA000FA7B324903F5D4735B000B441B8999B25A
:102EB0007B680C3223F812100023BB73BB7B102BF2
:102EC0001ED8F97BBC7BFA7BB87B284D0B46DB0018
:102ED0000B445B000B442B44234403F25E331B780A
:102EE000DCB279681346DB0013445B0013440B44E7
:102EF00003441E3322461A70BB7B0133BB73DDE7EC
:102F0000F97BFA7B19480B46DB000B445B000B4452
:102F1000034403F26F331B78D8B279681346DB00A1
:102F200013445B0013440B442F3302461A70F97BA1
:102F3000FA7B0E480B46DB000B445B000B4403445A
:102F400003F55C731B78D8B279681346DB00134431
:102F50005B0013440B44303302461A70FB7B013391
:102F6000FB738EE700BF1037BD46B0BDF4010020F3
:102F700080B582B000AF78607B6893F8783103F059
:102F80008103002B08D07B6893F8783183F002032B
:102F9000DAB27B6883F878217B6893F87931002B6B
:102FA0001CD17B6893F874311A467B68883233F8F9
:102FB0001230002B12D17B68B3F870311AB27B68E3
:102FC00093F87431194601238B401BB2DB431BB2CB
:102FD00013401BB29AB27B68A3F87021786800F0A6
:102FE0000FF87B6893F87831832B02D1034B0122D1
:102FF0001A7300BF0837BD4680BD00BFC01D00204A
:1030000080B582B000AF78607B6893F87831812B0F
:1030100002D0832B6FD096E07B6893F874311A4608
:10302000012393409AB24A4BDA827B6893F8743159
:103030001A46012393409AB2454BDA81444B5B8A8E
:103040009BB243F480539AB2414B5A82404B1B8A45
:103050009BB243F001039AB23D4B1A823D4A137969
:1030600043F0100313713C480FF0FAFB3A48FFF7A6
:10307000B9FC7B68B3F870217B68B3F872311340F8
:103080009BB21A467B6893F8743142FA03F303F05B
:103090000103002B06D07B6893F8743119467868D9
:1030A00000F0A0F87B68B3F870311A467B6893F89B
:1030B000743142FA03F303F00103002B07D12448D3
:1030C0000FF095F87B68FF2283F879213BE02048D8
:1030D0000FF09AF87B68B3F872311A467B6893F860
:1030E000743142FA03F3DBB203F00103DAB27B6816
:1030F00083F8792127E018480FF0B2FB1648FFF754
:1031000039FD13480FF080F8114B00229A82104BC2
:103110000022DA820E4B0022DA810D4B1B8A9BB211
:1031200023F001039AB20A4B1A820A4A13796FF309
:1031300004131371064B5B8A9BB223F480539AB23B
:10314000034B5A8200BF00BF0837BD4680BD00BF99
:10315000C01D0020F4010020A81E0020B0B584B0DE
:1031600000AF78607B6893F874311C461C480EF001
:10317000B4FE03461A467B68234483F800217B682B
:1031800093F874311A467B68134493F80031FB734B
:10319000FB7B002B20D07B6893F874311A467B6848
:1031A000134493F80021FB7BD31ADAB27B6893F8BF
:1031B00074311D46FB7B5C1E114609480EF0A9FECA
:1031C000034619467A682B01134423440A461A70B1
:1031D000FB7B013BFB73DBE700BF1037BD46B0BD97
:1031E000A81E002080B582B000AF78600B46FB704F
:1031F0007B68FA7812019918FB787A68134493F87F
:1032000000311A4603480FF0A6FD00BF0837BD463F
:1032100080BD00BFA81E002090B585B000AF7860CB
:103220007B68B3F87021624BA3F8D4227B68B3F8B3
:1032300072215F4BA3F8D6220023FB73FB7B0F2B7D
:1032400000F2B180F97BFB7B7A684C3112F82120C7
:10325000C2F30102D1B2564AA4339B0013441A7937
:1032600061F301021A71F97BFB7B7A684C3112F829
:103270002120C2F38102D1B24D4AA4339B001344F2
:103280001A7961F383021A71F97BFB7B7A684C31FE
:1032900012F82120C2F30012D1B2454AA4339B0098
:1032A00013441A7961F304121A71F97BFB7B7A6873
:1032B0004C3112F82120C2F34212D1B23C4AA4335D
:1032C0009B0013441A7961F347121A71F97BFB7B57
:1032D0007A68883132F81110354A03F59C735B0027
:1032E00013440A469A80FB7BFA7B79680B4493F877
:1032F00000012F491346DB0013449B000B44543359
:1033000002461A700023BB7397F90E30072B3DDC81
:10331000FA7B97F90E305B00796812010A44134476
:103320001B78FA7B97F90E0003F00F03D9B2204CFB
:103330001346DB00134403440C339B0023441A79E7
:1033400061F303021A71FA7B97F90E305B000133C7
:10335000796812010A4413441B78FA7B97F90E002E
:1033600003F00F03D9B2124C1346DB00134403449D
:103370000C339B0023441A7961F307121A7197F9F1
:103380000E30DBB20133DBB2BB73BDE7002109486D
:103390000EF0BFFD03461A46054B83F8D822FB7B8F
:1033A0000133FB734AE700BF1437BD4690BD00BF31
:1033B000F4010020A721002080B584B000AF786020
:1033C00078680FF053FD6C4BB3F8D4329AB27B6837
:1033D000A3F87021684BB3F8D6329AB27B68A3F891
:1033E00072210023FB73FB7B0F2B00F2AA80FB7B77
:1033F000F97B614AA4339B0013445B68C3F3010368
:10340000D8B27A684C3112F8213060F3010302F827
:103410002130FB7BF97B584AA4339B0013445B6843
:10342000C3F38103D8B27A684C3112F8213060F3CB
:10343000830302F82130FB7BF97B4F4AA4339B00C6
:1034400013445B68C3F30013D8B27A684C3112F8A6
:10345000213060F3041302F82130FB7BF97B464AEC
:10346000A4339B0013445B68C3F34213D8B27A6859
:103470004C3112F8213060F3471302F82130FB7B06
:10348000FA7B3D4903F59C735B000B449B8899B222
:103490007B68883223F81210FA7BF97B3648134692
:1034A000DB0013449B00034454331B78DAB27B687F
:1034B0000B4483F800210023BB7397F90E30072BD0
:1034C0003BDCFA7B97F90E102B481346DB001344C4
:1034D0000B440C339B0003445B68C3F30303D9B272
:1034E000FA7B97F90E305B000846796812010A44AE
:1034F000134402461A70FA7B97F90E101E481346C1
:10350000DB0013440B440C339B0003445B68C3F3A0
:103510000313D9B2FA7B97F90E305B0001330846EA
:10352000796812010A44134402461A7097F90E3062
:10353000DBB20133DBB2BB73BFE7FB7B0133FB7351
:1035400051E70D4B93F8D832DBB2FF2B14BF0123A8
:103550000023DBB2002B0AD07B6803F28F13064AEC
:1035600092F8D822D2B2114618460EF038FC00BFAD
:103570001037BD4680BD00BFF401002090B585B076
:1035800000AF78607B68012283F88E217B6803F2AC
:103590008F1318460EF0A1FC0346002B0AD07B685F
:1035A00003F27B1318460EF098FC0346002B01D162
:1035B000012300E00023002B39D000213D480EF00C
:1035C000A8FC034603F00F03DAB23B7B62F303036C
:1035D0003B733B7B43F010033B733B7B6FF3451323
:1035E0003B733B7B6FF386133B733B7B6FF3C713DC
:1035F0003B737B6803F28F1318460EF0CAFBF96821
:103600002D480EF06AFB00212A480EF082FC03468A
:103610001A46012303FA02F1284BDB8A9BB21AB245
:103620000BB213431BB29AB2244BDA821CE07B68C4
:1036300003F27B1318460EF050FC0346002B14BF18
:1036400001230023DBB2002B0ED07B6803F28F1422
:103650007B6803F27B13002118460EF05AFC0346E8
:10366000194620460EF0BBFB7B6803F28F13184609
:103670000EF033FC0346002B14BF01230023DBB202
:10368000002B12D000210B480EF043FC03461A46D3
:10369000012303FA02F1094BDB8A9BB21AB20BB287
:1036A00013431BB29AB2054BDA8200BF1437BD46F2
:1036B00090BD00BFBB210020DC1D0020C01D0020EC
:1036C00080B582B000AF78607B68002283F88E21DD
:1036D0007B68FF2283F87A211A48FFF74BFA1948D2
:1036E0000FF0BEF87B6803F27B1318460EF051FB17
:1036F000154800F04DF8154B1B8A9BB223F48073DC
:103700009AB2124B1A82114B1B8A9BB223F00E0302
:103710009AB20E4B1A8200210D480EF0FAFB0346B6
:103720001A4601239340D943084BDB8A9BB21AB255
:103730000BB213401BB29AB2044BDA8200BF0837B7
:10374000BD4680BDA81E0020141F0020C01D002003
:10375000BB21002080B582B000AF78607B68043365
:1037600018460EF00AFB7B681A3318460EF005FB6C
:10377000054B064A1A62786800F00AF87B6818461A
:103780000837BD4680BD00BF6C1E0020941E00207F
:1037900080B582B000AF786007480EF0FAFA0748AB
:1037A0000EF099FD064B00229A8278680FF05EFDBC
:1037B00000BF0837BD4680BD941E00206C1E00204F
:1037C000C01D002080B485B000AF78607B681B7896
:1037D000DAB22E4B83F824237B685B889AB22B4B9A
:1037E000A3F826230023FB73FB7B102B0ED8FA7B58
:1037F000FB7B79680A441279D1B2244A13440A4601
:1038000083F82823FB7B0133FB73EDE77B685B7D4B
:10381000DAB21E4B83F839237B689B7DDAB21B4BEF
:1038200083F83A237B68DB7DDAB2184B83F83C23BC
:103830007B681B8B9AB2154BA3F83E230023BB7306
:10384000BB7B102B0ED8BA7BBB7B79680A44927E77
:10385000D1B20E4A13440A4683F84023BB7B01339E
:10386000BB73EDE77B6893F82B30DAB2074B83F834
:1038700051237B6893F82C30DAB2044B83F852233F
:1038800000BF1437BD465DF8047B7047F40100208B
:1038900080B485B000AF78602F4B93F82433DAB250
:1038A0007B681A702C4BB3F826339AB27B685A8027
:1038B0000023FB73FB7B102B0ED8FA7BFB7B264986
:1038C0000A4492F82823D1B27A6813440A461A713E
:1038D000FB7B0133FB73EDE71F4B93F83933DAB20F
:1038E0007B685A751C4B93F83A33DAB27B689A7549
:1038F000194B93F83C33DAB27B68DA75164BB3F8A0
:103900003E339AB27B681A830023BB73BB7B102BB8
:103910000ED8BA7BBB7B10490A4492F84023D1B23F
:103920007A6813440A469A76BB7B0133BB73EDE792
:10393000094B93F85133DAB27B6883F82B20064B9E
:1039400093F85233DAB27B6883F82C2000BF143727
:10395000BD465DF8047B7047F401002090B585B04A
:1039600000AF78607B6801221A705E480EF0B5FAED
:103970000346002B14BF01230023DBB2002B00F011
:1039800087807B6800225A807B68043318460EF0DB
:1039900000FA54480EF0A1FA0346FB73FB7B002BA0
:1039A00027D07B681C1DFB7B013BDBB219464D48D1
:1039B0000EF0AFFA0346194620460EF010FAFB7BD4
:1039C000013BDBB2194647480EF0A3FA03461A46FC
:1039D000012303FA02F17B685B889BB21AB20BB237
:1039E00013431BB29AB27B685A80FB7B013BFB738B
:1039F000D4E77B68043318460EF06FFA03461C4682
:103A000039480EF04DFE03469C428CBF0123002333
:103A1000DBB2002B58D034480EF042FE0346BB7395
:103A20007B68043318460EF058FA03461A46BB7BEF
:103A3000934234BF01230023DBB2002B1DD07B68EF
:103A40001C1D7B680433BA7B114618460EF061FAE0
:103A50000346194620460EF0F7F97B680433BA7B1B
:103A6000114618460EF055FA03461946786800F0DC
:103A7000B7F8BB7B0133BB73D2E77B681C1D1A48C8
:103A80000EF00EFE0346194620460EF033FA1BE0F8
:103A90007B68043318460EF020FA03467B737B7B69
:103AA000002B11D07B681A1D7B7B013BDBB21946D2
:103AB00010460EF02EFA03461946786800F066F8B4
:103AC0007B7B013B7B73EAE77B6893F82D30002B0F
:103AD00004D07B685B889AB2044BDA8100BF14374C
:103AE000BD4690BD941E00206C1E0020C01D00200D
:103AF00090B585B000AF78607B68043318460EF04F
:103B0000ECF90346FB73FB7B002B2BD01D48FDF724
:103B1000E9F803461C467B681A1DFB7B013BDBB2C0
:103B2000194610460EF0F5F9034644FA03F303F084
:103B30000103002B0CBF01230023DBB2002B0DD0AF
:103B40007B681A1DFB7B013BDBB2194610460EF069
:103B5000E0F903461946786800F042F8FB7B013B28
:103B6000FB73D0E77B6800221A707B6893F82D30D6
:103B7000002B02D0044B0022DA8100BF1437BD466F
:103B800090BD00BF601E0020C01D002080B582B027
:103B900000AF78600B46FB700E4B5B68C3F381038C
:103BA000DBB2032B02D1FB78022B01D9012300E009
:103BB0000023002B04D0FB78194607480EF00FF9BC
:103BC000FB7819460548FDF789FB00BF0837BD465D
:103BD00080BD00BFF4010020941E00206C1E002058
:103BE00080B582B000AF78600B46FB700E4B5B680F
:103BF000C3F38103DBB2032B02D1FB78022B01D983
:103C0000012300E00023002B04D0FB78194607486D
:103C10000EF01AF9FB78194605480EF0E9FB00BFD3
:103C20000837BD4680BD00BFF4010020941E00206F
:103C30006C1E002090B585B000AF786039603B788D
:103C400003F01003DBB2002B00F0D8808C4B5B68D4
:103C5000C3F38103DBB2022B08D1894B5B68C3F34A
:103C60000103DBB2022B01D1012300E00023002B72
:103C70000BD03B78C3F30303DBB2194681480EF047
:103C8000AEF881480EF0C2FCE4E07B681B78DBB242
:103C900083F00103DBB2002B08D03B78C3F30303AE
:103CA000DBB219467868FFF771FFD3E03B78C3F3C6
:103CB0000303DBB2194678680FF055FB034683F027
:103CC0000103DBB2002B6BD07B681A1D3B78C3F37A
:103CD0000303DBB2194610460EF081F87B6804330B
:103CE00018460EF0FAF803461C4667480EF0D8FC5A
:103CF00003469C428CBF01230023DBB2002B46D03D
:103D000061480EF0CDFC0346FB737B680433184614
:103D10000EF0E3F803461A46FB7B934234BF0123BF
:103D20000023DBB2002B28D07B680433FA7B1146DA
:103D300018460EF0EEF8034619467868FFF750FF74
:103D40007B680433FA7B114618460EF0E2F803460E
:103D50001A460123934083F47F4383F0FF037A687C
:103D6000528892B212B21BB213401BB29AB27B6855
:103D70005A80FB7B0133FB73C7E77B681C1D4248FD
:103D80000EF08EFC0346194620460EF0B3F83B7841
:103D9000C3F30303DBB219467868FFF7F7FE11E0BF
:103DA0007B681A1D3B78C3F30303DBB21946104648
:103DB0000EF04AF83B78C3F30303DBB21946786888
:103DC000FFF70EFF7B685B889BB21AB23B78C3F3A8
:103DD0000303DBB2194601238B401BB253401BB2D5
:103DE0009AB27B685A807B6893F82D30002B31D0D3
:103DF0007B685B889AB2254BDA812BE0204B5B68AD
:103E0000C3F38103DBB2022B06D11D4B5B68C3F306
:103E10000103DBB2022B01D0012300E00023002BC1
:103E200010D07B681B78DBB283F00103DBB2002B80
:103E300010D03B78C3F30303DBB219467868FFF771
:103E4000CFFE07E03B78C3F30303DBB219460D480E
:103E50000DF0FAFF0E4B93F87931002B0BD10C4B80
:103E600093F87831812B06D17B685B889BB2194629
:103E700007480FF03FF900BF1437BD4690BD00BFA3
:103E8000F4010020941E00206C1E0020C01D0020A4
:103E90002C20002090B585B000AF78600846114610
:103EA0001A4603467B800B467B7013463B703B787B
:103EB000194620480FF081F90346C3F30103DBB232
:103EC0001C463B7819461B480FF077F90346C3F3AD
:103ED0008103DBB21A4621461748FDF7A9F90023F2
:103EE000BB600023FB73FB7B0F2B1FD87B8803F089
:103EF0000103002B13D0FB7B03F00F03DAB23B7AF4
:103F000062F303033B727B7803F00103DAB23B7A7E
:103F100062F304133B72B9687868FFF78BFE7B8805
:103F20005B107B80FB7B0133FB73DCE700BF143746
:103F3000BD4690BD2C2000206C1E002080B582B0B4
:103F400000AF78607B68012283F82D2003480EF0D3
:103F5000DFFB00BF0837BD4680BD00BF6C1E0020E0
:103F600080B582B000AF78607B68002283F82D2096
:103F700003480EF0DAFB00BF0837BD4680BD00BF26
:103F80006C1E002080B582B000AF78607B68144A58
:103F900004331146C022184610F03BFF7B68002214
:103FA00083F8C5207B68002283F8C6207B68002246
:103FB00083F8C7207B68002283F8C8207B684FF015
:103FC0000002C3F8CC207B68002283F8D0207868F8
:103FD00000F008F87B6818460837BD4680BD00BF72
:103FE0006C53010080B483B000AF78601C4B00229A
:103FF0005A821C4B002283F898237B68002283F8A6
:10400000D1207B68032283F8D2207B6817221A70A4
:104010007B68012283F8C4207B684FF00002C3F85C
:10402000CC207B68012283F8D0207B68002283F8B3
:10403000C7207B68002283F8C8200A4B002283F83F
:104040009923084B0022C3F8A023064B0022C3F893
:10405000A42300BF0C37BD465DF8047B704700BF4A
:10406000C01D0020F401002080B483B000AF786050
:10407000064B00225A827B68052283F8D12000BFBC
:104080000C37BD465DF8047B704700BFC01D0020A3
:1040900080B582B000AF78607868FFF7E5FF0F4821
:1040A0000DF0FCFD0E48FFF773FB7B68002283F8E0
:1040B000C8200C4B0022C3F8A4237B684FF00002F9
:1040C000C3F8CC207B68012283F8D0207B680022D3
:1040D00083F8D12000BF0837BD4680BDDC1D00201D
:1040E000141F0020F401002080B582B000AF78607A
:1040F0007B6893F8D130023B032B40D801A252F8E1
:1041000023F000BF3F4100001541000023410000A3
:10411000514100007868FFF7BBFF786800F084F831
:104120002DE07868FFF7B4FF174BD3F8A033013BBD
:10413000154AC2F8A433786800F08EF81FE078685A
:10414000FFF750FF786800F021F801F0F3F916E06E
:104150007B6893F8D230032B02D0042B07D00DE0FC
:104160007868FFF795FF786800F05EF806E07868F9
:10417000FFF78EFF786800F06FF800BF00BF00BF48
:104180000837BD4680BD00BFF401002080B582B075
:1041900000AF78600E48FFF7FBFA0E4B93F89833A8
:1041A000DBB2002B14BF01230023DBB2002B03D0B2
:1041B00078680FF0F7F807E07B68012283F8D120D8
:1041C000054B42F201025A8200BF0837BD4680BD4E
:1041D000141F0020F4010020C01D002080B483B013
:1041E00000AF78607B6817221A700D4B012283F8AC
:1041F00098237B6893F8C530002B03D07B6801229D
:1042000083F8C6207B68022283F8D120054B4FF447
:1042100000525A8200BF0C37BD465DF8047B7047E0
:10422000F4010020C01D002080B483B000AF78608E
:104230007B68032283F8D1207B68032283F8D22095
:10424000044B00225A8200BF0C37BD465DF8047B48
:10425000704700BFC01D002080B483B000AF7860FD
:104260007B68042283F8D1207B68042283F8D22063
:10427000044B00225A8200BF0C37BD465DF8047B18
:10428000704700BFC01D002080B483B000AF7860CD
:104290000B46FB70FB78002B0FD0FB780E2B0CD855
:1042A0007B6893F9C430DBB21B01DAB2FB781344AC
:1042B000DBB25AB27B681A7021E0FB78002B0FD179
:1042C0007B6893F9C430002B19D07B6893F9C43014
:1042D000DBB2013BDBB25AB27B6883F8C4200EE04C
:1042E0007B6893F9C430012B09DC7B6893F9C430F7
:1042F000DBB20133DBB25AB27B6883F8C420044BD3
:1043000001221A7000BF0C37BD465DF8047B704770
:104310007C2C002090B585B000AF7860AC4B9B78CA
:1043200003F00103DBB2002B14D1A94B9B7803F0FF
:104330000203DBB2002B0DD1A54B9B7803F00403E5
:10434000DBB2002B06D1A24B9B7803F00403DBB257
:10435000002B02D0786800F0D9FA9E480EF0F1FCEC
:104360000023BB609C4B1B78DBB2093B042B00F2A3
:10437000BA8201A252F823F0D54600008D43000016
:10438000E748000085470000374800007B681B7C39
:10439000002B57D08F480DF0A0FD0346012B02D013
:1043A000032B17D041E07B685C7A002189480DF02F
:1043B000B0FD03462344DBB203F00F03DAB27B689F
:1043C0009A727B685A7A7B68DA727B689A7A7B6821
:1043D0001A7343E07B685C7A00217E480DF099FDFA
:1043E00003462344DBB203F00F03DAB27B689A7210
:1043F0007B685C7A012177480DF08BFD03462344EE
:10440000DBB203F00F03DAB27B68DA727B685C7AA6
:10441000022170480DF07DFD03462344DBB203F01A
:104420000F03DAB27B681A7318E07B685A7A7B68EC
:104430009A727B685A7A7B68DA727B685A7A7B68F0
:104440001A730BE07B685A7A7B689A727B685A7A97
:104450007B68DA727B685A7A7B681A730023FB7375
:10446000FB7B032B00F2FB807B68DB881946FB7B20
:104470007A6813445B7A41FA03F303F00103002BDB
:1044800000F0E98053480DF028FD0346032B4BD87C
:1044900001A252F823F000BFA9440000C744000065
:1044A000E944000007450000FB7B002B37D14A4B55
:1044B0005B68C3F34213DBB21946FB7B1A464548DF
:1044C000FDF7EEFF2BE0FB7B03F00203002B28D16E
:1044D000414B5B68C3F34213DBB21946FB7B1A46C0
:1044E0003C48FDF7DDFF1CE0FB7B002B1BD13A4B6A
:1044F0005B68C3F34213DBB21946FB7B1A463548AF
:10450000FDF7CEFF0FE0344B5B68C3F34213DBB221
:104510001946FB7B1A462F48FDF7C2FF04E000BF97
:1045200002E000BF00E000BFFB7B032B00F29380A2
:1045300001A252F823F000BF494500006F4500007A
:10454000B745000009460000002122480EF01EFA7F
:10455000034603F00F03D9B21D4A137861F3030336
:1045600013701B4A937843F00103937073E019486A
:104570000DF0B3FC034603F00103012B03D07B686D
:10458000DB7B002B01D0012300E00023002B5DD05A
:10459000012110480EF0FAF9034603F00F03D9B2D7
:1045A0000B4A137861F307131370094A937843F0A9
:1045B000020393704AE007480DF08FFC0346032B7B
:1045C00003D07B68DB7B002B08D0012307E000BF12
:1045D000E4010020A81E0020F40100200023002B8D
:1045E00036D00221B5480EF0D1F9034603F00F038F
:1045F000D9B2B34A537861F303035370B04A937846
:1046000043F00403937023E0AC480DF066FC0346CE
:10461000032B03D07B68DB7B002B01D0012300E060
:104620000023002B16D00321A4480EF0AFF9034657
:1046300003F00F03D9B2A24A537861F30713537002
:104640009F4A937843F00803937003E000BF02E0B1
:1046500000BF00E000BFFB7B0133FB7300E77B681A
:104660009B7B83F00103DBB2002B02D0954B002231
:10467000DA810023BB73BB7B032B00F22D817B68A7
:104680009B7B83F00103DBB2002B08D08E4B1B69B0
:10469000C3F34333DBB20A2B01D0012300E0002334
:1046A000002B13D0BB7B194684480EF06FF90346EC
:1046B0001A46012303FA02F1824BDB899BB21AB23C
:1046C0000BB213431BB29AB27E4BDA81BB7B013330
:1046D000BB73D0E77B68DB881A467B685B7A42FA5B
:1046E00003F303F00103002B00F0F88073480DF092
:1046F000F4FB0346002B08D1744B5B68C3F34213F1
:10470000DBB2052B01D1012300E00023002B40F098
:10471000F5806E4B5B68C3F34213DBB21946674802
:10472000FEF71CF8002165480EF030F9034603F04F
:104730000F03DAB23B7A62F303033B723B7A43F036
:1047400010033B72B9686248FFF774FA7B689B7B81
:1047500083F00103DBB2002B00F0C080002157483A
:104760000EF014F903461A46012303FA02F1554BE1
:10477000DB899BB21AB20BB213431BB29AB2514BF4
:10478000DA81ABE07B68DB881A467B685B7A42FAA9
:1047900003F303F00103002B00F0A28047480DF063
:1047A0009CFB0346002B08D1484B5B68C3F34213C4
:1047B000DBB2052B01D1012300E00023002B40F0E8
:1047C0009F80424B5B68C3F34213DBB219463B4800
:1047D000FDF7C4FF002139480EF0D8F8034603F076
:1047E0000F03D9B2364A537861F3071353707B68CD
:1047F0009B7B83F00103DBB2002B08D0334B5B685B
:10480000C3F30013DBB2012B01D1012300E000232D
:10481000002B0AD0002129480EF0B8F803461A46AA
:10482000012393409AB2274BDA81254A937843F0CB
:104830000803937054E07B68DB881A467B685B7AD8
:1048400042FA03F303F00103002B4BD0214B93F802
:104850007831812B04D11F4B93F87931012B09D08A
:104860001C4B93F87831832B3CD11A4B93F87A3157
:10487000012B37D111480DF030FB0346002B0CBF44
:1048800001230023DBB2002B3CD105210B48FDF7AF
:1048900065FF002109480EF079F8034603F00F0385
:1048A000DAB23B7A62F303033B723B7A43F01003C4
:1048B0003B72B9680648FFF7BDF913E0A81E002057
:1048C000E4010020C01D002000F00F40F401002092
:1048D000141F00202C20002000BF04E000BF02E0D5
:1048E00000BF00E000BF7B689B7B002B02D0786894
:1048F00000F02EF978680EF0C2FD04E000BF02E07F
:1049000000BF00E000BF1437BD4690BD80B584B045
:1049100000AF78600023FB60654B1B78DBB2093B7E
:10492000042B00F2BA8001A252F823F06B49000078
:10493000414900009B4A0000F74900003F4A00003F
:104940005C4A93786FF3000393705A4A93786FF33D
:1049500041039370574A93786FF382039370554ADB
:1049600093786FF3C303937097E0002152480EF0E1
:104970000DF8034603F00F03DAB23B7B62F3030347
:104980003B733B7B6FF304133B73F9684B48FFF7B2
:1049900051F97B689B7B83F00103DBB2002B0AD0CB
:1049A000002145480DF0F2FF03461A4601239340CB
:1049B0009AB2434BDA813F4B9B7803F00103DBB2A1
:1049C000002B14D13B4B9B7803F00203DBB2002B8E
:1049D0000DD1384B9B7803F00403DBB2002B06D1DA
:1049E000344B9B7803F00803DBB2002B50D03348E4
:1049F000FEF7CEFE4CE02F4A93786FF3C30393701B
:104A00007B689B7B83F00103DBB2002B08D0284B33
:104A10005B68C3F30013DBB2012B01D1012300E07B
:104A20000023002B36D0002123480DF0AFFF0346B2
:104A30001A46012393409AB2214BDA812AE0214B96
:104A400093F87831812B04D11E4B93F87931012BE7
:104A500009D01C4B93F87831832B1DD1194B93F857
:104A60007A31012B18D1002113480DF08FFF034636
:104A700003F00F03DAB23B7B62F303033B733B7B30
:104A80006FF304133B73F9680C48FFF7D3F803E0A6
:104A900000BF02E000BF00E000BF7B689B7B002BF3
:104AA00002D0786800F054F800BF1037BD4680BDD2
:104AB000F4010020E4010020A81E0020141F0020A3
:104AC000C01D00202C20002080B582B000AF78608F
:104AD0000C48FFF745FA0C480EF0A2F90B4B1B8A65
:104AE0009AB27B681A80094BDB899AB27B685A803C
:104AF000064B9B8A9AB27B689A8000BF0837BD46F6
:104B000080BD00BF141F0020A81E0020C01D002073
:104B100080B582B000AF78600A48FFF70FFA0A4804
:104B20000EF070F97B681A88084B1A827B685A88E5
:104B3000064BDA817B689A88044B9A8200BF08375B
:104B4000BD4680BD141F0020A81E0020C01D0020EF
:104B500080B483B000AF78607B68DA88034B9A82B8
:104B600000BF0C37BD465DF8047B7047C01D0020B8
:104B700080B582B000AF78607868FFF7A5FF094B79
:104B800001229A76074B0022DA81064B00229A8294
:104B90007868FFF7DDFF7B6801229A7300BF083752
:104BA000BD4680BDC01D002080B483B000AF7860DA
:104BB0000B46FB707B68DB881AB2FB78012101FA97
:104BC00003F31BB253401BB29AB27B68DA807B6856
:104BD000DA88044B9A8200BF0C37BD465DF8047B2F
:104BE000704700BFC01D002080B582B000AF786064
:104BF0007B68DA88134BA3F8DA227B681B7C1846A3
:104C00000EF07BFC034603F00103D9B20D4A92F883
:104C1000DC3261F3000382F8DC327B68DB7B184610
:104C20000EF06BFC034603F00103D9B2054A92F87B
:104C3000DC3261F3410382F8DC3200BF0837BD4645
:104C400080BD00BFF401002080B582B000AF786065
:104C500078680EF0E0FB134BB3F8DA329AB27B6857
:104C6000DA80104BD3F8DC32C3F30003DBB25BB263
:104C700018460EF053FC03461A467B681A74094B1B
:104C8000D3F8DC32C3F34003DBB25BB218460EF05C
:104C900045FC03461A467B68DA7300BF0837BD46F9
:104CA00080BD00BFF401002080B483B000AF786005
:104CB0007B684FF000021A607B684FF07E525A60AA
:104CC0007B68134A9A607B689A687B68DA607B68C5
:104CD0004FF000025A617B684FF07C52DA617B68CA
:104CE0005A697B689A617B684FF07E521A627B68D2
:104CF00000225A627B6804229A627B684FF07C52E1
:104D00001A617B6818460C37BD465DF8047B704716
:104D10000AD7233C80B52DED028B84B000AF7860BC
:104D200087ED000A7B68D3ED037A97ED007A77EE82
:104D3000677AC7ED037AD7ED037AF5EEC07AF1EE24
:104D400010FA27D57B6893ED027A7B68D3ED007A61
:104D500037EE677AD7ED037A27EE278A7B6893EDE3
:104D6000037A7B68D3ED007A77EE677ADFED330A5A
:104D7000B0EE670A78680EF02DFEF0EE407A88EE0D
:104D8000277A7B68D3ED027A77EE277A7B68C3EDCA
:104D9000027A2DE0D7ED037AF5EEC07AF1EE10FA43
:104DA00026DD7B6893ED017A7B68D3ED027A37EEDE
:104DB000677AD7ED037A27EE278A7B6893ED017A2D
:104DC0007B68D3ED037A77EE677ADFED1C0AB0EEED
:104DD000670A78680EF0FEFDF0EE407A88EE277ADA
:104DE0007B68D3ED027A77EE277A7B68C3ED027A8F
:104DF0007B68D3ED027A7B6893ED007A7B68D3ED14
:104E0000016AB0EE661AF0EE470AB0EE670A7868FB
:104E10000EF0FDFDF0EE407A7B68C3ED027A7B6810
:104E20003A68DA607B689B6807EE903AB0EE670AF2
:104E30001037BD46BDEC028B80BD00BFBD37863547
:104E400080B483B000AF1A4B1B6CC3F38023DBB27A
:104E5000174983F00103DAB2B1F8403062F38A23D4
:104E6000A1F840301249B1F8403062F3CB23A1F8E9
:104E700040300023FB80FB884FF6FF729342E2D064
:104E800000233B603B680F2B0EDC094A3B6803F0B4
:104E90000F03D9B2D2F8803061F34813C2F88030E2
:104EA0003B6801333B60EDE7FB880133FB80E2E7C1
:104EB00000F00F4080B582B000AF00237B607B68BC
:104EC000DBB21A46002115480EF049FB7B68DBB2C5
:104ED0001A46032111480EF042FB7B68DBB21A46EA
:104EE00005210F480EF03BFB7B68DBB21A4601211F
:104EF0000C480EF034FB00233B603B68C72B05DCFD
:104F00000EF0F6FD3B6801333B60F6E77B68002B53
:104F10000CBF01230023DBB27B60D0E740F00F40E1
:104F2000C0F00F4080F00F4080B584B000AF7860D3
:104F30000B46FB70FB78284A32F813301A467B6820
:104F4000934201DA002343E0FB78234A103332F81E
:104F500013301A467B68934202DD4FF6FF7337E049
:104F6000FB781D4A32F813301A467B689B1A07EE0D
:104F7000903AF8EEE76AFB78174A103332F81330AC
:104F80001946FB78144A32F81330CB1A07EE903AE0
:104F9000B8EEE77AC6EE877AC7ED037AFB780E4A59
:104FA00010339B001344D3ED007AF0EE670A97EDBF
:104FB000030A0BF0B5FD87ED030AD7ED037A9FEDE9
:104FC000077A67EE877AFCEEE77A17EE903A9BB2A3
:104FD00018461037BD4680BDC01B002000FF7F472C
:104FE00080B59EB000AF002387F8773001233B6780
:104FF000A24BD3F81031C3F38063DBB2002B00D097
:10500000F6E79F4B01221A709E4B1B78002B00F095
:105010004882002387F8773097F877300F2BF3D842
:1050200001220A2198480EF09AFA01220B21964893
:105030000EF095FA954B4FF4F0729A6097F877302E
:105040005A01924B5A60924B1B7897F877209A42FC
:1050500004D100220B218C480EF081FA97F87730AA
:10506000042B02D13B6F002B11D197F87730052B21
:1050700002D13B6F002B0AD0804B1B69C3F3433333
:10508000DBB2012B05D197F87730002B01D101233A
:1050900000E00023002B04D000220A217A480EF001
:1050A0005EFA7B4B1B781A467A4B33F812301B138F
:1050B000774A12781046784A9B0013441A68774959
:1050C00000F110039B000B441A60714B1B781846CB
:1050D0006F4B1B7819466F4A00F1100332F813200A
:1050E0004B0007F178010B4423F8482C684B1B78E0
:1050F0005B0007F17802134433F8483C644A1278A5
:105100001146B3F52F7F8CBF01230023DAB207F1DC
:1051100078030B4403F8782C5D4B1B7818465C4BE6
:105120001B7819465E4A00F1100332F813204B0039
:1051300007F178010B4423F8282C554B1B785B00B2
:1051400007F17802134433F8283C1A13504B1B78AC
:1051500092B25B0007F178010B4423F8682C4C4BAA
:105160001B7807F17802134413F8783C002B10D019
:1051700097F87720464B1B785B0007F178010B44CA
:1051800033F8683C9A4204DA00220A213E480EF0C5
:10519000E6F93F4B1B7807F17802134413F8783C8B
:1051A000002B14D00122002137480EF0D8F901223B
:1051B000032135480EF0D3F90122052139480EF0BC
:1051C000CEF90122012131480EF0C9F913E0002285
:1051D00000212D480EF0C3F9002203212A480EF0C9
:1051E000BEF9002205212F480EF0B9F90022012155
:1051F00026480EF0B4F9214BD3F81031C3F3806385
:10520000DBB2002B11D001233B67214B1B781A46E0
:10521000224B40F2145123F812101D4B1B781F4AE9
:1052200010334FF6FF7122F81310144B1B69C3F3B0
:105230004333DBB2012B0CBF01230023DBB2002B75
:1052400043D0134B1B7807F17802134413F8783CD2
:10525000002B3AD03B6F002B26D00D4B1B78194604
:105260000B4B1B781A464B0007F178010B4433F8BF
:10527000481C0A4B23F8121027E000BF00F00F4033
:105280007F2C00208E2C002040F00F4080F00F403B
:105290008D2C0020A001002034540100C01B0020F0
:1052A000381B0020C0F00F408A4B1B781A46894BF0
:1052B0001B781846530007F17802134433F8481C52
:1052C000854A00F1100322F81310844B1B69C3F3C5
:1052D0004333DBB2052B0CBF01230023DBB2002BD1
:1052E00001D001233B677D4B1B69C3F34333DBB222
:1052F000062B0CBF01230023DBB2002B01D00023BF
:105300003B67764B1B69C3F34333DBB2082B0CBFFF
:1053100001230023DBB2002B58D0704B1B69C3F371
:105320004333DBB2082B0CBF01230023DBB2002B7D
:1053300000D0F2E7674B1B781A46674B33F8122010
:10534000644B1B786449103331F813309A422DD9DD
:10535000604B1B781A465F4B1B7819465E4B33F83F
:1053600012204B0007F178010B4423F8682C594BAD
:105370001B781846574B1B781946574A00F1100303
:1053800032F81320544B23F81120524B1B781A4645
:10539000504B1B781846530007F17802134433F83A
:1053A000681C4D4A00F1100322F81310494B1B787A
:1053B0000E2B08D801233B67464B1B780133DAB22A
:1053C000444B1A7002E0464B00221A70434B1B6993
:1053D000C3F34333DBB2072B0CBF01230023DBB243
:1053E000002B58D03D4B1B69C3F34333DBB2072B73
:1053F0000CBF01230023DBB2002B00D0F2E7354BBA
:105400001B781A46344B33F81220324B1B78324942
:10541000103331F813309A422DD92E4B1B781A468F
:105420002C4B1B7819462C4B33F812204B0007F1FC
:1054300078010B4423F8682C264B1B781846254B23
:105440001B781946244A00F1100332F81320224B2E
:1054500023F811201F4B1B781A461E4B1B78184649
:10546000530007F17802134433F8681C1A4A00F11C
:10547000100322F81310174B1B78002B08D00123C0
:105480003B67144B1B78013BDAB2124B1A7002E0F7
:10549000134B00221A7097F87730013387F8773072
:1054A000BAE5104B00221A700F4B186801230F4AFF
:1054B000094905F00FFD0346002B14BF012300230B
:1054C000DBB2002B01D0FFF7BBFC00BF7837BD4635
:1054D00080BD00BF8D2C0020C01B002000F00F40BD
:1054E0008E2C00207F2C002000010020BFC3C901AA
:1054F00080B483B000AF0346FB71FB79052B0BD161
:105500000B4B1B78DBB2092B06D0094B1B78DBB2A7
:105510000C2B01D0012300E00023002B01D0042339
:1055200000E0FB7918460C37BD465DF8047B7047F8
:10553000F401002098B500AF954B5B68C3F30013EE
:10554000DBB21AB2924B1B78DBB2013B012101FAAC
:1055500003F31BB213431CB28E48FCF71FFA034639
:10556000C3F30103DBB20133012202FA03F31BB2DE
:1055700023431BB29AB2884B1A82874B1B7BDBB248
:10558000002B0AD0844B1B8A9BB223F00E039AB2E5
:10559000814B1A82804B00221A737D4B1B78DBB241
:1055A0000A2B0CBF01230023DBB2002B07D07A4B60
:1055B0001B8A9BB223F00E039AB2774B1A82744B6C
:1055C0005B68C3F34213DBB2002B14BF012300233B
:1055D000DBB2002B59D06E4B1B78DBB2092B09D004
:1055E0006B4B1B78DBB20A2B04D0694B1B78DBB208
:1055F0000C2B01D1012300E00023002B0FD0644BC2
:105600005B68C3F34213DBB21846FFF771FF034632
:105610000433DBB2012219465F480CF0AFFD5C4B4E
:105620001B78DBB20E2B0CBF01230023DBB2002B57
:105630002BD0574B93F89933DBB2002B0CBF0123CF
:105640000023DBB21A460F2153480CF097FD534B51
:1056500093F8D130052B12D0052B16DC032B02D08A
:10566000042B06D011E0012208214B480CF086FDE6
:105670000BE00122072148480CF080FD05E00122E3
:10568000012145480CF07AFD00BF454B9B7B002B68
:1056900008D0414B5B8A9BB243F480439AB23E4BA5
:1056A0005A8207E03C4B5B8A9BB223F480439AB258
:1056B000394B5A82364B1B78DBB20D2B0BD1394B51
:1056C00093F87831812B06D1364B93F87931FF2B43
:1056D00001D0012300E00023002B18D0314B93F8B8
:1056E0007931002B0AD0012B11D12B4B1B8A9BB295
:1056F00043F480739AB2284B1A8208E0264B1B8A27
:105700009BB243F480639AB2234B1A8200BF204BB2
:105710001B78DBB20A2B0CBF01230023DBB2002B6A
:1057200020D01F4B1B7C002B07D01B4B1B8A9BB22E
:1057300043F004039AB2184B1A82194BDB7B002BFF
:1057400008D0154B1B8A9BB243F008039AB2124B48
:105750001A8207E0104B1B8A9BB243F002039AB2F5
:105760000D4B1A82104B1B78002B07D00F4B1B7868
:105770001A46102108480CF001FD06E00C4B1B787E
:105780001A46102104480CF0F9FC00BF98BD00BF78
:10579000F40100206C1E0020C01D0020441F0020CA
:1057A000182000202C200020802C0020832C00209A
:1057B000822C002090B583B000AFA7490978797199
:1057C000797901390E2901F2668001A050F821F0A3
:1057D0000D580000755900003B5A0000FF5A0000A8
:1057E000DF5B0000055C00002B5C00002D5D00000D
:1057F000135E0000D15F0000876100009D62000021
:1058000025640000FD65000003670000934B1B78D2
:10581000DBB20C2B1ED0914B1B78DBB20E2B19D0B8
:105820008E4B5B68C3F38103DBB2032B12D08B4B2F
:105830001B78DBB20F2B0DD0884B1B78DBB20D2B06
:1058400008D0874B9B7B83F00103DBB2002B01D098
:10585000012300E00023002B37D0804B5B68C3F3AB
:105860000013DBB283F00103D9B27C4A137961F3F0
:1058700004131371794B1B78DBB20B2B0CBF012384
:105880000023DBB2002B08D0744B5B68C3F300131A
:10589000DBB2194673480DF045FD704B1B78DBB247
:1058A000092B04D06D4B1B78DBB20A2B01D10123ED
:1058B00000E00023002B08D0684B5B68C3F30013A3
:1058C000DBB2194668480DF0E2F9644B1B78DBB295
:1058D0000D2B0BD1654B93F87831832B04D0634BA0
:1058E00093F87831032B01D1012300E00023002B32
:1058F00019D05A4B5B68C3F30013DBB283F001038A
:10590000D9B2564A137961F30413137157480DF055
:10591000A0FC0346002B0CBF01230023DBB2194679
:1059200052480DF082FC4D4B1B78DBB20E2B0CBFA6
:1059300001230023DBB2002B00F07E874C4B93F851
:10594000D130052B08D0052B00F37687032B07D029
:10595000042B09D000F070BF45480DF023FD07E08F
:105960004348FEF781FB03E04148FEF77DFB00BFA3
:1059700000F062BF3A4B9B7B83F00103DBB2002B4C
:1059800006D0364B1B78DBB20A2B01D0012300E096
:105990000023002B41D0314B1B78DBB20D2B14BF01
:1059A00001230023DBB2002B1FD02C4B5B68C3F319
:1059B0000103DBB2002B14BF01230023DBB2002B59
:1059C0002BD02C4B0022DA81244A13796FF3010388
:1059D0001371294B1B78DBB203F00303D9B21F4AC2
:1059E000137961F38303137117E0204B93F8783137
:1059F000812B12D11D4B93F87931012B0DD16FF30F
:105A00000102022363F383026FF30412052363F39D
:105A10004712114615480DF0BCFB104B1B78DBB24A
:105A20000A2B0CBF01230023DBB2002B00F00687FA
:105A30000B4B0022DA7300F001BF094B9B7B83F014
:105A40000103DBB2002B19D0044B1B78DBB20A2B0D
:105A500014D0012313E000BF792C0020F4010020B2
:105A600018200020141F0020A81E00202C20002039
:105A7000441F0020C01D0020F40500200023002B3F
:105A800029D0A34B1B78DBB20D2B14BF01230023BD
:105A9000DBB2002B1FD09E4B5B68C3F30103DBB26C
:105AA000012B14BF01230023DBB2002B13D0994B31
:105AB0000022DA81964A1379012161F301031371FF
:105AC000954B5B78DBB203F00303D9B2904A1379AC
:105AD00061F3830313718E4B1B78DBB20A2B0CBF6F
:105AE00001230023DBB2002B00F0BC868B4B1B7C18
:105AF00083F00103DAB2894B1A7400F0B3BE874A0F
:105B0000927B82F00102D2B2002A06D0804A12783B
:105B1000D2B20A2A01D0012200E00022002A4ED08F
:105B20007B4A1278D2B20D2A14BF01220022D2B2CF
:105B3000002A2CD0764B5B68C3F30103DBB2022B47
:105B400014BF01230023DBB2002B38D0704A137935
:105B5000022161F3010313716F4B9B78DBB203F0F9
:105B60000303D9B26A4A137961F383031371684B53
:105B70005B68C3F38103DBB2032B0CBF012300235B
:105B8000DBB2002B1BD0634B0722DA8117E0644A9B
:105B900092F87821812A12D1614A92F87921012A5A
:105BA0000DD1022262F301036FF383036FF3041339
:105BB000052262F34713194659480DF0EAFA544B8F
:105BC0001B78DBB20A2B0CBF01230023DBB2002BB6
:105BD00000F04A86514B0122DA7300F045BE4F4B6C
:105BE0009B7B83F00103DBB2002B00F03F86484A29
:105BF0001379012161F347131371464B01229A7601
:105C000000F034BE454B9B7B83F00103DBB2002BDD
:105C100000F02E863E4A1379022161F34713137177
:105C20003C4B01229A7600F023BE3C4B9B7B83F0D9
:105C30000103DBB2002B00F01D86354B1B78DBB275
:105C40000E2B0CBF01230023DBB2002B1DD0354BE4
:105C500093F8D130042B15D0324B93F8D130022B6E
:105C600004D0304B93F8D130032B0ED12D4B93F849
:105C7000D130022B02D12B48FEF70AFA2948FEF751
:105C8000EBFA02E02748FEF72FFA214B1B78DBB234
:105C90000D2B0CBF01230023DBB2002B2DD0204B9A
:105CA00093F87831812B40F0E5851F48FDF770FDB2
:105CB0001B480DF092F91A4B93F87931002B13D150
:105CC000012119480DF02EFB15480DF028FA034666
:105CD0001C4613480DF082FA034601222146124861
:105CE000FEF7D8F800F0C6BD00210F480DF01AFBF2
:105CF0000B48FDF785F900F0BDBD054A1379032176
:105D000061F347131371034B01229A7600F0B2BD81
:105D1000F4010020C01D0020F40500201820002000
:105D20002C200020441F0020141F0020B24B9B7B1E
:105D300083F00103DBB2002B00F09E85AF4B1B7894
:105D4000DBB20E2B0CBF01230023DBB2002B1DD0D6
:105D5000AB4B93F8D130032B15D0A94B93F8D1302E
:105D6000022B04D0A64B93F8D130042B0ED1A44BB8
:105D700093F8D130022B02D1A148FEF789F9A0484F
:105D8000FEF752FA02E09E48FEF7AEF99B4B1B78F5
:105D9000DBB20D2B0CBF01230023DBB2002B2DD077
:105DA000984B93F87831812B40F066859648FDF743
:105DB000EFFC94480DF0F9F8924B93F87931002BF1
:105DC00013D1012190480DF0ADFA8E480DF0A7F9DE
:105DD00003461C468B480DF001FA0346012221467A
:105DE0008948FEF757F800F047BD002186480DF0BE
:105DF00099FA8448FDF704F900F03EBD7F4A137913
:105E0000042161F347131371804B01229A7600F04D
:105E100033BD794B9B7B83F00103DBB2002B00F099
:105E20002D85764B5B68C3F34213DBB2002B0CBFAE
:105E300001230023DBB2002B05D0704A1379052122
:105E400061F3471313716D4B1B78DBB20E2B0CBF44
:105E500001230023DBB2002B02D06948FEF718F9BA
:105E6000664B1B78DBB20B2B0CBF01230023DBB28C
:105E7000002B25D064480DF00FFA604B5B68C3F32C
:105E80000103DBB2022B08D15C4B5B68C3F38103D7
:105E9000DBB2032B01D1012300E00023002B0FD044
:105EA000564A13796FF383031371544B5B68C3F342
:105EB0008103DBB21A46564B9A70544B0022DA81AA
:105EC0004E4B1B78DBB2092B0CBF01230023DBB246
:105ED000002B07D0494A1379052161F34713137149
:105EE00000F0CCBC454B1B78DBB20A2B0CBF012366
:105EF0000023DBB2002B08D046480CF04FFF45488A
:105F0000FCF770FD4348FCF735FE3C4B1B78DBB2D9
:105F10000D2B06D13B4B93F87831812B01D0012317
:105F200000E00023002B02D03648FDF7C9FB334BBD
:105F30001B78DBB20D2B06D1324B93F87831812BD5
:105F400001D1012300E00023002B0BD02D480DF0E0
:105F50005CF82D48FDF71CFC00212B480DF0E2F900
:105F600000F08CBC00212B480CF075FE234A1379FD
:105F70006FF3041313712448FDF70AFC26480CF054
:105F8000BAFB24480CF01EFF0346012B0CBF012373
:105F90000023DBB2002B08D0184A137943F010031A
:105FA00013711C48FCF71EFD0AE0144A13796FF3C5
:105FB000041313711748FCF715FD1648FCF7DAFDBA
:105FC0000E4B09221A70114B01229A7600F056BC32
:105FD000094B9B7B83F00103DBB2002B00F0508464
:105FE000064B1B78DBB20D2B18D1064B93F878319A
:105FF000812B13D1012312E018200020F40100208E
:10600000441F00202C200020141F0020C01D002051
:10601000F4050020A81E00206C1E00200023002B89
:1060200040F08884A74B1B78DBB20D2B06D1A64B22
:1060300093F87831812B01D0012300E00023002B5D
:1060400002D0A148FDF73CFB9E4B1B78DBB20B2B2B
:106050000CBF01230023DBB2002B25D09B480DF0A1
:106060001BF9984B5B68C3F30103DBB2022B08D129
:10607000944B5B68C3F38103DBB2032B01D1012393
:1060800000E00023002B0FD08E4A13796FF38303B7
:1060900013718C4B5B68C3F38103DBB21A468C4BE4
:1060A0009A708C4B0022DA81864B1B78DBB20E2B68
:1060B0000CBF01230023DBB2002B02D08648FDF782
:1060C000E7FF804B1B78DBB2092B09D07D4B1B7897
:1060D000DBB20C2B04D07B4B1B78DBB20D2B01D138
:1060E000012300E00023002B12D0764B1B78DBB29B
:1060F000092B0CBF01230023DBB2002B02D0774811
:106100000CF04CFE7548FCF76DFC7448FCF732FD52
:106110006C4B1B78DBB20A2B14BF01230023DBB2CC
:10612000002B00F0AD8301216C480CF094FD674812
:10613000FDF72EFB6A480CF0DEFA68480CF042FED0
:106140000346012B0CBF01230023DBB2002B08D038
:106150005C4A137943F0100313716048FCF742FC6A
:106160000AE0584A13796FF3041313715B48FCF784
:1061700039FC5A48FCF7FEFC524B0A221A70554B68
:1061800001229A767CE3574B9B7B83F00103DBB2C1
:10619000002B00F077834B4B1B78DBB20E2B0CBF30
:1061A00001230023DBB2002B02D04B48FDF770FF28
:1061B000444B1B78DBB2092B09D0424B1B78DBB276
:1061C0000A2B04D03F4B1B78DBB20C2B01D10123EF
:1061D00000E00023002B1AD03A4B1B78DBB2092BCE
:1061E00002D00A2B04D007E03C480CF0D7FD03E0B6
:1061F0003A480CF0D3FD00BF3848FCF7F3FB3748B2
:10620000FCF7B8FC2F4A13796FF3041313712D4B6D
:106210001B78DBB20D2B06D12B4B93F87831812BF9
:1062200001D0012300E00023002B07D02648FDF712
:1062300047FA244A13796FF304131371214B1B7827
:10624000DBB20D2B06D1204B93F87831812B01D195
:10625000012300E00023002B07D01B480CF002FFB5
:1062600001211A480DF05EF80CE31848FDF790FA8A
:10627000144B5B68C3F30013DBB2194613480DF0EF
:1062800051F817480CF037FA0E4B0B221A700F48D2
:106290000DF025F80F4B00229A76F3E2114B9B7B11
:1062A00083F00103DBB2002B00F0EE82054B1B787C
:1062B000DBB20D2B18D1044B93F87831812B13D11D
:1062C000012312E0F40100202C200020141F0020E4
:1062D000F4050020C01D0020441F0020A81E00203F
:1062E0006C1E0020182000200023002B40F0248387
:1062F0009C4B1B78DBB20D2B06D19B4B93F878316E
:10630000812B01D0012300E00023002B02D096480E
:10631000FDF7D6F9934B1B78DBB20B2B0CBF012397
:106320000023DBB2002B25D090480CF0B5FF8D4B3D
:106330005B68C3F30103DBB2022B08D1894B5B68B6
:10634000C3F38103DBB2032B01D1012300E000235F
:10635000002B0FD0834A13796FF383031371814BA2
:106360005B68C3F38103DBB21A46814B9A70814BA1
:106370000022DA817B4B1B78DBB20E2B0CBF012392
:106380000023DBB2002B02D07B48FDF781FE754B6A
:106390001B78DBB2092B0CBF01230023DBB2002BDF
:1063A00002D07648FCF71EFB6E4B1B78DBB20A2B43
:1063B00004D06C4B1B78DBB20D2B01D1012300E024
:1063C0000023002B05D06D48FCF70CFB6B48FCF755
:1063D000D1FB002169480CF03EFC624B1B78DBB21C
:1063E0000C2B14BF01230023DBB2002B0ED063481B
:1063F000FCF7F8FA5D48FDF7CBF961480CF06EF94F
:10640000584B0C221A705B4B01229A76554A13792D
:106410006FF304131371574B00229A82554B0022DD
:10642000DA8131E2574B9B7B83F00103DBB2002B17
:1064300000F02C824B4B1B78DBB20B2B0CBF0123E3
:106440000023DBB2002B25D048480CF025FF454B3C
:106450005B68C3F30103DBB2022B08D1414B5B68DD
:10646000C3F38103DBB2032B01D1012300E000233E
:10647000002B0FD03B4A13796FF383031371394B11
:106480005B68C3F38103DBB21A46394B9A70394B10
:106490000022DA81334B1B78DBB20E2B0CBF0123B9
:1064A0000023DBB2002B02D03348FDF7F1FD2F486B
:1064B000FDF76EF92B4B1B78DBB20D2B14BF0123BC
:1064C0000023DBB2002B5FD0264B1B78DBB2092BFD
:1064D00009D0244B1B78DBB20C2B04D0214B1B784A
:1064E000DBB20A2B01D1012300E00023002B05D0F1
:1064F0002248FCF777FA2148FCF73CFB194B0D22A8
:106500001A7002211D480CF0A6FB1D480CF0F3F890
:1065100015480CF027FD0023FB710023BB71BB79EC
:106520000F2B12D8BB7919460F480CF064FE0346B6
:10653000012B0CBF01230023DBB2002B01D0012370
:10654000FB71BB790133BB71E9E7074B93F87831F5
:10655000812B47D1FB79002B44D00348FCF708FD81
:1065600040E000BFF40100202C200020141F002078
:10657000F4050020C01D0020441F0020A81E00209C
:106580006C1E002018200020AD48FCF7F1FCAC4840
:106590000CF05FFE0346002B14BF01230023DBB287
:1065A000002B03D00021A6480CF03FFEA44B93F82B
:1065B0007831812B16D1A24B93F87931002B11D170
:1065C0000121A0480CF0AEFE9D480CF0A8FD03464A
:1065D0001C469B480CF002FE0346012221469948C6
:1065E000FDF758FC984BDB899BB27B807B889AB285
:1065F000954BDA81944B01229A7647E1934B9B7B32
:1066000083F00103DBB2002B00F04281904B1B783A
:10661000DBB20B2B0CBF01230023DBB2002B25D0F8
:1066200088480CF039FE8A4B5B68C3F30103DBB288
:10663000022B08D1864B5B68C3F38103DBB2032BCB
:1066400001D1012300E00023002B0FD0804A1379F1
:106650006FF3830313717E4B5B68C3F38103DBB27B
:106660001A467C4B9A70784B0022DA81784B1B7863
:10667000DBB20D2B06D1724B93F87831812B01D10F
:10668000012300E00023002B40F05881704B1B7861
:10669000DBB20D2B06D16A4B93F87831812B01D0F8
:1066A000012300E00023002B02D06548FDF708F825
:1066B000674B1B78DBB20E2B0CBF01230023DBB230
:1066C000002B05D0624A13796FF304131371DFE0D6
:1066D0005F4A13796FF3041313715F48FCF74AFAAA
:1066E00000215D480CF0B7FA594B0E221A7055483C
:1066F000FDF74EF859480BF0FEFF5948FDF746FDEF
:10670000C6E0534B1B78DBB20E2B06D0504B1B78E8
:10671000DBB20B2B01D0012300E00023002B5FD064
:106720004A4B9B7B83F00103DBB2002B25D0484B07
:106730001B78DBB2092B04D0454B1B78DBB20A2B4C
:1067400001D1012300E00023002B12D042480CF0BD
:1067500025FB4148FCF746F93D4B5B68C3F300134A
:10676000DBB283F00103DBB2002B02D03A48FCF726
:1067700001FA3648FEF7FCF98CE034480CF071FE63
:10678000334B1B78DBB20C2B14BF01230023DBB28D
:10679000002B7FD030480BF0A0FB0346002B05D127
:1067A0002D480CF00FFB0346002B01D0012300E025
:1067B0000023002B08D0264A137943F010031371ED
:1067C0002548FCF70FF965E0214A13796FF30413AC
:1067D00013712148FCF706F91F48FCF7CBF959E083
:1067E00018480CF0B3FD034683F00103DBB2002B25
:1067F00005D0174A13796FF30413137104E0144A98
:10680000137943F010031371114B1B78DBB20E2B7D
:106810000CBF01230023DBB2002B3BD00C4B93F8C1
:106820009933DBB2002B0CBF01230023DBB21A46E5
:10683000074B83F899232DE000BF2CE000BF2AE02E
:106840002C200020141F0020C01D00201820002034
:10685000F4010020F4050020A81E00206C1E00207A
:10686000441F002000BF16E000BF14E000BF12E08C
:1068700000BF10E000BF0EE000BF0CE000BF0AE068
:1068800000BF08E000BF06E000BF04E000BF02E078
:1068900000BF00E000BF2B4B1B78DBB20D2B06D1F5
:1068A000294B93F87831812B01D1012300E000239B
:1068B000002B1ED024480CF091FC034619462248B8
:1068C0000CF07BFC0346C3F30103DBB21C461E48FD
:1068D0000CF084FC034619461B480CF06EFC034682
:1068E000C3F38103DBB21A4621461848FAF7A0FC2D
:1068F0001DE0144B1B78DBB20D2B06D1124B93F825
:106900007831832B01D1012300E00023002B0ED12D
:106910000C4B5B68C3F30103DBB21946094B5B68A0
:10692000C3F38103DBB21A460848FAF781FCFEF78D
:1069300001FE04E000BF02E000BF00E000BF0C3732
:10694000BD4690BDF40100202C2000206C1E0020CC
:1069500080B500AF404B00221A70404B00221A81D4
:106960003F4B93F87831812B02D13D48FCF700FB77
:106970003C480BF092FB3C480BF090F93B480BF085
:1069800073FC3B480BF0A7FC3A480BF002FA3A487C
:106990000BF004FF39480CF069FC3848FCF7F8FEAE
:1069A0002F480CF063FA314B2F4A9A604FF4806203
:1069B00000212A480EF03BFA284B012283F8E022FE
:1069C000264B0B221A702E4B0B221A70FEF7F2FE8A
:1069D000224A13796FF301031371204A13796FF37D
:1069E000830313711D4B5B68C3F30103DBB21946CC
:1069F0001A4B5B68C3F38103DBB21A461C48FAF7F3
:106A000017FC164A1379042161F347131371134AD3
:106A100013796FF3041313711A4B00221A70194B78
:106A200000225A70174B00229A7011480BF063FE37
:106A300011480CF004F9144B00221A70134B002279
:106A40001A70134B00221A700B480CF0DBF90B483C
:106A5000FDF774FA00BF80BD782C0020F4010020FF
:106A60002C200020C01D0020DC1D0020601E002006
:106A70006C1E0020941E0020A81E0020141F002061
:106A8000792C0020F40500207A2C00207B2C00209B
:106A90007C2C002080B584B000AF0346FB715448C5
:106AA000FCF7E0F85348FCF7B7FB5348FEF79CF8B7
:106AB0005248FCF787FE524B00221A70514B93F854
:106AC000D130022B02D14F48FDF7E2FA4E4B1B7832
:106AD000DBB20D2B0BD1474B93F87831812B04D0CF
:106AE000444B93F87831012B01D1012300E00023BE
:106AF000002B02D03F48FCF73BFA434B1B78DBB23C
:106B00000E2B0BD13F4B93F8D130012B04D03D4BD2
:106B100093F8D130002B01D1012300E00023002B9A
:106B200007D03A480BF0B9FA394B0B221A70FEF72E
:106B300041FE344B93F8C630002B1CD0354BDB683C
:106B4000FB60314BD3F89C33324AD3602E4AFB684A
:106B5000C2F89C33304B1868012300222D4904F001
:106B6000B9F90346002B14BF01230023DBB2002B2D
:106B700001D0FEF765F94222284929480EF049F96B
:106B8000254B1868FB795B0001331A4602231E4926
:106B900004F0A0F90346002B14BF01230023DBB24D
:106BA000002B01D0FEF74CF94FF4806216491D48C6
:106BB0000EF02FF9144B93F89833DBB2002B14BF6F
:106BC00001230023DAB20F4B83F8C5200D4B0022BE
:106BD00083F8C6200A4B01221A70134B01221A7047
:106BE000124B00221A7000BF1037BD4680BD00BF97
:106BF000A81E00202C20002018200020141F002098
:106C00007F2C0020441F0020F4010020C01D002024
:106C1000792C002050280020000100207C1B00203F
:106C2000D6040020F41600208C2C0020822C00209A
:106C300080B5ADF5836D00AF0246FB1D1A70A94B00
:106C400000221A70A84B01221A70A84B1868FB1D6D
:106C50001B785B0001331A4607F10C01022304F094
:106C600081F80346002B14BF01230023DBB2002B65
:106C700001D0FEF7E5F807F10C0393F8E032012BA1
:106C800008D19B4B1B69C3F34333DBB2022B01D00A
:106C9000012300E00023002B00F0F580FFF758FEF1
:106CA00007F10C031B78C7F8143407F10C031B79A8
:106CB000C3F30013DBB2C7F8103407F10C021379E9
:106CC0006FF30413137107F10C034FF4806219463C
:106CD00088480EF09EF88848FCF7A4F88748FCF72F
:106CE0006BFB8748FDF7B0FF8648FCF7D1FDD7F86E
:106CF00014340B2B07D0D7F81434DAB2824B1A7045
:106D0000FEF758FD09E0804B09221A70FEF752FD8C
:106D10007D4B0B221A70FEF74DFDD7F814340E2B65
:106D200009D1794B0B221A70FEF744FD764B0E22E7
:106D30001A70FEF73FFDD7F814340D2B09D1724BB2
:106D40000B221A70FEF736FD6F4B0D221A70FEF7FC
:106D500031FDD7F81034002B08D0664B5B68C3F3C5
:106D60000013DBB2002B01D1012300E00023002B34
:106D700004D0654B01221A70FEF71CFDD7F81434BD
:106D8000092B43D107F10C031B79C3F34213DBB288
:106D9000A7F80E34B7F80E34042B05D05A4B08224E
:106DA0001A70FEF707FD04E0574B07221A70FEF732
:106DB00001FDB7F80E34052B26D801A252F823F0B6
:106DC000D96D0000E16D0000E96D0000F16D00007B
:106DD000F96D0000016E00004B4B00221A7013E0A9
:106DE000494B05221A700FE0474B06221A700BE040
:106DF000454B07221A7007E0434B08221A7003E044
:106E0000414B09221A7000BFFEF7D4FCD7F81434A6
:106E10000C2B13D13C4B09221A70FEF7CBFC3A4BDA
:106E200001221A70FEF7C6FC374B01221A70FEF7DA
:106E3000C1FC354B0C221A70FEF7BCFCD7F8143499
:106E40000A2B03D0D7F81434092B0DD1D7F81034FE
:106E5000002B09D02C4B01221A70FEF7ABFC2A4BF9
:106E600001221A70FEF7A6FCFEF764FB4FF4806265
:106E7000204926480DF0CDFF254B01221A701A4BF0
:106E800000221A7011E0FFF763FD224B01221A70F5
:106E9000FEF750FBFB1D1B781846FFF7FBFD1C4B54
:106EA00001221A70104B00221A70124B93F898337B
:106EB000DBB2002B14BF01230023DAB2164B83F898
:106EC000C520154B002283F8C620144AFB1D1B78F1
:106ED0001370044B01221A7000BF07F58367BD468B
:106EE00080BD00BF7F2C0020822C002000010020EC
:106EF00000F00F40F4010020A81E00202C200020EC
:106F000018200020141F0020792C0020F4160020E7
:106F10008C2C0020832C0020441F0020842C002077
:106F200080B483B000AF0346FB71044AFB79D37091
:106F300000BF0C37BD465DF8047B7047007006400B
:106F400080B483B000AF0346FB71074B9B79DAB284
:106F50000549FB791343DBB28B7100BF0C37BD468B
:106F60005DF8047B704700BF0070064080B400AF3E
:106F7000064B9B79DBB2054A43F02003DBB29371E9
:106F800000BFBD465DF8047B704700BF007006403F
:106F900080B400AF064B9B79DBB2054A23F0200397
:106FA000DBB2937100BFBD465DF8047B704700BF44
:106FB0000070064080B500AF0A4B1B78022B0BD146
:106FC000094B01221A70074B01221A70002200217E
:106FD00006480DF0F2F902E0054B00221A7000BFDE
:106FE00080BD00BF882C0020872C00200070064048
:106FF000822C002080B500AF03480DF00FFA034B40
:1070000000221A7000BF80BD00700640872C00204F
:1070100080B584B000AF504B1A78504B1B789A4221
:1070200000F096804D4B1B785A1CD1B24B4A117020
:1070300019464B4A0B469B000B445B001A443B1D10
:107040001068516803C312891A807B79042B7FD1A1
:107050003B7A013B162B76D801A252F823F000BFF1
:10706000BD700000DD700000477100004771000036
:107070004771000047710000477100004771000030
:107080004771000047710000477100004771000020
:107090004771000047710000477100004771000010
:1070A0004771000047710000477100003371000014
:1070B00047710000FD7000003B710000294B1B78F8
:1070C000002B42D0284B1B78002B3ED07B7A1E2B06
:1070D0003BD87B7A1846FFF7ABFD36E0214B1B7897
:1070E000002B34D0204B1B78002B30D07B7A1E2B0A
:1070F0002DD87B7A1846FFF7CDFC28E0194B0122EA
:107100001A701A4B1B78002B0DD0422218491948CF
:107110000DF07FFE4FF48062174918480DF079FE9C
:10712000124B00221A70104B01221A70FEF702FA5D
:107130000EE00D4B01221A700AE00A4B00221A7071
:10714000FEF7F8F904E000BF02E000BF00E000BF76
:1071500000BF1037BD4680BD8A2C00208B2C00203C
:10716000F40C0020832C0020802C0020822C002096
:107170007C1B0020D6040020F4010020F41600201F
:1071800080B582B000AFAD4B4FF400421A82AC4ADA
:10719000D2F8803043F4F073C2F88030A84AB2F8D5
:1071A00040306FF38A23A2F84030A54AB2F840304D
:1071B00043F40063A2F84030FFF7CAFBA14B002262
:1071C0001A70A14B01221A70A04B00221A70A04B1A
:1071D0001868012300229F4903F0C4FD0346002BD9
:1071E00014BF01230023DBB2002B01D0FDF728FEE2
:1071F000984B1B68984A934206D1964B9B68B3F50F
:10720000087F01D0FDF756FE8D4B1B69C3F3433356
:10721000DBB2012B09D18A4BD3F81031C3F3806361
:10722000DBB2002B01D0012300E00023002B17D09C
:10723000834B1B69C3F34333DBB2012B07D0804B75
:10724000D3F81031C3F38063DBB2002B01D00123EC
:1072500000E00023002B03D07E4B00221A60E7E7FA
:107260007C4B1B687C4A93427ED07A4B7A4A1A60E8
:10727000784B4FF408729A60764B00225A60754B37
:10728000764ADA607648FBF7EDFC7648FBF7C4FFF8
:107290007548FDF7A9FC7548FCF794FA00237B605C
:1072A0007B681E2B20DC7B68714A02FB03F33F33B3
:1072B0001A46704BC3F89C23654B18687B685B00CB
:1072C00001331A4602236B4903F004FE0346002BE8
:1072D00014BF01230023DBB2002B01D0FDF7B0FD6A
:1072E0007B6801337B60DBE700233B603B680F2B4F
:1072F00018DC614A3B6840F2145122F813105E4AD0
:107300003B6810334FF6FF7122F813105A4A3B685E
:1073100010339B0013444FF07E521A603B680133D8
:107320003B60E3E74A4B186801234C4A524903F09B
:10733000D1FD0346002B14BF01230023DBB2002B39
:1073400001D0FDF77DFD424B186801230022414921
:1073500003F0C0FD0346002B14BF01230023DBB262
:10736000002B01D0FDF76CFD394B186801233B4A17
:10737000414903F0F7FC0346002B14BF012300230F
:10738000DBB2002B01D0FDF75BFD2D4B1B69C3F376
:107390004333DBB20F2B09D1294BD3F81031C3F3A0
:1073A0008063DBB2002B01D0012300E00023002B1F
:1073B00017D0234B1B69C3F34333DBB20F2B07D02A
:1073C0001F4BD3F81031C3F38063DBB2002B01D025
:1073D000012300E00023002B03D0284B01221A7068
:1073E000E7E7264B1B78002B11D025480CF0D4F88A
:1073F000FDF7F6FD1E20FFF71BFCFEF79BF80F487C
:10740000F9F7A2FB00211F480CF0EBF80EE01E205C
:10741000FFF70EFCFEF78EF80848F9F795FB002100
:1074200018480CF0DEF816480CF0B6F8164B01229E
:107430001A7000BF0837BD4680BD00BFC01D0020C8
:1074400000F00F40832C00208C2C0020822C002088
:1074500000010020502800204B45454EBFC3C90104
:10746000A81E00202C20002018200020141F00201F
:107470001C4E0E00F4010020C01B00208E2C0020AA
:1074800000600340007003407F2C002080B500AFF7
:10749000574B00229A72574B1B69C3F34333DBB23D
:1074A000002B0CBF01230023DBB2002B2AD0524B50
:1074B0001B78002B20D0514B1B78002B0CBF0123D5
:1074C0000023DBB21A464D4B1A704C4B1B78002B35
:1074D00015D04B4B1B78002B11D0422249494A480A
:1074E0000DF097FC4FF48062484949480DF091FC3B
:1074F000434B00221A7002E01E20FFF7CBFAFEF782
:1075000019F873E0414B1B78DBB2093B052B64D8BB
:1075100001A252F823F000BF317500003D75000054
:10752000497500008575000091750000AB7500007D
:1075300038480BF059FCFDF7FDFF4EE035480BF0E5
:1075400053FCFDF7F7FF48E02A4B1B69C3F34333B5
:10755000DBB20B2B0CBF01230023DBB2002B39D095
:107560002D480BF083FE2C48FCF712F9274B5B6883
:10757000C3F30013DBB2194627480BF0D3FEFDF727
:10758000D9FF27E023480BF02FFCFDF7D3FF24E0C1
:1075900022480BF06BFC21480BF0E4FC1F48FBF782
:1075A0002FFD1E48FBF7E4FC17E0124B1B69C3F3E9
:1075B0004333DBB20E2B0CBF01230023DBB2002BC5
:1075C0000AD01748FCF70EFD1548FCF7DFFDFDF764
:1075D000B1FF01E000BF00E000BF124B9B7B002B1E
:1075E00004D010480BF0ADFFFDF7A4FF00BF80BD35
:1075F000C01D002000F00F40802C0020832C0020B4
:10760000822C00207C1B0020D6040020F4010020E6
:10761000F4160020A81E0020141F00202C2000209B
:10762000441F00201820002090B583B000AF0DF05B
:10763000D8FB0DF0AAFA0DF07AFB954B00221A70D8
:10764000934B00229A70924B9B78DBB2904A63F086
:107650003F03DBB29370FFF79BFC8E4B02221A7044
:1076600000218D480BF0F5FF8C4B18680023052294
:10767000002101F081FE0CF03BFA0CF039FA0CF01D
:1076800037FA864B1B68184603F0E4FD0346002BCF
:1076900014BF01230023DBB2002B01D0FDF7D0FB88
:1076A0007E4B1B68184603F025FD0346002B14BFD4
:1076B00001230023DBB2002B01D0FDF7C1FB774B88
:1076C0001B68184603F0C6FD0346002B14BF0123B8
:1076D0000023DBB2002B01D0FDF7B2FB0DF021FB44
:1076E0006E4B1B68D3F888326D4A93420ED96B4BB0
:1076F0001B68D3F88C32B3F5007F07D1674B1B684A
:10770000184603F003FB0346002B01D0012300E0E1
:107710000023002B01D0FDF793FBFFF731FD614BF8
:107720001B78002B5AD0604B1B78002B1DD140F2E8
:10773000E1225E495E480DF05EFB0346002B14BF5C
:1077400001230023DBB2002B0FD0574B01221A700C
:10775000584B1B78002B06D0574B1B78002B02D0C0
:10776000FFF728FC01E0FDF7E5FE0023FB71FB7944
:107770000F2B30D84C4B1B78002B28D1FB794F4A6C
:1077800032F813301946FB79494A03F5B8735B00A8
:1077900013445B889BB2CB1A18460DF028FB0346B6
:1077A000282BCCBF01230023DBB2002B0FD03E4B94
:1077B00001221A703F4B1B78002B06D03E4B1B78E2
:1077C000002B02D0FFF7F6FB01E0FDF7B3FEFB79DB
:1077D0000133FB71CBE7334B00221A70FFF718FC23
:1077E000374B9B7ADBB2012B0CBF01230023DBB2AA
:1077F000002B01D0FFF74AFE324B1B69C3F3433322
:10780000DBB2052B14D12A4B1B78DBB20E2B0FD029
:107810002D4B9B7B83F00103DBB2002B08D0244B64
:107820005B68C3F38103DBB2032B01D0012300E0CB
:107830000023002B4ED01E4B1B78DBB20B2B14BF4A
:1078400001230023DBB2002B0CD0204B1B7883F0EC
:107850000103DBB2002B05D01B48FDF735F91B4BAC
:1078600001221A70124B1B899BB2DB439BB2002290
:10787000194613480AF049FC0D4B1B899BB20122A3
:1078800019460F480AF041FC114B01221A703BE0E7
:1078900000700640882C002000D00040000100202D
:1078A000BEC3C901812C0020822C0020F4160020C8
:1078B000F4010020802C0020832C0020381B0020A5
:1078C000C01D002000F00F40182000207E2C00205A
:1078D0007D2C00209C4B1B78002B15D09B4B1B89CB
:1078E0009BB21846FAF7A6F899480AF0D6FB994BCE
:1078F0001B78002B05D09848FDF70AF9954B00221C
:107900001A70914B00221A7094480AF023FA034629
:10791000002B3FF404AF91480AF0FDF90346904A6A
:1079200013608D4B9B7B002B11D08D4B1B7803F08C
:107930001003DBB2002B3FF4F2AE894B1B78C3F38C
:107940000303DBB219468448FDF72EF9E7E6854BC1
:107950001B69C3F34333DBB2052B0DD17B4B1B7883
:10796000DBB20E2B08D07C4B9B7B83F00103DBB298
:10797000002B01D0012300E00023002B19D0734B12
:107980001B899BB21AB2764B1B78C3F30013DBB290
:107990001946734B1B78C3F30303DBB201FA03F3FD
:1079A0001BB253401BB29AB2684B1A81664B01223C
:1079B0001A706B4B1B7803F01003DBB2002B0CD05A
:1079C00069480AF070FC0346002B06D0674B93F819
:1079D000D130012B01D1012300E00023002B02D084
:1079E0006248FCF7FBFB594B1B78DBB20B2B04D036
:1079F000564B1B78DBB20E2B01D1012300E0002394
:107A0000002B4ED0514B1B78DBB20E2B13D1574BB2
:107A100093F8D130052B0ED153480AF044FC0346AD
:107A2000002B08D14F4B1B69C3F34333DBB2002B50
:107A300001D1012300E00023002B04D04B480BF0C0
:107A4000B1FCFDF777FD414B1B78DBB20E2B18D153
:107A5000464B93F8D130032B04D0444B93F8D130EC
:107A6000042B0ED140480AF01EFC0346002B08D020
:107A70003C4B1B69C3F34333DBB2002B01D1012321
:107A800000E00023002B07D03848FCF7EDFA384817
:107A9000FBF77EFEFDF74EFD314B19683448FCF7CD
:107AA000C9F82A4B1B78DBB20D2B0CBF0123002336
:107AB000DBB2002B00F0AA812E4B93F87831812B9A
:107AC0002ED12C4B93F87931002B02D0012B06D00C
:107AD0009CE1234B19682648FCF7ACF896E1204B53
:107AE0001B7803F01003DBB2002B0CD01C4B1B786F
:107AF000C3F30303DBB219461F48FAF7ADF91D487B
:107B0000FBF72CFB82E1164B1B78C3F30303DBB2BC
:107B1000194619480AF0E6FE1648FBF71FFB75E107
:107B2000144B93F87831832B28D10D4B1B78C3F37A
:107B30000303DBB219460F480BF05DFB0346002B35
:107B40001CD001231BE000BF7D2C0020F40100208D
:107B5000C01D00207E2C002018200020DC1D0020ED
:107B6000F805002000F00F40601E0020441F002098
:107B7000141F00202C200020A81E00200023002B12
:107B800000F04481AE4B1B7803F01003DBB2002BF6
:107B900000F08F80AB4B93F88E31002B23D1A84B94
:107BA0001B78C3F30303DBB27B71A54B1B78C3F3D4
:107BB0000303DBB21946A4480AF011F9A2480AF0FF
:107BC0008CF90346012B8CBF01230023DBB2002B71
:107BD00006D001219C480AF09CF90346BB7195E050
:107BE000FF23BB7192E0002198480AF092F9034606
:107BF0001A46934B1B78C3F30303DBB29A420CBFC4
:107C000001230023DBB2002B04D0FF237B71FF2371
:107C1000BB717BE08A4B1B78C3F30303DBB27B7140
:107C2000874B1B78C3F30303DBB2194687480AF07E
:107C3000D6F8002185480AF06CF903461A4601235C
:107C400003FA02F1824BDB8A9BB21AB20BB21343E6
:107C50001BB29AB27E4BDA827C480AF03EF90346A8
:107C6000012B8CBF01230023DBB2002B1ED001218E
:107C700076480AF04EF90346BB71012173480AF0B9
:107C800048F903461A4601239340D943704BDB8AD7
:107C90009BB21AB20BB213401BB29AB26C4BDA828F
:107CA000BB79194669480AF0CFF82FE0FF23BB7172
:107CB0002CE0644B93F88E31002B23D1604B1B7862
:107CC000C3F30303DBB2BB715D4B1B78C3F3030348
:107CD000DBB219465C480AF0B7F85B480AF0FDF8D9
:107CE0000346002B14BF01230023DBB2002B06D078
:107CF000002155480AF00DF903467B7106E0FF2389
:107D00007B7103E0FF237B71FF23BB71BB79FF2BEA
:107D100024D04C4BFF2283F87A214E48FAF72AFFF1
:107D20004C480AF09DFD4C48FBF732FD484B1B8A3E
:107D30009BB223F480739AB2454B1A82444B1B8A40
:107D40009BB223F480639AB2414B1A82404B1B8A48
:107D50009BB223F00E039AB23D4B1A827B79FF2B24
:107D600054D07B79194637480BF0FCF90346002BB9
:107D700002D0012B1BD049E0324B002283F87A213C
:107D80007B7919462F480BF0DCF9034619467B79BD
:107D900001223148FCF77EF8FDF7CCFB2C4B1B8A07
:107DA0009BB243F480639AB2294B1A822EE0254B92
:107DB000012283F87A212748FAF714FE7B791946C5
:107DC00020480BF0FAF90346C3F30103DBB21C466B
:107DD0007B7919461B480BF0F0F90346C3F3810386
:107DE000DBB21A4621461D48F9F722FA7B7919467B
:107DF0001448FBF7F7F9FDF79DFB154B1B8A9BB267
:107E000043F480739AB2124B1A8200BF144B1B7852
:107E1000DBB20C2B0CBF01230023DBB2002B3BD0C9
:107E20000F4B5B68C3F30013DBB283F00103DBB2DB
:107E3000002B17D0024B19680748FBF7FBFE2BE01D
:107E4000F80500202C200020A7210020BB210020C5
:107E5000C01D0020A81E0020141F00206C1E002042
:107E6000F4010020244B1B7803F01003DBB2002B3D
:107E700009D0214B1B78C3F30303DBB219461F481B
:107E8000F9F7EAFF08E01C4B1B78C3F30303DBB2EE
:107E900019461A480AF026FD194B1B78DBB20A2B4B
:107EA00004D0174B1B78DBB2092B01D1012300E072
:107EB0000023002B3FF433AC0F4B1B7803F010036F
:107EC000DBB2002B09D00C4B1B78C3F30303DBB2EE
:107ED00019460A48F9F7C0FF08E0074B1B78C3F3BF
:107EE0000303DBB2194605480AF0FCFC044B1B787F
:107EF000DBB20A2B13E400BFF8050020A81E002007
:107F0000F401002080B500AF1C4B1B69C3F3433361
:107F1000DBB2002B14BF01230023DBB2002B27D0E0
:107F2000164B1B69C3F34333DBB21A46144B1A706A
:107F3000124B1B69C3F34333DBB20C2B0CBF012381
:107F40000023DBB2002B13D00E4A137943F0100349
:107F500013710C4B1B78DBB20C2B0CBF01230023DD
:107F6000DBB2002B02D00848FAF73CFDFDF7E2FA3D
:107F7000012106480BF035FB00BF80BD00F00F402B
:107F8000782C0020F4010020A81E0020007003407F
:107F900080B582B000AF274805F03AFA78607B6878
:107FA00003F40033002B27D0224B1B69C3F340435B
:107FB000DBB283F00103DBB2002B0BD01E4B1B782E
:107FC000DBB283F00103DBB2002B15D01B48FCF7BA
:107FD000A1F911E01A4B1B78DBB283F00103DBB28D
:107FE000002B09D01548FCF791FC134B01221A70A5
:107FF000022114480BF0F5FA7B6803F4F033002BF0
:108000000CD0114B1B7883F00103DBB2002B05D0A1
:108010000E4B1B78002B01D0FFF774FF79680548E1
:1080200005F00EFABFF34F8F00BF00BF0837BD4603
:1080300080BD00BF00F00F407A2C002018200020E7
:108040007B2C0020007003408E2C00207F2C002011
:1080500080B500AF0122012116480BF0ADFA0121D5
:1080600014480BF0DAFA144B1B69C3F34333DBB249
:10807000002B14BF01230023DBB2002B15D00E4BC5
:108080001B69C3F34333DBB21A460C4B1B78DBB2DC
:108090009A420CBF01230023DBB2002B07D0074B11
:1080A0001B78DAB2064B1A7001E0FDF783FB00BFC4
:1080B00080BD00BF0070034000F00F40782C00200E
:1080C000792C002080B500AF0122022105480BF079
:1080D00073FA022103480BF0A0FA034B00221A7036
:1080E00000BF80BD007003407A2C002080B582B0B4
:1080F00000AF012200215E480BF05EFA5D4B1B7859
:1081000083F00103DBB2002B00F0AD805A480AF087
:10811000CAF80346BB80594B1B78DBB20E2B0BD140
:10812000574B93F8D130022B06D0554B93F8D130F2
:10813000012B01D0012300E00023002B00F08D80F3
:10814000BB88002B02D14F4B00221A704E4B1B698B
:10815000C3F34333DBB20E2B09D14A4B1B78DBB29E
:1081600083F00103DBB2002B01D0012300E00023E8
:10817000002B5AD0454B01229A76454B01221A70AA
:108180003F4B93F9C430022B1ED0022B29DC002B6D
:108190000ED0012B25D100224FF6FF713B4809F08C
:1081A000B4FF012248F20101384809F0AEFF18E09F
:1081B00000224FF6FF71354809F0A7FF0122012187
:1081C000324809F0A2FF0CE000224FF6FF712F4861
:1081D00009F09BFF01224FF400412C4809F095FF64
:1081E00000BF0023FB71FB790F2B39D8BA88FB79CC
:1081F00042FA03F303F00103002B12D0FB79194676
:108200001F48FCF741F8FB79002B0AD0FB790E2BB5
:1082100007D8FB790133DBB21A460E211B480AF05E
:1082200000F8FB790133FB71DDE7174B1B69C3F3E2
:1082300043330123002B13D0154B1B78002B08D0A0
:10824000002248F20101114809F05FFF104B0022A3
:108250001A700948F8F72AFD02E00748F8F726FDEA
:108260000A48F8F7B5F900BF0837BD4680BD00BF22
:10827000007003408E2C0020601E0020F4010020BE
:10828000441F00207C2C002000F00F40C01D002067
:10829000852C002084B090B400AF07F1080484E876
:1082A0000F00474B1B7883F00103DBB2002B64D037
:1082B000444B1B78C3F30303DBB207F1080232F827
:1082C00013301A11404B1A613E4B1B78C3F3030362
:1082D000DBB2103307F1080232F813301A113B4BAE
:1082E0001A63384B1B78C3F30313DBB207F10802A0
:1082F00032F813301A11364B1A61324B1B78C3F324
:108300000313DBB2103307F1080232F813301A11ED
:108310002D4B1A622B4B5B78C3F30303DBB207F1DF
:10832000080232F813301A11274B9A61254B5B78FB
:10833000C3F30303DBB2103307F1080232F8133042
:108340001A11214B9A621F4B5B78C3F30313DBB204
:1083500007F1080232F813301A111C4B9A64194BBA
:108360005B78C3F30313DBB2103307F1080232F872
:1083700013301A11154B1A621DE0164B1B781A4662
:10838000154B33F812301B11104A93640E4A936157
:108390000F4A13610C4A13610E4B1B780F4A1033BE
:1083A00032F813301B11094A1362074A9362064AD6
:1083B0001362064A136300BFBD4690BC04B0704709
:1083C0008E2C0020E401002000900B400080034030
:1083D000009003408D2C0020A00100207C1B002079
:1083E00080B500AF764B1B78DBB20D2B75D00D2B13
:1083F00000F3BA800A2B02DC092B03DAB4E00C2B61
:108400003DD0B1E06F4BDB7A002B05D0012200217B
:108410006D480BF0A4F804E0002200216A480BF03C
:108420009EF8684B1B7B002B05D001220321664878
:108430000BF095F804E00022032163480BF08FF85D
:10844000604B5B7B002B05D0012205215F480BF0C0
:1084500086F804E0002205215C480BF080F8594BB7
:108460009B7B002B05D00122012159480BF077F8A6
:10847000A3E00022012156480BF071F89DE0514B1A
:108480009B78C3F30003DBB21A4600214E480BF081
:1084900066F84C4B9B78C3F34003DBB21A460321CA
:1084A00049480BF05CF8474B9B78C3F38003DBB281
:1084B0001A46052145480BF052F8424B9B7B002B96
:1084C00005D00122012142480BF049F875E0002255
:1084D00001213F480BF043F86FE03E4B93F87831B1
:1084E000832B41D13B4B93F87A31002B3CD0354B59
:1084F000DB7A002B05D00122002133480BF02FF846
:1085000004E00022002130480BF029F82D4B1B7BA2
:10851000002B05D0012203212B480BF020F804E0AA
:108520000022032128480BF01AF8264B5B7B002B16
:1085300005D00122052125480BF011F804E00022A6
:10854000052122480BF00BF81E4B9B7B002B05D01E
:10855000012201211E480BF002F82EE00022012129
:108560001B480AF0FCFF28E0164B9B78C3F300037E
:10857000DBB21A46002114480AF0F1FF114B9B7838
:10858000C3F34003DBB21A4603210F480AF0E7FFAA
:108590000C4B9B78C3F38003DBB21A4605210B48D2
:1085A0000AF0DDFF074B9B78C3F3C003DBB21A462A
:1085B000012107480AF0D3FF00BF00BF80BD00BF04
:1085C000F4010020E401002040F00F40C0F00F4013
:1085D00080F00F402C20002080B500AF8A4B93F92B
:1085E00003301A46884B1B78C3F30303DBB29A426D
:1085F0000BD1854B93F90730002B16D1824B9B781A
:1086000003F00103DBB2002B0FD0012201217F48D0
:108610000AF0A5FF7C4B1B78C3F30303DBB25AB20D
:10862000794BDA70784B0122DA72774BDB7A012BC7
:1086300007D90022012175480AF091FF724B0022F0
:10864000DA72714BDB7A002B05D06F4BDB7A01338A
:10865000DAB26D4BDA726C4B9B78C3F30003DBB27A
:108660005AB2694BDA71684B93F904301A46664B7B
:108670001B78C3F30313DBB29A420BD1624B93F91D
:108680000830002B16D1604B9B7803F00203DBB25D
:10869000002B0FD0012202215C480AF060FF5A4BE8
:1086A0001B78C3F30313DBB25AB2574B1A71564B04
:1086B00001221A73544B1B7B012B07D90022022184
:1086C00052480AF04CFF504B00221A734E4B1B7B52
:1086D000002B05D04C4B1B7B0133DAB24A4B1A738B
:1086E000494B9B78C3F34003DBB25AB2464B1A7234
:1086F000454B93F905301A46434B5B78C3F30303AC
:10870000DBB29A420BD1404B93F90930002B16D1C2
:108710003D4B9B7803F00403DBB2002B0FD001220A
:1087200006213B480AF01BFF374B5B78C3F303037A
:10873000DBB25AB2344B5A71334B01225A73324B6B
:108740005B7B012B07D90022062131480AF007FF85
:108750002D4B00225A732C4B5B7B002B05D02A4BF0
:108760005B7B0133DAB2284B5A73274B9B78C3F3F8
:108770008003DBB25AB2244B5A72234B93F9063072
:108780001A46214B5B78C3F30313DBB29A420BD139
:108790001D4B93F90A30002B16D11B4B9B7803F02D
:1087A0000803DBB2002B0FD00122022119480AF086
:1087B000D6FE154B5B78C3F30313DBB25AB2124BF0
:1087C0009A71114B01229A730F4B9B7B012B07D996
:1087D000002202210F480AF0C2FE0B4B00229A73BE
:1087E000094B9B7B002B05D0074B9B7B0133DAB2F7
:1087F000054B9A73044B9B78C3F3C003DBB25AB2A8
:10880000014B9A7200BF80BDE401002040F00F4090
:10881000C0F00F4080F00F40F0B595B00EAF0023D0
:10882000FB750023FB75FB7D0F2B15D8FA7DFB7DB7
:10883000A74931F81210A74A22F81310FA7DFB7DE0
:10884000A349103231F81210A24A103322F8131043
:10885000FB7D0133FB75E6E79F4BB3F840209D4B52
:10886000A3F840209D4B1B78DBB20E2B10D19C4B04
:1088700093F8D130032B09D0994B93F8D130042BC6
:1088800004D0974B93F8D130052B01D1012300E0A0
:108890000023002B00F0B681914B93F8C630002BDB
:1088A00002D0904B1B6802E08C4BD3F89C33FB60EA
:1088B0008B4B93F8D130032B60D189480AF08AFDA5
:1088C000B0EE407A864BD3ED337A77EE277A844B3D
:1088D000C3ED337A824BD3ED337AB1EE0C7AF4EEFA
:1088E000C77AF1EE10FA0DDB7D4BD3ED337AB1EEA2
:1088F0000C7A77EEC77A7A4BC3ED337A784B012244
:1089000083F8D020764BD3ED337AFCEEE77AC7EDCF
:10891000017A3B79DAB2724B83F8C820704B93F836
:10892000D030002B2AD0704B18686C4BD3F8A4338E
:108930005A1C6A49C1F8A423FA681A4401236B49F6
:1089400002F010FA0346002B14BF01230023DBB210
:10895000002B01D0FCF774FA604BD3F8A0235F4BD7
:10896000D3F8A433B3FBF2F102FB01F29B1A5B4A8A
:10897000C2F8A4335A4B002283F8D020584B93F806
:10898000D130042B77D156480AF024FDB0EE407A5E
:10899000534BD3ED337A77EEC77A514BC3ED337A2D
:1089A0004F4BD3ED337AF5EEC07AF1EE10FA0DD5D8
:1089B0004B4BD3ED337AB1EE0C7A77EE877A484B96
:1089C000C3ED337A464B012283F8D020444BD3EDDC
:1089D000337AFCEEE77AC7ED017A3B79DAB2404BA5
:1089E00083F8C8203E4B93F8D030002B43D03B4B4C
:1089F000D3F8A433002B14BF01230023DBB2002BD8
:108A000019D0394B1868354BD3F8A4335A1E334963
:108A1000C1F8A423FA681A440123344902F0A2F9E8
:108A20000346002B14BF01230023DBB2002B1ED012
:108A3000FCF706FA1BE02C4B1868284BD3F8A4234C
:108A4000FB681A440123294902F08CF90346002BE4
:108A500014BF01230023DBB2002B01D0FCF7F0F997
:108A60001E4BD3F8A033013B1C4AC2F8A4331C4B65
:108A7000002283F8D0201A4B93F8C83019461C48BE
:108A80001A4A0B465B010B445B0013441946422310
:108A90001A460CF0BEF9114B93F89933DBB2002B58
:108AA00014BF01230023DBB2002B23D00023FB756E
:108AB000FB7D0F2B1ED8FA7DFB7D074931F8121084
:108AC0000B4A22F81310FB7D0133FB75F0E700BF62
:108AD000381B00207C1B0020A0010020F401002096
:108AE000441F00205C2800200001002040080020D6
:108AF000FC0500209D4E6D4606F110040FCC0FC5FD
:108B00000FCC0FC50FCC0FC523682B8096E80F0044
:108B1000FFF7C0FB964809F0C6FB0346BB82002363
:108B2000FB75FB7D0F2B27D8FB7D924A103332F863
:108B3000133040F21452934208D9FB7D012202FA0D
:108B400003F39AB2BB8A1343BB8211E0FB7D894ACF
:108B5000103332F81330B3F52F7F09D2FB7D012299
:108B600002FA03F39BB2DB439AB2BB8A1340BB8287
:108B7000FB7D0133FB75D4E7BB8A19467C4809F0BD
:108B800083FB7D4B93F8D130052B2FD1BB8A002B73
:108B900025D00023FB75FB7D0F2B0BD8FA7DFB7DC9
:108BA000744931F81210754A22F81310FB7D013315
:108BB000FB75F0E7714E6D4606F110040FCC0FC542
:108BC0000FCC0FC50FCC0FC523682B8096E80F0084
:108BD000FFF760FB674ABB8AA2F84030C1E0634BF5
:108BE000B3F84020634BA3F84020BAE0BB8A002BC7
:108BF00003D15E4BB3F8403000E0BB8A5D4AA2F877
:108C00004030AEE00023FB75FB7D0F2B31D8FB7DA0
:108C1000584A103332F8133040F2145293420DD9AF
:108C2000544BB3F84020FB7D012101FA03F39BB2C2
:108C300013439AB24F4BA3F8402016E0FB7D4D4AF8
:108C4000103332F81330B3F52F7F0ED2494BB3F8FF
:108C50004020FB7D012101FA03F39BB2DB439BB271
:108C600013409AB2434BA3F84020FB7D0133FB75C0
:108C7000CAE7404BB3F8403019463D4809F004FBC1
:108C80003F4B1B78DBB20E2B06D13B4B93F8D13018
:108C9000022B01D1012300E00023002B51D0364BE1
:108CA00093F8C530002B02D0364B1B6802E0344BE2
:108CB000D3F89C333B61304B93F8C7305A1CD1B288
:108CC0002D4A82F8C71019462F4A0B465B010B4408
:108CD0005B001344294A1846114642231A460CF0F9
:108CE00098F8254B93F8C720284BA3FB0213D11A01
:108CF00049080B4499080B46DB005B1AD31ADAB219
:108D00001D4B83F8C7201C4B93F8C730002B18D19C
:108D10001F4B18681A4BD3F8A0335A1C1849C1F8D6
:108D2000A0233A691A440123174902F0D3F80346F5
:108D3000002B14BF01230023DBB2002B01D0FCF772
:108D40007FF80E4E6D4606F110040FCC0FC50FCC08
:108D50000FC50FCC0FC523682B8096E80F00FFF7D7
:108D600099FA00BF1C37BD46F0BD00BFFC050020CE
:108D7000601E0020A0010020441F00207C1B00205A
:108D8000F40100205C2800204006002025499224A0
:108D90000001002090B583B000AF0221B44803F079
:108DA000ADFC38603A680221B14803F0E9FCB14BF0
:108DB0001B78002B00F0B9800023FB71FB790F2B8F
:108DC00000F2B080FB792C2202FB03F3AA4A1A447A
:108DD000FB79AA4931F8133007EE903AF8EE677A3A
:108DE0000A21DFEDA72AB0EE672ADFEDA61A9FED74
:108DF000A61ADFEDA60A9FEDA60A10460AF07FFC30
:108E0000FB792C2202FB03F3A24A1A44FB799B490B
:108E1000103331F8133007EE903AF8EE677A0A21F2
:108E2000DFED972AB0EE672ADFED9B1A9FED9B1AC4
:108E3000DFED960A9FED960A10460AF060FCFB797A
:108E40002C2202FB03F38C4A1A44FB798B4931F83C
:108E5000133007EE903AF8EE677AB0EE670A1046E4
:108E60000AF0E8FCF0EE407AFB79FCEEE77A17EEC8
:108E7000902A91B28A4A22F81310FB792C2202FB25
:108E800003F3844A9C18FB797C4A103332F8133080
:108E90001A46FB7919461046FCF746F8034607EEDA
:108EA000903AF8EE677AB0EE670A20460AF0C2FC04
:108EB000F0EE407AFB79FCEEE77A17EE902A91B259
:108EC000774A103322F81310FB791B01754A1A44B4
:108ED000FB79734931F8133007EE903AF8EE677A70
:108EE000B0EE671ADFED690A9FED690A10460AF0D5
:108EF000D3FDFB791B016B4A1A44FB796A4903F5E0
:108F0000B8735B000B445B889BB207EE903AF8EEB7
:108F1000677AB0EE670A10460AF0DBFDFB79013391
:108F2000FB714BE7534B00221A700023BB71BB79D6
:108F30000F2B70D8BB792C2202FB03F34E4A1A4444
:108F4000BB794E4931F8133007EE903AF8EE677A64
:108F5000B0EE670A10460AF06DFCF0EE407ABB797D
:108F6000FCEEE77A17EE902A91B24D4A22F81310E0
:108F7000BB791B014B4A1A44BB79494931F813307C
:108F800007EE903AF8EE677AB0EE670A1046FBF704
:108F9000C1FEF0EE407ABB79FCEEE77A17EE902A3C
:108FA00091B2424A22F81310BB792C2202FB03F340
:108FB000384A9C18BB79314A103332F813301A46BC
:108FC000BB7919461046FBF7AFFF034607EE903A10
:108FD000F8EE677AB0EE670A20460AF02BFCF0EE56
:108FE000407ABB79FCEEE77A17EE902A90B22C49D2
:108FF00003F1100221F81200BA792949103331F82F
:1090000013002A4902F11003024621F81320BB790C
:109010000133BB718BE7264B1B78002B20D0FFF769
:10902000FBFBFFF7D9FAFFF7DBF9224BD3F89830B7
:10903000204B4FF0FF32C3F898201F4BD3F89830E5
:109040001D4B4FF0FF32C3F898201C4BD3F89830DB
:109050001A4B4FF0FF32C3F89820194B01221A70B7
:10906000BFF34F8F00BF00BF0C37BD4690BD00BFA0
:10907000008000408C2C0020D0210020A001002086
:109080000AD7A33D9A99993E66D6A34300FF7F472E
:109090000000000090240020CDCCCC3D99C1F544C7
:1090A000F41A002050270020F4010020381B002073
:1090B0007F2C0020008003400090034000900B4074
:1090C000812C002080B582B000AF584B1B78002B5C
:1090D0002CD0574B0222DA70564B1B78DBB2062B92
:1090E0000CBF01230023DBB2002B07D0FDF782FF6A
:1090F000514B02221A704F4B00221A704D4B1B78B5
:10910000DBB2052B94BF01230023DBB2002B00F060
:109110008680484B1B78DBB25A1CD1B2454A11708D
:109120001946434B454A525C1A7178E0404BDB7854
:10913000DBB23B603B6803F01003002B0ED0102025
:10914000FDF7EEFE3B6803F04003002B06D15020F4
:10915000FDF7F6FE0220FDF7E3FE63E0344B9B795A
:10916000FB713B6803F04003002B1BD0344B002203
:109170001A70FDF7FBFE2E4BC0229A702C4B304A22
:109180001278D2B21B79D9B22E4B99542A4B0322B2
:109190001A705020FDF7D4FE4220FDF7C1FE244B8B
:1091A0009B79FB71FB7903F05003002B25D05020F5
:1091B000FDF7C6FEFDF7ECFE1D4BC8229A7002209B
:1091C000FDF7AEFE204B1B785A1CD1B21E4A11701F
:1091D0001A4613469B0013445B001C4A13440A22A0
:1091E000184918460BF015FE2022002115480BF0F7
:1091F0001EFE114B02221A7014E00D4A104B1B7810
:10920000DBB2591CC8B20E49087019461379DAB29C
:109210000C4B5A5445F2020105480AF063FABFF3B9
:109220004F8F00BF0837BD4680BD00BF872C002090
:1092300000700640862C0020882C00202C54010051
:10924000892C0020D40C00208A2C0020F40C002053
:10925000B0B582B000AF786039607B68012B43D134
:109260003B684FF6FF7293423ED1214808F009FF58
:10927000204808F007FD204808F0EAFF1F4809F0E1
:109280001EF81F4808F079FD1E4809F06BFA1E48C9
:10929000FAF760FA1D48FAF775FE1D480AF0AFF8B4
:1092A0001C4809F0CBFD1C4B0F241D46002C05DB90
:1092B0002846FBF7F9FC2C35013CF7E7174B0F2448
:1092C0001D46002C05DB2846FBF7EEFC2C35013C47
:1092D000F7E7134B0F241D46002C05DB28460AF048
:1092E000C0FB1035013CF7E700BF0837BD46B0BDF5
:1092F000C01D0020DC1D0020601E00206C1E002010
:10930000941E0020A81E0020141F0020441F0020CF
:10931000182000202C200020D021002090240020A4
:109320005027002080B483B000AF03463960FB7142
:1093300097F90730002B0ADB3B68DAB20C4997F942
:1093400007301201D2B20B4483F800230AE03B68D5
:10935000DAB20849FB7903F00F03043B1201D2B2E1
:109360000B441A7600BF0C37BD465DF8047B70478E
:1093700000E100E000ED00E090B585B000AFF860DE
:10938000B9607A603B60FB68002B05D1144B154A2D
:109390004A21154806F090FC144B154ADA62134B2B
:1093A00020221A63FB68114A1A60FB681B68114A85
:1093B0001A60FB681C68002002F086FB03466360AD
:1093C000FB681B680C4A9A65FB680C4A1A6179684D
:1093D0005120FFF7A7FF00BF1437BD4690BD00BF67
:1093E000745401008C5401007C540100E42A0020D4
:1093F000502A002000100B40482B0020D02A0020CB
:1094000080B582B000AF786039607B68002B06D1F0
:10941000084B094A4FF4A471084806F04DFC7B68DC
:109420001B683968184601F0A1FF03461846083743
:10943000BD4680BD74540100D05501009C5401000C
:1094400080B582B000AF78607B68002B06D1084BF6
:10945000084A40F24F11084806F02EFC7B681B6852
:1094600018460AF0C3FB034618460837BD4680BDC0
:10947000745401006C5701009C54010080B582B007
:1094800000AF786039607B68002B06D1084B094A31
:109490004FF4AB71084806F00FFC7B681B68396815
:1094A000184601F0A1FF034618460837BD4680BDA7
:1094B00074540100845701009C54010080B58EB0A3
:1094C00000AF78607B68002B06D11C4B1C4A4FF420
:1094D000D8711C4806F0F0FB07F12C0300221A603B
:1094E0005A6007F10C032022002118460BF09FFC64
:1094F00000237B630C23FB6000233B6103233B754C
:1095000002237B75104BBB6207F10C033B63002306
:10951000FB627B681B6807F12C02114618460AF0B3
:10952000FEFB78637B6B002B02D040F2097300E0F6
:10953000002318463837BD4680BD00BF7454010073
:109540007C5501009C5401000800F9FF80B586B0ED
:1095500000AFF860B9607A60BB68002B06D1154B8C
:10956000154A4FF4E571154806F0A6FBFB681B6829
:10957000B96818460AF0D3FB78617B69002B10D0DC
:10958000BB681B68002B02D0F868FFF797FF7B6869
:10959000002B08D07B68013B7B607B69002BE5D109
:1095A00002E000BF00E000BF7B6918461837BD46E7
:1095B00080BD00BFA8540100905501009C540100DB
:1095C00080B58EB000AF78607B68002B06D1204B51
:1095D000204A40F20B21204806F06EFB07F12C03D5
:1095E00000221A605A6007F10C032022002118465D
:1095F0000BF01DFC00237B630D23FB607B685B6A23
:109600001B043B6101237B7507F10C033B630023C3
:10961000FB6207F12C03032219467868FFF796FFD7
:1096200078637B6B002B0BD1BB6903F48073002B39
:10963000EAD0BB695B0A03F00F03072B02D1E3E713
:1096400000BF00E000BF7B6B18463837BD4680BDC9
:10965000745401009C5501009C54010080B594B0E5
:1096600000AF786039607B68002B06D1334B344AF9
:109670004FF40B71334806F01FFB07F13C03002247
:109680001A605A6007F11C032022002118460BF0D3
:10969000CEFB07F1080300221A605A609A60DA6074
:1096A0001A610023FB647B683033BB640422002111
:1096B000B86C0BF0BCFB7868FFF782FF0346002B09
:1096C00002D04FF4E36335E07B685B6A1946786843
:1096D000FFF796FE0346002B02D040F2157329E0F7
:1096E0001623FB61012387F825300423FB60012347
:1096F0003B61BB6C7B6107F11C033B6407F1080312
:10970000FB637B681B6807F13C02114618460AF0B0
:1097100006FBF864FB6C002B0BD1BA6A0A4B1340B2
:10972000002B06D1BB6C1B687B647B6C1ABA3B6850
:109730001A60FB6C18465037BD4680BD745401005A
:10974000B45501009C5401000800F9FF80B58EB0AB
:1097500000AF78607B68002B06D11A4B1A4A40F2A2
:1097600059211A4806F0A8FA07F12C0300221A60C2
:109770005A6007F10C032022002118460BF057FB1A
:1097800000237B630323FB6000233B6108237B757D
:1097900007F10C033B630023FB627B681B6807F146
:1097A0002C02114618460AF0BAFA78637B6B002B3C
:1097B00003D1BB691A0C7B685A627B6B1846383739
:1097C000BD4680BD74540100E85501009C54010061
:1097D00080B594B000AFF860B9607A603B60FB6818
:1097E000002B06D12E4B2F4A40F275212E4806F051
:1097F00063FABB6D002B06D12C4B2A4A40F276212E
:10980000294806F059FA07F1440300221A605A6009
:1098100007F124032022002118460BF008FB07F172
:10982000100300221A605A609A60DA601A610023FD
:10983000FB6406237B62BB68DB0763F07F43BB628C
:10984000BA6A7B689B000F2101FA03F3DB431340E4
:10985000BB62BA6A7B689B00396801FA03F3134361
:10986000BB62012387F82D3040237B610123BB615C
:10987000BB6DFB6107F12403BB6407F110037B643C
:10988000FB681B6807F14402114618460AF047FAC4
:10989000F864FB6C002BFB6C18465037BD4680BD4E
:1098A00074540100F45501009C540100B0540100AF
:1098B00080B584B000AF786039607B68002B06D13A
:1098C0005C4B5D4A4FF425715C4806F0F5F93B6846
:1098D000002B06D15A4B584A40F29521574806F0C2
:1098E000EBF97B6803F51A73FB603B681B681B0F81
:1098F000DAB2FB681A703B681B681B0EDBB203F020
:109900000F03DAB2FB685A703B681B68DB0DDBB2F1
:1099100003F00103DBB2002B06D0FB685B8843F049
:1099200001039AB2FB685A803B681B681B0DDBB2CF
:1099300003F00703DAB2FB681A713B681B681B0C63
:10994000DBB203F00F03DAB2FB685A713B681B68A5
:10995000DB0BDBB203F00103DBB2002B06D0FB68AC
:109960005B8843F002039AB2FB685A803B681B682D
:109970009B0ADBB203F01E03DAB2FB689A713B6804
:109980001B68DBB203F00303DAB2FB68DA713B68F1
:109990005A68FB689A60FB685B78022B0ED0022B3A
:1099A0001ADC002B02D0012B04D015E07B680122C9
:1099B0009A6214E07B6802229A6210E07B680422BB
:1099C0009A627B68B3F86A3203F00203002B05D079
:1099D0007B6808229A6201E000BF00E000BF7B685C
:1099E00093F86D3203F00403002B05D07B68DB6A2B
:1099F00043F004027B68DA627B6893F86F3203F00D
:109A00000103002B05D07B68DB6A43F080027B6892
:109A1000DA627B6893F86F3203F00203002B05D003
:109A20007B68DB6A43F040027B68DA6200BF103774
:109A3000BD4680BD74540100085601009C540100CD
:109A4000B854010080B59AB000AF78607B68002BF5
:109A500006D14A4B4A4A40F2CE214A4806F02CF938
:109A600007F1400300221A605A6007F12003202208
:109A7000002118460BF0DBF907F10C0300221A60F5
:109A80005A609A60DA601A617B6830337B66002323
:109A90003B6608220021786E0BF0C9F97B685B6A8F
:109AA00019467868FFF7ACFC0346002B02D040F261
:109AB00015735EE033233B62012387F829300023CE
:109AC0007B6208233B6101237B617B6EBB6107F1F5
:109AD0000C033B6407F120037B647B681B6807F180
:109AE0004002114618460AF01AF938663B6E002B00
:109AF0003ED1FA6A244B1340002B39D17B681B6896
:109B00005B7A022B06D0022B2ADC002B2BD0012BF8
:109B100011D025E07B6E1B68BB65BB6D1ABA7B6EEE
:109B20001A607B6E04331A687B6E0433FA65FA6D33
:109B300012BA1A6018E07B6E1B68FB64FB6C5BBAA0
:109B4000BB64BA6C7B6E1A607B6E04331A687B6EE2
:109B500004337A657A6D52BA3A653A6D1A6003E059
:109B60004FF4E16305E000BF796E7868FFF7A0FE6F
:109B70003B6E18466837BD4680BD00BF7454010077
:109B8000185601009C5401000800F9FF80B5A0B0F0
:109B900002AFF860B9607A60FB68002B06D1994B80
:109BA000994A4FF44371994806F086F8FB683033C0
:109BB0007B6707F1100300221A605A609A60002345
:109BC0003B6740220021786F0BF031F9FB689B6AFC
:109BD000012B06D9FB68B3F8503203F48063002BE5
:109BE00002D14FF4E1632DE17B6F00937B68BA688B
:109BF0000021F868FFF7ECFD0346002B02D040F28D
:109C000009731FE1FB681B685B7A022B06D0022BED
:109C100066DC002B67D0012B2CD061E07B6F1B68CA
:109C2000FB65FB6D1ABA7B6F1A607B6F04331A6891
:109C30007B6F04333A663A6E12BA1A607B6F083350
:109C40001A687B6F08337A667A6E12BA1A607B6F75
:109C50000C331A687B6F0C33BA66BA6E12BA1A608C
:109C60007B6F10331A687B6F1033FA66FA6E12BA84
:109C70001A6039E07B6F1B68BB63BB6B5BBA7B63AD
:109C80007A6B7B6F1A607B6F04331A687B6F0433C7
:109C90003A643A6C52BAFA63FA6B1A607B6F083313
:109CA0001A687B6F0833BA64BA6C52BA7A647A6CF9
:109CB0001A607B6F0C331A687B6F0C333A653A6D10
:109CC00052BAFA64FA6C1A607B6F10331A687B6FB1
:109CD0001033BA65BA6D52BA7A657A6D1A6003E0CC
:109CE0004FF4E163AEE000BF7B6F1B689BB27B83E8
:109CF0007B6F04331B681B0C9BB23B837B6F04336D
:109D00001B689BB2FB827B6F08331B681B0C9BB2EA
:109D1000BB827B6F08331B689BB27B827B6F0C33EB
:109D20001B681B0C9BB23B827B6F0C331B681B02B6
:109D30009AB27B6F10331B681B0E13433B67BB68E3
:109D40005B0007F17802134433F8683C1A467B68DD
:109D500042FA03F303F00103002B09D0BB689B0018
:109D60003A6F22FA03F303F00F037A689A4202D0A3
:109D70004FF4E16366E07B6F00937B68BA68012172
:109D8000F868FFF725FD0346002B02D040F2097367
:109D900058E0FB681B685B7A022B06D0022B2EDC96
:109DA000002B35D0012B13D029E07B6F0C331A68C0
:109DB0007B6F0C33FA62FA6A12BA1A607B6F103347
:109DC0001A687B6F10333A633A6B12BA1A6020E05C
:109DD0007B6F0C331A687B6F0C333A623A6A52BA63
:109DE000FA61FA691A607B6F10331A687B6F10335F
:109DF000BA62BA6A52BA7A627A6A1A6009E04FF4B1
:109E0000E1631FE074540100245601009C540100DA
:109E100000BF7B6F0C331B681B029AB27B6F103341
:109E20001B681B0E13433B67BB689B003A6F22FA0B
:109E300003F303F00F037A689A4202D040F21673DC
:109E400000E0002318467837BD4680BD80B58EB04F
:109E500000AF786039607B68002B06D1244B254A1F
:109E600040F27D31244805F027FF07F12C03002242
:109E70001A605A6007F10C032022002118460AF0EC
:109E8000D6FF00237B637B685B6A19467868FFF71F
:109E9000B7FA0346002B02D040F2157323E00623E5
:109EA000FB6001237B753B68002B03D03B68012BD3
:109EB00003D005E000233B6104E002233B6101E0A5
:109EC000042310E007F10C033B630023FB627B6873
:109ED0001B6807F12C021146184609F020FF786331
:109EE0007B6B002B7B6B18463837BD4680BD00BFAF
:109EF00074540100385601009C54010080B584B0B0
:109F000000AF786039607B68002B06D1914B924A94
:109F100040F2A331914805F0CFFE3B68002B06D1FB
:109F20008F4B8D4A4FF469718C4805F0C5FE7B68F4
:109F300003F51373FB603B680C331B689B0FDAB2AD
:109F4000FB681A703B680C331B681B0CDAB2FB68A9
:109F50005A703B680C331B681B0ADAB2FB689A70B4
:109F60003B680C331B68DAB2FB68DA703B68083375
:109F70001B681B0D9AB2FB689A803B6808331B680C
:109F80001B0CDBB203F00F03DAB2FB689A713B687B
:109F900008331B6803F40043002B06D0FB681B89C1
:109FA00043F001039AB2FB681A813B6808331B68CF
:109FB00003F48043002B06D0FB681B8943F00103A8
:109FC0009AB2FB681A813B6808331B6803F400539C
:109FD000002B06D0FB681B8943F004039AB2FB6890
:109FE0001A813B6808331B6803F48053002B06D0AA
:109FF000FB681B8943F008039AB2FB681A81FB686F
:10A000001B78002B02D0012B79D0ACE03B680833E1
:10A010001B689A0040F6FC731340FA68D360FB6833
:10A02000DA683B6804331B689B0F1A43FB68DA60ED
:10A030003B6804331B68DB0EDBB203F00703DAB2C4
:10A04000FB681A743B6804331B681B0EDBB203F019
:10A050000703DAB2FB685A743B6804331B681B0DB4
:10A06000DBB203F00E03DAB2FB689A743B68043388
:10A070001B689B0CDBB203F00703DAB2FB68DA74EF
:10A080003B6804331B68DB0BDBB203F00703DAB277
:10A09000FB681A75FB68DB685A1CFB681B7D023382
:10A0A0009A407B68C3F88822FB689B791A46012393
:10A0B00003FA02F27B68C3F88C227B68D3F88C32F7
:10A0C000B3F5007F4ED07B68D3F888327A68D2F837
:10A0D0008C2202FB03F27B68C3F888227B684FF472
:10A0E0000072C3F88C227B68D3F888227B68D3F88F
:10A0F0008C32B2FBF3F27B68C3F8882232E07B68D3
:10A100004FF40072C3F88C223B6808331B681B04B1
:10A1100003F47C12FB68DA60FB68DA683B6804339E
:10A120001B681B0C1A43FB68DA60FB68DB684FF6A0
:10A13000FE72934205D97B68DB6A43F010027B68AC
:10A14000DA62FB68DB6801339A027B68C3F8882215
:10A1500009E000BF745401004C5601009C540100FA
:10A16000C054010000BF3B6804331B689B0BDBB28B
:10A1700003F00103DBB2002B06D0FB681B8943F020
:10A1800010039AB2FB681A813B6804331B68DB0931
:10A19000DBB203F07F03DAB2FB685A753B68043325
:10A1A0001B68DBB203F07F03DAB2FB689A753B6889
:10A1B0001B689B0EDBB203F00703DAB2FB68DA75AB
:10A1C0003B681B689B0DDBB203F00F03DAB2FB6840
:10A1D0001A763B681B685B0DDBB203F00103DBB250
:10A1E000002B06D0FB681B8943F040039AB2FB6842
:10A1F0001A813B681B68DB0BDBB203F00103DBB2A7
:10A20000002B06D0FB681B8943F080039AB2FB68E1
:10A210001A813B681B689B0BDBB203F00103DBB2C6
:10A22000002B06D0FB681B8943F480739AB2FB684D
:10A230001A813B681B685B0BDBB203F00103DBB2E6
:10A24000002B06D0FB681B8943F400739AB2FB68AD
:10A250001A813B681B681B0BDBB203F00103DBB206
:10A26000002B06D0FB681B8943F480639AB2FB681D
:10A270001A813B681B689B0ADBB203F00303DAB266
:10A28000FB685A7600BF1037BD4680BD80B58EB0E2
:10A2900000AF78607B68002B06D1234B234A4FF434
:10A2A0008161234805F008FD07F12C0300221A60A4
:10A2B0005A6007F10C032022002118460AF0B7FD6E
:10A2C00000237B630923FB607B685B6A1B043B61A3
:10A2D00003237B7507F10C033B630023FB627B6860
:10A2E0001B6807F12C021146184609F018FD786327
:10A2F0007B6B002B10D17B6803F1300007F10C035E
:10A300000C33102219460AF084FD7B68303319465D
:10A310007868FFF7F3FD02E040F209737B637B6B23
:10A3200018463837BD4680BD745401005C560100A4
:10A330009C54010080B584B000AF786039607B68C0
:10A34000002B06D1324B334A40F22641324805F009
:10A35000B3FC3B68002B06D1304B2E4A40F227411C
:10A360002D4805F0A9FC7B6803F50E73FB603B6884
:10A370000C331B681B0EDAB2FB681A703B680C3397
:10A380001B681B0A9AB2FB685A803B680C331B6837
:10A39000DAB2FB681A713B6808331B681B0EDAB22D
:10A3A000FB685A713B6808331B681B0CDAB2FB6808
:10A3B0009A713B6808331B681B0ADAB2FB68DA71D2
:10A3C0003B6808331B68DAB2FB681A723B680433D7
:10A3D0001B681B0EDAB2FB685A723B6804331B68B9
:10A3E0001A02FB68DA60FB68DA683B681B681B0EC0
:10A3F0001A43FB68DA603B681B681B0A9BB2C3F315
:10A400000B039AB2FB681A8200BF1037BD4680BDAD
:10A4100074540100685601009C540100C8540100A6
:10A4200080B58CB000AF78607B68002B06D1204BE4
:10A43000204A40F23F41204805F03EFC07F1280346
:10A4400000221A605A6007F10803202200211846F2
:10A450000AF0EDFC0223BB600023FB6003237B7446
:10A4600007F10803FB620023BB627B681B6807F1EE
:10A4700028021146184609F052FC0346002B11D160
:10A480007B6803F1300007F108030C3310221946F2
:10A490000AF0BFFC7B68303319467868FFF74AFF43
:10A4A000002301E040F2097318463037BD4680BDF5
:10A4B00074540100785601009C54010080B58EB0A0
:10A4C00000AF786039607B68002B06D1334B344A8B
:10A4D00040F25741334805F0EFFB07F12803002213
:10A4E0001A605A6007F108032022002118460AF07A
:10A4F0009EFC01237B634FF47A733B632923BB608B
:10A500003B68FB6004237B743DE000217868FEF724
:10A5100077FF0346002B00D035E007F10803FB620C
:10A520000023BB627B681B6807F1280211461846AE
:10A5300009F0F5FB78637B6B002B02D040F20973C6
:10A5400027E07B69002B1BDA7B6903F08043002B3B
:10A5500005D07B68DB6A43F002027B68DA627B69C4
:10A5600003F08073002B05D07B68DB6A43F0200288
:10A570007B68DA627A697B68C3F83422002308E0DA
:10A580000A2000F065FF3B6B5A1E3A63002BBCD1DA
:10A590007B6B18463837BD4680BD00BF7454010040
:10A5A000885601009C54010080B58EB000AF7860E1
:10A5B0007B68002B06D1234B234A40F28E4123486F
:10A5C00005F07AFB07F1280300221A605A6007F1B0
:10A5D00008032022002118460AF029FC0A237B6385
:10A5E00000233B630823BB604FF4D573FB60092352
:10A5F0007B7407F10803FB620023BB627B681B6866
:10A6000007F128021146184609F089FB38633B6BB5
:10A61000002B09D17B69DBB2AA2B03D040F20C736B
:10A620003B6301E000233B637B6B013B7B637B6B04
:10A63000002B02D03B6B002BE0D13B6B1846383728
:10A64000BD4680BD74540100B05601009C54010009
:10A6500080B584B000AF78607B68002B06D1344BA6
:10A66000344A40F2B541344805F026FB40F21B73F2
:10A67000FB607B6893F89332032B28D001220021E2
:10A680007868FFF783FAF860FB68002B19D17B68C4
:10A69000012283F890227B681A687B685B69002B33
:10A6A00006D07B685B6925498B4228BF0B4600E0DA
:10A6B000224B1946104609F071FA02467B681A626D
:10A6C00030E0FB68B3F5E16F2CD100232BE07B6811
:10A6D00093F89032012B22D8012200217868FFF7ED
:10A6E00055FAF860FB68002B1BD17B68012283F8C8
:10A6F00090227B681A687B685B69002B06D07B68B8
:10A700005B690E498B4228BF0B4600E00B4B194694
:10A71000104609F043FA02467B681A6201E000BF66
:10A7200000E000BFFB6818461037BD4680BD00BF83
:10A7300074540100CC5601009C54010080F0FA02D0
:10A7400080B582B000AF786039607B68002B06D19D
:10A75000424B434A40F22651424805F0ADFA3B686D
:10A76000002B06D1404B3E4A40F227513D4805F0B0
:10A77000A3FA3B681B689B0FDAB27B6883F87422EC
:10A780003B681B685B0FDBB203F00103DAB27B6846
:10A7900083F875223B681B689AB27B68A3F876221F
:10A7A0003B685A687B68C3F878223B6808331B68AB
:10A7B0001B0EDAB27B6883F87C223B6808331B6887
:10A7C0001B0CDAB27B6883F87D223B6808331B6878
:10A7D0001B0BDBB203F00F03DAB27B6883F87E2237
:10A7E0003B6808331B689BB21B029AB23B680C3370
:10A7F0001B681B0E9BB213439AB27B68A3F880229E
:10A800003B680C331B681B0CDBB29B08DAB27B681D
:10A8100083F882223B680C331B681B0CDBB203F00D
:10A820000303DAB27B6883F883223B680C331B682E
:10A830001B0ADBB21B09DAB27B6883F884223B680F
:10A840000C331B681B0ADBB203F00F03DAB27B6820
:10A8500083F8852200BF0837BD4680BD74540100CF
:10A86000E05601009C540100D054010080B598B01E
:10A8700000AF78607B68002B06D1554B554A40F2FB
:10A880003951554805F018FA0023FB6507F14003DC
:10A8900000221A605A6007F1200320220021184686
:10A8A0000AF0C5FA07F10C0300221A605A609A6098
:10A8B000DA601A610023BB657B6830337B65402218
:10A8C0000021786D0AF0B3FA7868FEF779FE034646
:10A8D000002B02D04FF4E36375E07B685B6A194696
:10A8E0007868FEF78DFD0346002B02D040F2157309
:10A8F00069E00D233B62012387F8293040233B6147
:10A9000001237B617B6DBB6107F120037B6407F151
:10A910000C033B647B681B6807F140021146184634
:10A9200009F0FDF9B865BB6D002B04D1FA6A2B4B19
:10A930001340002B02D040F2097344E07B681B688F
:10A940005B7A022B06D0022B34DC002B35D0012B96
:10A9500017D02FE00023FB650FE0FB6D9B007A6DA5
:10A9600013441A68FB6D9B00796D0B443A653A6D90
:10A9700012BA1A60FB6D0133FB65FB6D0F2BECD92E
:10A980001CE00023FB6511E0FB6D9B007A6D134416
:10A990001A68FB6D9B00796D0B44FA64FA6C52BA2D
:10A9A000BA64BA6C1A60FB6D0133FB65FB6D0F2B4B
:10A9B000EAD903E04FF4E16305E000BF796D786800
:10A9C000FFF7BEFE002318466037BD4680BD00BFBE
:10A9D00074540100F05601009C5401000800F9FF76
:10A9E00080B582B000AF78600B46FB707B68002BAF
:10A9F00006D10A4B0A4A40F27E510A4805F05CF93A
:10AA00007B6818687B685B6AFA78194600F06EFC10
:10AA1000034618460837BD4680BD00BF7454010088
:10AA2000005701009C54010080B594B000AFF8605D
:10AA3000B9607A603B60FB68002B06D1484B494AFD
:10AA400040F29D51484805F037F9BB68002B06D10C
:10AA5000464B444A40F29E51434805F02DF9BB6DE8
:10AA6000002B06D1424B3F4A40F29F513E4805F031
:10AA700023F93B68B3F5007F06D03E4B394A4FF4CB
:10AA8000B461394805F018F907F1480300221A604B
:10AA90005A6007F128032022002118460AF0C7F95E
:10AAA00007F1140300221A605A609A60DA601A6192
:10AAB000FB68DB6A03F00203002B03D03B68B3F5AD
:10AAC000007F0ED1FB68D3F88C323A689A4208D8DE
:10AAD0003B68B3F5805F04D83B6803F00303002BA9
:10AAE00002D040F20C7337E0F868FEF769FD0346C8
:10AAF000002B02D04FF4E3632EE03B68BB61BB6DDB
:10AB0000FB61BB683B6201233B75BB6D012B01D12F
:10AB1000112300E01223BB627B68FB62FB68DB6AE7
:10AB200003F00203002B04D1FB6ABA6902FB03F3B2
:10AB3000FB62012387F831300F4B7B6407F1280358
:10AB4000FB6407F11403BB6407F1480303221946B1
:10AB5000F868FEF7FBFC034618465037BD4680BD3B
:10AB600074540100105701009C540100D45401009A
:10AB7000DC540100E85401000800F9FF80B594B0EE
:10AB800000AFF860B9607A603B60FB68002B06D1CB
:10AB9000574B584A40F2CE51574805F08DF8BB68E4
:10ABA000002B06D1554B534A40F2CF51524805F085
:10ABB00083F8BB6D002B06D1514B4E4A4FF4BA615E
:10ABC0004D4805F079F83B68B3F5007F06D04D4B52
:10ABD000484A40F2D151484805F06EF807F1440365
:10ABE00000221A605A6007F124032022002118462F
:10ABF0000AF01DF907F1100300221A605A609A60EA
:10AC0000DA601A61FB68DB6A03F00203002B03D0F1
:10AC10003B68B3F5007F0ED1FB68D3F88C323A68FD
:10AC20009A4208D83B68B3F5805F04D83B6803F0CC
:10AC30000303002B02D040F20C7354E0F868FEF7D7
:10AC4000BFFC0346002B02D04FF4E3634BE000BF90
:10AC5000FB681B68184608F0B3FF0346002BF7D1CA
:10AC600001233B743B687B61012387F82D30264B21
:10AC70003B64BB6D012B01D1182300E019237B62DB
:10AC80007B68BB62FB68DB6A03F00203002B04D124
:10AC9000BB6A7A6902FB03F3BB62FB6DBA6D1A6093
:10ACA000BB6DBB61BB683B6207F12403BB6407F16A
:10ACB00010037B6407F1440303221946F868FEF78A
:10ACC00045FCF864FB6C002B0CD0F96DF868FEF7BE
:10ACD000C5FC0346002B05D1FB6D1B68002B01D082
:10ACE0000023FB64FB6C18465037BD4680BD00BF97
:10ACF00074540100185701009C540100D454010001
:10AD0000DC540100E85401000800F9FF80B582B06E
:10AD100000AF78607B68002B06D10F4B0F4A40F2E2
:10AD20005E610F4804F0C8FF7B68B3F8543203F447
:10AD30000073002B06D17B68B3F8543203F48063B0
:10AD4000002B01D0012300E0002303F00103DBB25C
:10AD500018460837BD4680BD7454010024570100D1
:10AD60009C54010080B58CB002AFF860B9607A6085
:10AD70003B60FB68002B06D1504B514A40F26661A4
:10AD8000504804F099FFBB68002B06D14E4B4C4A4B
:10AD900040F267614B4804F08FFF3B68002B06D1FF
:10ADA0004A4B474A4FF4CD61464804F085FF3A6864
:10ADB0007B681A44FB68D3F888329A4206D9444B20
:10ADC0003F4A40F269613F4804F076FF0023FB618F
:10ADD000BB687B610123FB76FB68303323F0030300
:10ADE00004333B613B683B625FE0FB695B02BA682E
:10ADF00013447B61FB685B7F83F00103DBB2002BB4
:10AE000015D0FB7E83F00103DBB2002B04D17B69FC
:10AE100003F00303002B0AD001237B624FF400727E
:10AE2000002138690AF003F80023FB7610E03B6A42
:10AE3000B3F5803F08D33B6AA3F57F43FF3B3B62FA
:10AE40004FF6FF737B6203E03B6A7B6200233B6249
:10AE5000FB7E002B01D0796900E039697A68FB69D3
:10AE60001A447B6A00934FF40073F868FFF7DCFD27
:10AE70000346002B02D040F209731AE0FA697B6A9C
:10AE80001344FB61FB685B7F83F00103DBB2002BA3
:10AE90000BD0FB7E83F00103DBB2002B05D04FF417
:10AEA00000723969786909F0B4FF3B6A002B9CD1C4
:10AEB000002318462837BD4680BD00BF74540100EA
:10AEC000385701009C540100D4540100DC540100A7
:10AED0001455010080B58CB002AFF860B9607A609B
:10AEE0003B60FB68002B06D1514B524A40F29E61F9
:10AEF000514804F0E1FEBB68002B06D14F4B4D4A90
:10AF000040F29F614C4804F0D7FE3B68002B06D10D
:10AF10004B4B484A4FF4D461474804F0CDFE3A68A1
:10AF20007B681A44FB68D3F888329A4206D9454BAD
:10AF3000404A40F2A161404804F0BEFE00237B621B
:10AF400000233B6100233B620123FB77FB68303326
:10AF500023F003030433BB613B683B625FE03A6864
:10AF60003B6AD31A5B02BA6813447B61FB685B7F60
:10AF700083F00103DBB2002B15D0FB7F83F00103CC
:10AF8000DBB2002B04D17B6903F00303002B0AD052
:10AF900001237B624FF400727969B86909F039FFC7
:10AFA0000023FB7709E03B6AB3F5803F03D34FF6FC
:10AFB000FF737B6201E03B6A7B62FB7F002B01D069
:10AFC000796900E0B9697A683B681A443B6AD21A29
:10AFD00007F1100301937B6A00934FF40073F86844
:10AFE000FFF7CCFD0346002B02D040F209731AE0B4
:10AFF0003B693A6AD31A3B62FB685B7F83F00103CB
:10B00000DBB2002B0BD0FB7F83F00103DBB2002B04
:10B0100005D04FF400720021B86909F008FF3B6ABF
:10B02000002B9CD1002318462837BD4680BD00BFA9
:10B0300074540100485701009C540100D45401008D
:10B04000DC5401001455010080B584B000AF786075
:10B050007B68002B06D1244B244A4FF4E26124483C
:10B0600004F02AFE0023FB600023BB60FB6843F46E
:10B070004813FB607B68012283F893227868FEF70F
:10B08000DFF90346002B03D040F21373BB6026E0C8
:10B090007868FFF789FA0346002B0AD1FB6843F072
:10B0A0008043FB607B68DB6A43F008027B68DA62FE
:10B0B00009E07868FEF7C4F90346002B03D040F29C
:10B0C0001373BB600BE0F9687868FFF7F7F9034684
:10B0D000002B03D040F21473BB6000E000BFBB68DC
:10B0E00018461037BD4680BD745401005857010002
:10B0F0009C54010080B582B000AF78607B68002B63
:10B1000006D14E4B4E4A40F286714E4804F0D4FDB3
:10B110007B681B7F012B06D04B4B494A40F287715D
:10B12000484804F0C9FD7B680022DA627B681B682E
:10B130000021184608F03CFE7B681B68434918460E
:10B1400008F02CFD02467B681A627B681B68184673
:10B1500008F016FD7868FFF777FF034640F22A7281
:10B16000934202D140F22A7364E07868FFF758F9FD
:10B170000346002B02D040F20D735BE07868FEF7C7
:10B18000E5FA0346002B02D040F20E7352E07868D5
:10B19000FFF77CF80346002B02D040F20F7349E022
:10B1A00001217868FFF71CFC0346002B02D04FF406
:10B1B000E2633FE07B681B682549184608F0EEFC17
:10B1C00002467B681A627868FEF73CFC0346002B57
:10B1D00002D040F211732DE07B68DB6A03F00403B8
:10B1E000002B0FD001217868FEF730FE0346002BBC
:10B1F00002D040F212731DE07B681B6801211846E3
:10B2000008F0D6FD4FF400717868FEF737F9034671
:10B21000002B02D040F20A730CE07868FFF718FAAE
:10B220000346002B02D040F21B7303E07868FFF75F
:10B230001DFB002318460837BD4680BD745401002D
:10B24000785701009C54010044550100801A060003
:10B2500040787D0180B582B000AF78607B68002BBC
:10B2600006D11E4B1E4A40F2D6711E4804F024FD42
:10B270007B681B69002B06D11B4B194A40F2D77122
:10B28000184804F019FD7B681B7F83F00103DBB2D3
:10B29000002B09D07B681B68184600F0EDF80346C8
:10B2A000002B01D0012315E07B681B691B78012B63
:10B2B00004D07B681B691B78022B07D17B681A6856
:10B2C0007B681B691946104608F008FD7B6801225F
:10B2D0001A77002318460837BD4680BD7454010014
:10B2E000945701009C5401006055010080B58EB058
:10B2F00000AFF860B9601346FB7107F1300300221C
:10B300001A605A6007F1100320220021184609F044
:10B310008EFD07233B61FB79002B05D0BB681B0426
:10B320007B6101237B7603E000237B6100237B7636
:10B3300007F110037B6300233B6307F130031946D9
:10B34000F86808F0ECFC0346002B04D1FA69064BC0
:10B350001340002B02D040F2097300E0002318468E
:10B360003837BD4680BD00BF0800F9FF80B58CB0FE
:10B3700000AF7860396007F1280300221A605A6034
:10B3800007F1080320220021184609F050FD372359
:10B39000BB603B681B04FB6001237B7407F108035F
:10B3A000FB620023BB6207F128031946786808F0A6
:10B3B000B6FC0346002B04D17A690A4B1340002BDC
:10B3C00002D040F2097308E07B6903F02003002BF0
:10B3D00002D140F20C7300E0002318463037BD461E
:10B3E00080BD00BF0800F9FF80B58CB000AF786069
:10B3F000396007F1280300221A605A6007F1080338
:10B4000020220021184609F012FD1023BB603B6882
:10B41000FB6001237B7407F10803FB620023BB621E
:10B4200007F128031946786808F079FC0346002BD9
:10B4300004D17A69054B1340002B02D040F2097306
:10B4400000E0002318463037BD4680BD0800F9FFF4
:10B4500080B582B000AF78607B684FF47A7202FBEF
:10B4600003F30449184600F0A5FE00BF0837BD46A7
:10B4700080BD00BF000E270780B584B000AF7860A4
:10B480007B68002B05D1154B154AB021154804F0F7
:10B4900013FC7B689B6D002B05D1134B104AB12127
:10B4A000104804F009FC7B68FB60FB6802225A72BA
:10B4B000FB6802229A72FB688022DA60FB688022B5
:10B4C0001A61FB681A68FB6808331946104602F0D7
:10B4D00053FC002318461037BD4680BDA05701001D
:10B4E000F0570100B0570100D857010080B584B073
:10B4F00000AF78600023FB6009E00E4AFB6852F859
:10B5000023307A689A4206D0FB680133FB60FB68FF
:10B51000012BF2D900E000BFFB68012B05D9064BD7
:10B52000064A3521064804F0C7FBFB681846103769
:10B53000BD4680BD0058010010580100745801003C
:10B540003458010080B584B000AF786039603B6842
:10B55000002B05D13E4B3F4A42213F4804F0ACFB53
:10B560007868FFF7C3FF03463C4A52F82330184679
:10B5700008F038FC3B685B7803F003023B681B79FA
:10B580009B0003F00C031343FB603B685B79042BC7
:10B5900003D0FB6843F01003FB603B68DB785B0182
:10B5A00003F06003FA681343FB603B68DB79002B10
:10B5B00003D0FB6843F08003FB607B68FA689A6005
:10B5C0007B68DB6823F00F03FB603B685B79042B2F
:10B5D00006D03B685B7903F00303FA681343FB6012
:10B5E0003B689B79002B03D0FB6843F00403FB60AE
:10B5F0003B689B78002B03D0FB6843F00803FB609B
:10B600007B68FA68DA607B681B6A23F00303FB60DF
:10B610003B681B7803F00303FA681343FB607B6805
:10B62000FA681A623B681B7A002B06D07B685B6A5B
:10B6300043F008027B685A6205E07B685B6A23F08E
:10B6400008027B685A6200BF1037BD4680BD00BF4C
:10B65000445801008858010034580100085801007E
:10B6600080B586B000AFF860B9607A60BB68012B26
:10B6700006D9174B174A40F2C711174804F01CFBB4
:10B680007B68002B06D1154B124A4FF4E471124827
:10B6900004F012FB7B681B6803F01F037B617B686F
:10B6A0005B79002B03D07B6943F020037B617B68CF
:10B6B0001B79002B03D07B6943F040037B61FB685F
:10B6C000BA68796943F8221000BF1837BD4680BDBB
:10B6D00054580100945801003458010044580100A6
:10B6E00080B584B000AF786039603B68012B06D923
:10B6F0000C4B0D4A40F2E5110C4804F0DDFA002332
:10B70000FB607B683A6853F8223003F08003002B1B
:10B7100003D0FB6843F08003FB60FB6818461037DA
:10B72000BD4680BD54580100AC580100345801009A
:10B7300080B483B000AF7860084B1B6823F44022CC
:10B740007B689B0403F44023044913430B6000BF50
:10B750000C37BD465DF8047B704700BF00700440A5
:10B7600080B483B000AF78600B4B03F58053043393
:10B770001B6823F440327B681B0403F44033064902
:10B780001A4301F5805304331A6000BF0C37BD46DD
:10B790005DF8047B704700BF0070044080B582B044
:10B7A00000AF1A4B1B7BDBB203F00303022B22D04A
:10B7B000022B23D8002B02D0012B0ED01EE0144BFD
:10B7C0001B68002B05D1134B134ADA21134804F0F0
:10B7D00073FA0F4B1B687B6013E0114B1B68002B47
:10B7E00005D1104B0C4ADF210C4804F065FA0C4BD4
:10B7F0001B687B6005E00C4B7B6002E000237B60F4
:10B8000000BF7B6818460837BD4680BD0040064033
:10B81000582B0020C858010028590100DC580100AD
:10B820005C2B0020EC580100006CDC0280B582B07B
:10B8300000AFFFF7B3FF7860254B1B78DBB2DB0866
:10B84000DBB203F00703FB70FB787A6822FA03F39C
:10B850007B601F4B5B78DBB21B09DBB203F0030399
:10B86000BB701B4B1B7BDBB203F003037B70BB780D
:10B87000002B02D07B78002B02D07B78022B21D1C9
:10B88000FB78072B14D0072B19DC052B02DC002BCF
:10B8900003DA14E0062B04D011E07B685B097B60BF
:10B8A00011E07B680B4AA2FB03231B097B600AE0C3
:10B8B0007B68094AA2FB0323DB087B6003E00023CB
:10B8C0007B6000E000BF7B6818460837BD4680BD3E
:10B8D00000400640CDCCCCCCABAAAAAA80B483B0A1
:10B8E00000AF0E4B9B79DBB203F00103002B03D1B9
:10B8F0000B4B1B687B600AE00A4B1A68074B1B7AEC
:10B90000DBB25B0803F0070322FA03F37B607B687A
:10B9100018460C37BD465DF8047B70470040064072
:10B92000040100200801002080B582B000AF094B5F
:10B930009B79DBB203F01003002B03D1FFF776FFF6
:10B94000786002E0044B1B687B607B681846083710
:10B95000BD4680BD004006400401002080B485B093
:10B9600000AF78607B6849F69702934202D80023C3
:10B97000FB7308E07B68074A934202D80123FB73FC
:10B9800001E00223FB73FB7B18461437BD465DF8CC
:10B99000047B704700127A0080B582B000AF0E4B76
:10B9A0001B78DBB25BB2002B0EDA0C4B1B68002B52
:10B9B00006D10B4B0B4A40F267110B4804F07CF99F
:10B9C000064B1B687B6001E000237B607B681846A8
:10B9D0000837BD4680BD00BF00500640582B0020F0
:10B9E0000059010040590100DC58010080B582B0C7
:10B9F00000AF1A4B1B689B0C03F00303032B21D0F1
:10BA0000032B23D8002B02D0022B0CD01EE0FFF713
:10BA1000C3FF0346B3F5004F02D14FF4004300E0EB
:10BA200000237B6015E00E4B1B68002B06D10D4BED
:10BA30000D4A4FF4C1710D4804F03EF9084B1B68E4
:10BA40007B6006E04FF47A737B6002E000237B604A
:10BA500000BF7B6818460837BD4680BD00700440B3
:10BA60005C2B00200C59010058590100DC580100E2
:10BA700080B582B000AF124B03F5805304331B68CE
:10BA80001B0C03F00303032B0ED0032B0FD8002B4A
:10BA900002D0012B04D00AE000F090F9786009E0B0
:10BAA00000F0E6F9786005E0064B7B6002E00023D9
:10BAB0007B6000BF7B6818460837BD4680BD00BF6D
:10BAC00000700440006CDC0280B584B000AF034617
:10BAD000FB71FB79132B00F28E8001A252F823F048
:10BAE00031BB000031BB000051BB000071BB000046
:10BAF00091BB0000F7BB0000B1BB0000B9BB000068
:10BB0000C1BB0000F7BB0000F7BB0000C9BB0000D1
:10BB1000D1BB0000D9BB0000E1BB0000F7BB0000B7
:10BB2000F7BB0000F7BB0000E9BB0000EFBB000063
:10BB300000F012F90246344B03F5825304331B68BC
:10BB40001B0F03F00F030133B2FBF3F3FB6055E06F
:10BB500000F002F902462C4B03F5825304331B68B4
:10BB60001B0E03F00F030133B2FBF3F3FB6045E060
:10BB700000F0F2F80246244B03F5825304331B68AD
:10BB80001B0D03F00F030133B2FBF3F3FB6035E051
:10BB900000F0E2F802461C4B03F5825304331B68A5
:10BBA0001B0C03F00F030133B2FBF3F3FB6025E042
:10BBB000FFF75EFFF86021E0FFF718FFF8601DE077
:10BBC000FFF7EAFEF86019E008F08BFAF86015E07C
:10BBD00000F036F9F86011E000F0F0F8F8600DE0E0
:10BBE00000F046F9F86009E0084BFB6006E04FF40E
:10BBF0007A73FB6002E00023FB6000BFFB6818461D
:10BC00001037BD4680BD00BF00700440006CDC02F0
:10BC100080B582B000AF78600A497B685A6801F548
:10BC2000825304331A607B681B781846FFF798FD2F
:10BC30007B685B781846FFF77BFD00BF0837BD4681
:10BC400080BD00BF0070044080B584B000AF786054
:10BC500039600123FB73394808F0ECF97B68002B4D
:10BC60000CD1374B03F5805304331B68344923F45C
:10BC7000802201F5805304331A6045E03B68314A65
:10BC8000934214D03B682F4A93422CD83B682E4AEB
:10BC9000934213D03B682C4A934224D83B682B4AEA
:10BCA000934219D03B682A4A93420ED01BE0244BA2
:10BCB00003F58253083309221A6017E0204B03F57D
:10BCC0008253083302221A6010E01D4B03F58253A1
:10BCD000083305221A6009E0194B03F58253083333
:10BCE00000221A6002E00023FB7300BF144B03F52F
:10BCF000805304331B6823F4E02211497B681A4304
:10BD000001F5805304331A600C4808F079F97B6818
:10BD1000B3F5E02F0DD10F4B032283F844210D4BD7
:10BD200093F84031DBB20B4A63F07F03DBB282F859
:10BD30004031FB7B18461037BD4680BD12003410E1
:10BD400000700440000E270700D8B805006CDC0224
:10BD500000A24A040020074080B582B000AF164B15
:10BD60009B79DBB29B0803F003033B603B68032B2A
:10BD70001AD801A252F823F091BD000099BD00002D
:10BD8000A1BD000089BD000000F072F878600EE0EF
:10BD900000F014F878600AE0FFF7A0FD786006E094
:10BDA000FFF7FCFC786002E000237B6000BF7B684B
:10BDB00018460837BD4680BD0040064080B584B0B7
:10BDC00000AF1D4B5B78DBB203F00203002B06D102
:10BDD000194B9B79DBB203F02003002B02D0002328
:10BDE000FB6024E0FFF7A0FDB860BB68002B02D128
:10BDF000BB68FB601BE0104BDB78DBB25B09DBB29E
:10BE000003F00303FB710C4BDB78DBB2DB09DBB225
:10BE100003F00103BB71FA79BB790849520013445E
:10BE200031F813301A46BB6802FB03F3FB60FB6872
:10BE300018461037BD4680BD0040064070590100CD
:10BE400080B582B000AF094B1B78DBB203F0020370
:10BE5000002B02D100237B6002E0FFF73FFD7860FA
:10BE60007B6818460837BD4680BD00BF00400640CD
:10BE700080B584B000AF1C4B9B79DBB203F040036C
:10BE8000002B02D10023FB6028E008F023F9B86002
:10BE9000BB68002B06D1154B154A40F2F921154815
:10BEA00003F00AFF104B1B79DBB203F01F03DBB278
:10BEB0000133FB71FB79BA68B2FBF3F3BB600A4B49
:10BEC0005B79DBB203F01F03DBB21833BB71BA79C5
:10BED000BB6802FB03F3BB60BB68FB60FB681846F2
:10BEE0001037BD4680BD00BF004006401C59010010
:10BEF00080590100DC58010080B485B000AF0346D2
:10BF0000FB71174B1B7BDBB203F00302FB799A42F8
:10BF100002D00123FB7301E00023FB73104B1B7B5A
:10BF2000DBB223F00303DAB2FB7903F00303DBB2E5
:10BF30000B491343DBB20B73FB7B002B09D040F2A0
:10BF4000DC53BB6000E000BFBB685A1EBA60002B28
:10BF5000F9D1002318461437BD465DF8047B7047BD
:10BF60000040064080B584B000AF78607B68002B4D
:10BF700006D11E4B1E4A40F2F9311E4803F09CFECA
:10BF80000023FB737B685B7803F01F03DAB2FB7B53
:10BF90001343FB73184AFB7B1371174B5B79DBB2BE
:10BFA00023F01F03DAB27B689B7803F01F03DBB238
:10BFB00011491343DBB24B710F4B1B79DAB27B682B
:10BFC0001B781343DBB20C4A43F04003DBB213711E
:10BFD00000BF094B9B79DBB203F04003002BF8D084
:10BFE00000BF00BF1037BD4680BD00BF4C580100E8
:10BFF00094590100DC5801000040064080B584B02F
:10C0000000AF78607B681B681846FFF7A7FC034603
:10C01000FB737B681B791946194808F041F8194BE6
:10C020005B78DBB223F03C03DAB2FB7B1B01DBB2B3
:10C0300003F03003DBB21343DAB27B685B7911495A
:10C040001343DBB24B707B68063319460C4808F08B
:10C050000DF87B685B79002B0DD0094B1B78DBB2A8
:10C060005BB2002B07DA00BF064B9B79DBB203F013
:10C070000203002BF8D000BF1037BD4680BD00BFC3
:10C08000005006400040064080B582B000AF034635
:10C090003960FB713B68002B06D1254B254A40F2E5
:10C0A0006971254803F008FE244B5B78DBB2234A14
:10C0B00023F00203DBB25370204B1B78DBB203F09A
:10C0C0003B03DBB21D4A63F07F03DBB2137000BF9A
:10C0D0001A4B9B79DBB203F01C03082BF8D1174BEA
:10C0E0005B79DBB2154A23F04003DBB2537100BF2A
:10C0F000124B9B79DBB203F02003002BF8D1386898
:10C10000FFF730FF0D4B5B79DBB20C4A43F0400385
:10C11000DBB2537100BF094B9B79DBB203F0200304
:10C12000002BF8D0002318460837BD4680BD00BF5D
:10C130004C580100A8590100DC580100004006409D
:10C1400080B582B000AF03463A60FB710B46BB710D
:10C150003B68002B06D1134B134A40F6820113486B
:10C1600003F0AAFDFB791846FFF7C6FEBB793968D4
:10C170001846FFF789FF0E4B1B78DBB20C4A03F021
:10C180003F03DBB2137000BF094B9B79DBB29B0806
:10C1900003F00303032BF7D1002318460837BD46ED
:10C1A00080BD00BF4C580100BC590100DC580100A3
:10C1B00000400640B0B584B000AF786039607B685D
:10C1C000002B05D11F4B204AF321204803F074FDBA
:10C1D0007B6818464FF000013B681A464FF0000399
:10C1E00002FB01F500FB03F42C44A0FB02016318E1
:10C1F0001946174A4FF0000303F0E2FB02460B46D4
:10C20000C7E90223D7E90223012B08BF002A05D37F
:10C21000104B0D4AF5210D4803F04EFDD7E9020100
:10C220004FF000024FF00003820842EA81728B084F
:10C23000C7E90223BB68184607F06DFF00BF10373F
:10C24000BD46B0BDD0590100045A0100E0590100BB
:10C2500040420F00F059010080B584B000AF786013
:10C260000023FB6006E00D4A7B68934206D0FB6822
:10C270000133FB60FB68002BF5D000E000BFFB68DA
:10C28000002B05D0064B074A3B21074803F014FD5D
:10C29000FB6818461037BD4680BD00BF0010024045
:10C2A000185A0100505A0100405A010080B582B06E
:10C2B00000AF78607868FFF7CFFF044B184607F0AF
:10C2C0003AFF00BF0837BD4680BD00BF01003C10EB
:10C2D00080B582B000AF78603960786807F045FFBC
:10C2E0000346002B05D0094B1B68396878689847CE
:10C2F00004E0074B1B68396878689847BFF34F8F95
:10C3000000BF00BF0837BD4680BD00BF6C2B0020BA
:10C31000702B002080B500AF094B1B68002B06D1A5
:10C32000084B094A40F69301084803F0C5FC044B4A
:10C330001B6819460648FFF7CBFF00BF80BD00BF52
:10C34000602B0020945A0100DC5A0100885A010039
:10C3500000C0024080B500AF094B5B68002B06D1DE
:10C36000084B094A40F69B01084803F0A5FC044B22
:10C370005B6819460648FFF7ABFF00BF80BD00BFF2
:10C38000602B0020AC5A0100F45A0100885A0100C9
:10C3900000D0024080B500AF094B9B68002B06D14E
:10C3A000084B094A40F6A301084803F085FC044BFA
:10C3B0009B6819460648FFF78BFF00BF80BD00BF92
:10C3C000602B0020C45A01000C5B0100885A010058
:10C3D00000C00A4080B584B000AF78600023FB60E5
:10C3E00006E00D4A7B68934206D0FB680133FB6090
:10C3F000FB68002BF5D000E000BFFB68002B05D0E8
:10C40000064B074A4A21074803F056FCFB681846CA
:10C410001037BD4680BD00BF00800040245B010096
:10C42000D45B0100485B010080B584B000AFF860C8
:10C43000B9607A60BB680F2B05D94E4B4E4A582124
:10C440004E4803F039FC7B68002B05D14C4B4A4A1F
:10C4500059214A4803F030FC7B6803F01F03002B8E
:10C4600005D0484B444A5A21444803F025FC7B68D8
:10C470001A68F968BB6880335B010B441A607B68FB
:10C480009B8899B2FA68BB6880335B01134404331C
:10C490000A461A807B68DB8899B2FA68BB688033E9
:10C4A0005B01134406330A461A807B689A68F96870
:10C4B000BB685B010B4403F5805308331A607B684B
:10C4C000DA68F968BB685B010B4403F580530C33F1
:10C4D0001A607B681A69F968BB685B010B4403F555
:10C4E000805310331A607B689B8A99B2FA68BB68E4
:10C4F0005B01134403F5805314330A461A807B68AA
:10C50000DB8A99B2FA68BB685B01134403F5805378
:10C5100016330A461A807B689A69F968BB685B0122
:10C520000B4403F5805318331A60FA68BB685B014B
:10C53000134403F580531C3300221A807B689B8BC5
:10C5400099B2FA68BB685B01134403F580531C334E
:10C550000A461A807B68DB8B99B2FA68BB685B017C
:10C56000134403F580531E330A461A8000BF103768
:10C57000BD4680BD545B0100E85B0100485B0100E3
:10C58000885B0100945B010080B584B000AF7860E7
:10C5900039603B68002B05D1204B214A7821214886
:10C5A00003F08AFB7868FFF715FF1F4B184607F06A
:10C5B000EFFD7B680022DA607B684FF0FF325A6241
:10C5C0007B684FF0FF32DA627B681B68FB60FB68B8
:10C5D00023F05603FB603B689B789B0003F004024A
:10C5E0003B685B781B0103F010031A433B681B7820
:10C5F0009B0103F040031A433B68DB785B0003F0C8
:10C6000002031A43FB68134343F08003FB607B681B
:10C61000FA681A6000BF1037BD4680BDB45B0100E8
:10C62000F85B0100485B01000100401080B582B05A
:10C6300000AF786039603B680F2B05D9084B094A79
:10C64000C421094803F038FB3B6880335B017A68FA
:10C650001344184600F00AF800BF0837BD4680BDF5
:10C66000545B0100045C0100485B010080B582B0AE
:10C6700000AF78607B68002B06D11C4B1C4A40F24F
:10C68000A7111C4803F018FB7B6803F01F03002B65
:10C6900006D0194B164A4FF4D471164803F00CFB20
:10C6A0007B6800221A607B6800229A807B680022E7
:10C6B000DA807B6800229A607B680022DA607B68FF
:10C6C00000221A617B6800229A827B680022DA824B
:10C6D0007B6800229A617B6808229A837B6800222B
:10C6E000DA8300BF0837BD4680BD00BF885B01000C
:10C6F000185C0100485B0100945B010080B584B0C8
:10C7000000AF786039603B680F2B06D9194B1A4A85
:10C7100040F2CD21194803F0CFFA0023FB607A687C
:10C720003B685B01134403F580531C331B889BB2A9
:10C73000DB0903F00103FA681343FB607B68DA6AE4
:10C740003B6822FA03F35B0003F00203FA68134329
:10C75000FB607B685A6A3B6822FA03F39B0003F094
:10C760000403FA681343FB60FB6818461037BD46A4
:10C7700080BD00BF545B0100285C0100485B0100E4
:10C7800080B584B000AFF860B9607A60BB680F2BE9
:10C7900006D9134B134A40F2E521134803F08CFAF3
:10C7A0007B6803F00103002B03D0BB68DAB2FB689F
:10C7B0001A777B6803F00203002B03D0BB68DAB260
:10C7C000FB689A777B6803F00403002B03D0BB68F7
:10C7D000DAB2FB68DA7700BF1037BD4680BD00BF14
:10C7E000545B0100445C0100485B010090B589B0D6
:10C7F00000AF78607B68002B06D1554B554A40F25C
:10C800002351554803F058FA7B689B687A68127C7C
:10C81000DA777B689A687B681B7C5B01134403F5BD
:10C8200080531C331B889BB203F08003002B14BF82
:10C8300001230023BB767B68DB68002B0CD17B686F
:10C840001B68002B7FD07B681C687B685968BA7EA8
:10C8500000237868A04776E07B689A687B681B7C39
:10C860005B01134403F5805318331B687B617B68BD
:10C87000DB681A467B699B1A7B617B695B093B61BC
:10C88000BB7E002B02D03B69FB760EE03B69002BA0
:10C8900004D03B69DBB2013BDBB205E07B681B7D6A
:10C8A0005BB2DBB2013BDBB2FB767B685B7C5AB2EE
:10C8B00097F91B309A4213D17B68DB7CFB737B6852
:10C8C0001B7DBB7397F90F2097F90E309A4204D164
:10C8D0007B68DB7C5BB2FB6112E00023FB610FE055
:10C8E000FB7E7A68527C52B29B1AFB61FB69002B7B
:10C8F00006DA7B681B7D5BB21A46FB691344FB6159
:10C9000097F91B207B685A747B68DB7C5BB2DAB2D8
:10C91000FB69DBB2D31ADBB25AB27B68DA747B688C
:10C920001B68002B07D07B681C687B685968FB6913
:10C93000BA7E7868A047BB7E002B04D07B689B68DA
:10C940007A68127C1A7700BF2437BD4690BD00BFBD
:10C95000C45B0100645C0100485B010080B500AF6E
:10C96000044B1B681846FFF741FFBFF34F8F00BF12
:10C9700000BF80BD742B002080B500AF044B5B6806
:10C980001846FFF733FFBFF34F8F00BF00BF80BDD6
:10C99000742B002080B500AF044BDB681846FFF70E
:10C9A00025FFBFF34F8F00BF00BF80BD742B002059
:10C9B00080B500AF044B1B691846FFF717FFBFF3A4
:10C9C0004F8F00BF00BF80BD742B002080B500AF2B
:10C9D000044B5B691846FFF709FFBFF34F8F00BF99
:10C9E00000BF80BD742B002080B500AF044B9B6955
:10C9F0001846FFF7FBFEBFF34F8F00BF00BF80BD9F
:10CA0000742B002080B500AF044BDB691846FFF79C
:10CA1000EDFEBFF34F8F00BF00BF80BD742B002021
:10CA200080B500AF044B1B6A1846FFF7DFFEBFF36B
:10CA30004F8F00BF00BF80BD742B002080B500AFBA
:10CA4000044B5B6A1846FFF7D1FEBFF34F8F00BF60
:10CA500000BF80BD742B002080B500AF044B9B6AE3
:10CA60001846FFF7C3FEBFF34F8F00BF00BF80BD66
:10CA7000742B002080B500AF044BDB6A1846FFF72B
:10CA8000B5FEBFF34F8F00BF00BF80BD742B0020E9
:10CA900080B500AF044B1B6B1846FFF7A7FEBFF332
:10CAA0004F8F00BF00BF80BD742B002080B500AF4A
:10CAB000044B5B6B1846FFF799FEBFF34F8F00BF27
:10CAC00000BF80BD742B002080B500AF044B9B6B72
:10CAD0001846FFF78BFEBFF34F8F00BF00BF80BD2E
:10CAE000742B002080B500AF044BDB6B1846FFF7BA
:10CAF0007DFEBFF34F8F00BF00BF80BD742B0020B1
:10CB000080B500AF054B1B68054A12681146054801
:10CB10009847BFF34F8F00BF00BF80BDB82B0020E8
:10CB2000B42B002000000C4080B500AF054B1B6803
:10CB3000054A1268114605489847BFF34F8F00BF5A
:10CB400000BF80BDBC2B0020B42B002000000C4097
:10CB500080B500AF054B1B68054A126811460548B1
:10CB60009847BFF34F8F00BF00BF80BDC02B002090
:10CB7000B42B002000000C4080B500AF054B1B68B3
:10CB8000054A1268114605489847BFF34F8F00BF0A
:10CB900000BF80BDC42B0020B42B002000000C403F
:10CBA00080B500AF0B4B1B68002B06D10A4B0B4A1C
:10CBB00040F683510A4803F07FF80A4B1B68054A88
:10CBC0001268114608489847BFF34F8F00BF00BF57
:10CBD00080BD00BFC82B0020AC5C0100C85C010018
:10CBE0009C5C0100CC2B00200040024080B584B04A
:10CBF00000AF78600423BB600023FB6009E00F4AAC
:10CC0000FB6852F823307A689A4207D0FB680133F8
:10CC1000FB60FA68BB689A42F1D300E000BFFA6893
:10CC2000BB689A4205D3064B064A5021064803F0DA
:10CC300043F8FB6818461037BD4680BDE05C010034
:10CC4000005D0100B45D01001C5D010080B586B08F
:10CC500000AF786039600023FB7500233B6100233F
:10CC6000FB607B68464A934211D07B68454A9342F9
:10CC70000DD07B68444A934209D07B68434A934273
:10CC800005D0434B434A5B21434803F015F87B68CA
:10CC90009B6DFB60FB6843F00803FB607B685B6E89
:10CCA0003B610023FB750BE0FB7DDB0005330122BC
:10CCB00002FA03F33A6913433B61FB7D0133FB75D1
:10CCC000FA7D7B682E498B4213D07B682D498B42BD
:10CCD0000DD07B682C498B4207D07B682B498B4257
:10CCE00001D1042306E07F2304E0012302E00123B5
:10CCF00000E004239342D7D87B683A695A667B6880
:10CD0000D3F88C303B613B6943F0B4033B613B6833
:10CD100003F08003002B03D03B6943F4F8533B61DD
:10CD20003B6803F07003002B1ED03B6943F4F813FB
:10CD30003B613B6803F01003002B03D0FB6843F01A
:10CD40001003FB603B6803F02003002B03D0FB685B
:10CD500043F02003FB603B6803F04003002B03D04B
:10CD6000FB6843F04003FB607B68FA689A657B6868
:10CD70003A69C3F88C2000BF1837BD4680BD00BF9C
:10CD8000008003400090034000A0034000900B404F
:10CD9000285D0100C45D01001C5D010080B586B006
:10CDA00000AF7860396000237B6100233B617B68C2
:10CDB000454A934214D07B68444A93420ED07B6824
:10CDC000434A934208D07B68424A934201D10823E8
:10CDD00007E04FF0FF3304E0022302E0022300E00B
:10CDE0000823FB7397F90F30B3F1FF3F05D13A4B9E
:10CDF0003A4A98213A4802F05FFF7B68D3F88C30BA
:10CE000043F004027B68C3F88C207B685B6E3B6157
:10CE100000237B610BE07B69DB000533012202FA12
:10CE200003F33A6913433B617B6901337B6197F9F3
:10CE30000F305B087A699A42EDD37B683A695A668B
:10CE40007B68D3F898303B6197F90F30012202FAE2
:10CE500003F35B423A6913403B6197F90F304FF09F
:10CE6000FF3202FA03F3DA433B6813403A69134393
:10CE70003B617B683A69C3F898207B689B6D3B6196
:10CE80003B6803F48073002B04D03B6943F002033A
:10CE90003B6103E03B6923F002033B613B6803F421
:10CEA0000073002B04D03B6943F001033B6103E0B6
:10CEB0003B6923F001033B617B683A699A6500BFD7
:10CEC0001837BD4680BD00BF00800340009003407E
:10CED00000A0034000900B40545D0100D45D0100B0
:10CEE0001C5D010080B584B000AF786039603B689C
:10CEF000002B05D1374B384ADF21384802F0DCFEE1
:10CF00003B685B6803F0F003002B01D101235DE077
:10CF10007868FFF76BFE0346314A52F82330184613
:10CF200007F050F93B681B7B5B0103F0600343F0A3
:10CF300005027B685A653B685B6819467868FFF7AD
:10CF400085FE3B689B6819467868FFF727FF3B68BA
:10CF50001B7803F007027B681A603B685B789B01D3
:10CF6000DAB23B689B7E5B0203F400731A437B6872
:10CF7000C3F884203B681B7E1A467B68DA653B68F1
:10CF80005B7E1A467B681A673B685A697B68DA667B
:10CF90003B689B7B9B01DAB23B681B6903F03F0354
:10CFA0001A437B689A667B68DB6FFB60FB6823F43F
:10CFB0007063FB603B685B7B1B0203F47063FA6881
:10CFC0001343FB607B68FA68DA6700231846103762
:10CFD000BD4680BD4C580100E85D01001C5D0100AC
:10CFE000F05C010080B58AB000AFF860B96011460E
:10CFF0001A460B46FB711346BB71BB68002B06D16A
:10D000007C4B7D4A4FF4C1717C4802F055FE7B6B2E
:10D01000002B06D17A4B784A40F28311774802F010
:10D020004BFE3B6B002B06D1764B734A4FF4C2711B
:10D03000724802F041FEFB79002B06D1724B6E4A1A
:10D0400040F285116D4802F037FEFB686F4A93424B
:10D0500012D0FB686E4A93420ED0FB686D4A934231
:10D060000AD0FB686C4A934206D06C4B624A40F28D
:10D070008711624802F020FEFB681B6803F007037B
:10D080007A6B22FA03F37B61BB79012B0CD1FB682D
:10D090001B6843F02002FB681A603B6B5B007A69F7
:10D0A000B2FBF3F37B620BE0FB681B6823F020020A
:10D0B000FB681A607A693B6BB2FBF3F3013B7B625E
:10D0C0007B6AB3F5803F01D3012335E1FB687A6ABF
:10D0D0009A600023FB7629E1BB689B78642B01D919
:10D0E000012329E1BB79002B02D0BB79012B3FD171
:10D0F000BB681B78FA680133DB0013445B683B6153
:10D100003B6923F03C033B61BB685B789B003A6959
:10D1100013433B613B6943F020033B61BB681B78D1
:10D12000FA680133DB0013443A695A60BB689B78A4
:10D13000002B02D100233B6211E0BB689B781A46AA
:10D140007B6A03FB02F3364AA2FB03235B093B62C3
:10D150003A6A7B6A9A4202D37B6A01333B62BB68BC
:10D160001B78FA680133DB0013443A6A9A60D7E00F
:10D17000BB681B781946FB68244A934214D0FB68AD
:10D18000234A93420ED0FB68224A934208D0FB68A0
:10D19000214A934201D1042307E06FF0004304E0E9
:10D1A000012302E0012300E004238B4201D8012384
:10D1B000C2E0BB68DB78642B01D90123BCE0BB680B
:10D1C000DB78002B02D10023FB610AE0BB68DB782F
:10D1D0001A467B6A03FB02F3114AA2FB03235B0995
:10D1E000FB61BB689B78002B1CD100233B620023B2
:10D1F000FB6129E0645D0100F45D01001C5D01003C
:10D20000785D01008C5D0100A05D0100008003409D
:10D210000090034000A0034000900B40285D0100F7
:10D220001F85EB51BB689B781A467B6A03FB02F3B0
:10D23000434AA2FB03235B093B623A6A7B6A9A4238
:10D2400002D37B6A01333B62BB681B785B00FA68E0
:10D250000133DB0013445B683B613B6923F03C0313
:10D260003B61BB685B789B003A6913433B61BB68D9
:10D270001B785B00FA680133DB0013443A695A609B
:10D28000BB681B785B000133FA680133DB00134491
:10D290005B683B613B6923F03C033B61BB685B78A7
:10D2A0009B003A6913433B61BB681B785B00013309
:10D2B000FA680133DB0013443A695A60FB685A6E1E
:10D2C000BB681B78DB00012101FA03F31A43FB68FA
:10D2D0005A66BB681B785B00FA680133DB001344B5
:10D2E000FA699A60BB681B785B000133F9693A6A96
:10D2F0000A44F9680133DB000B449A60BB79032BC5
:10D300000ED1BB681B7801221946F86806F09DFF14
:10D31000BB681978BB681B791A46F86806F06CFF81
:10D32000BB680533BB60FB7E0133FB76FA7EFB797D
:10D330009A42FFF4D1AE002318462837BD4680BD7F
:10D340001F85EB5180B584B000AF78600023FB608F
:10D3500009E00E4AFB6852F823307A689A4206D0F8
:10D36000FB680133FB60FB68042BF2D900E000BFCF
:10D37000FB68042B05D9064B064A4321064802F0F8
:10D380009BFCFB6818461037BD4680BD185E010047
:10D390002C5E01005C5E0100505E010080B586B02D
:10D3A00000AFF860B9607A607B68002B05D1154B3F
:10D3B000154A6421154802F07FFC01237B617B68DC
:10D3C0001B78002B0AD1FB685A697969BB6801FA9E
:10D3D00003F3DB431A40FB685A610FE07B685B781C
:10D3E0001A46B968F86806F059FFFB685A69796906
:10D3F000BB6801FA03F31A43FB685A6100BF183790
:10D40000BD4680BD44580100705E0100505E0100C1
:10D4100080B584B000AF78607868FFF793FF03466B
:10D42000FB73FB7B054A52F82330BB60BB68D3F823
:10D43000A03018461037BD4680BD00BF045E010015
:10D4400080B584B000AF786039607868FFF77AFF04
:10D450000346FB73FB7B064A52F82330BB60BB6874
:10D460003A68C3F8A02000BF1037BD4680BD00BF9A
:10D47000045E010080B584B000AF78600023FB60DB
:10D4800009E00E4AFB6852F823307A689A4206D0C7
:10D49000FB680133FB60FB68022BF2D900E000BFA0
:10D4A000FB68022B05D9064B064A9F21064802F06D
:10D4B00003FCFB6818461037BD4680BD0C5F0100B9
:10D4C000185F0100605F01003C5F010080B584B01F
:10D4D00000AF786039607B68DB78FB737B689B7892
:10D4E000BB73BB7B03F02003002B04D1FB7B03F059
:10D4F0001003002B05D0094B1B68396878689847E2
:10D5000004E0074B1B68396878689847BFF34F8F72
:10D5100000BF00BF1037BD4680BD00BFDC2B002020
:10D52000E02B002080B586B000AFF860B9607A606B
:10D53000BB68002B06D1354B354A40F236213548C1
:10D5400002F0BAFB7B68002B06D1334B304A40F225
:10D550003721304802F0B0FBF868FFF78BFF034635
:10D560002E4A52F82330184606F0B5FEFB6800221A
:10D570001A70FB6800225A70FB6800229A70FB68E0
:10D58000FF22DA70FB6800225A71FB6850229A7100
:10D59000FB680022DA71FB689B78DBB203F07F0343
:10D5A000DAB2FB689A7045F21201F86806F0ADFE37
:10D5B000BB685B687A681946F86800F031F8FB6868
:10D5C0009B79FB75FB7D03F07F03FB75BB685B7884
:10D5D000DB01DAB2FB7D1343FB75FB7D23F00F0308
:10D5E000FB75BB681B7A03F00F03DAB2FB7D1343B4
:10D5F000FB75FB68FA7D9A71BB681B78DB01DAB2B8
:10D60000FB689A7000BF1837BD4680BD485F0100B7
:10D61000705F01003C5F0100785D0100005F010068
:10D6200080B48DB000AFF860B9607A604FF0FF331E
:10D63000FB620023BB6200237B620123FB610023AA
:10D6400087F8233044E0FB6A002B46D097F823305C
:10D65000FA6902FA03F3BB61002387F822302CE059
:10D6600097F82230274A32F813301A46BB6903FB79
:10D6700002F37A68B2FBF3F37B61BA687B699A4282
:10D6800003D9BA687B69D31A02E07A69BB68D31AF6
:10D690003B613A69FB6A9A420AD297F82330BB622F
:10D6A00097F822307B623B69FB623B69002B09D013
:10D6B00097F82230013387F8223097F822303F2B39
:10D6C000CED900E000BF97F82330013387F823302C
:10D6D00097F82330022BB6D900E000BFBB6ADBB25B
:10D6E0009B01DAB27B6ADBB203F03F03DBB2134388
:10D6F000DAB2FB685A7000BF3437BD465DF8047B70
:10D70000704700BF805E010080B500AF034B1B680F
:10D7100019460348FFF7DAFE00BF80BDD02B00207A
:10D720000060064080B500AF034B9B681946034874
:10D73000FFF7CCFE00BF80BDD02B002000600E4064
:10D7400080B584B000AF78600023FB6006E00D4A2E
:10D750007B68934206D0FB680133FB60FB68002BBB
:10D76000F5D000E000BFFB68002B05D0064B074A50
:10D770003421074802F0A0FAFB6818461037BD466E
:10D7800080BD00BF00600340805F0100B05F01000A
:10D79000A45F010080B584B000AF786039603B6859
:10D7A000002B05D11F4B204A4621204802F084FA65
:10D7B0007868FFF7C5FF1E4B184606F071FE7B68C0
:10D7C0001A681C4B1340FB603B681B789B0403F4F6
:10D7D00040223B685B781B0303F4E0431A433B6839
:10D7E000DB781B0203F470631A433B689B789B0051
:10D7F00003F00C031343FA681343FB603B681B7987
:10D80000002B03D0FB6843F00203FB607B68FA68DF
:10D810001A600121786806F05DFE00BF1037BD4632
:10D8200080BD00BF44580100C05F0100A45F01003B
:10D8300016003C10F180F3FF80B584B000AF786033
:10D840000023FB6006E00D4A7B68934206D0FB682C
:10D850000133FB60FB68002BF5D000E000BFFB68E4
:10D86000002B05D0064B074A3721074802F024FA5F
:10D87000FB6818461037BD4680BD00BF00700340EE
:10D88000CC5F0100FC5F0100F05F010080B584B057
:10D8900000AF786039603B68002B05D1204B214AEE
:10D8A0004621214802F008FA7868FFF7C5FF1F4BB0
:10D8B000184606F02BFE7B681B6823F002027B688B
:10D8C0001A600023FB7312E0FB7B7A681B01134490
:10D8D00003F584731A68FB7B22F0070279681B0149
:10D8E0000B4403F584731A60FB7B0133FB73FB7BF2
:10D8F000032BE9D93B681B78002B06D07B681B689B
:10D9000023F001027B681A6005E07B681B6843F026
:10D9100001027B681A6000BF1037BD4680BD00BFA2
:10D92000445801000C600100F05F010017003C103A
:10D9300080B582B000AF78600A4806F001FE094861
:10D9400006F018FE074806F0FBFD7B6800221A600F
:10D950007B681B6843F001027B681A6000BF0837D0
:10D96000BD4680BD09003C1080B500AF0B4B1B6865
:10D97000002B06D10A4B0B4A40F63D310A4802F013
:10D980009BF90A4B1B68054A1268114608489847DC
:10D99000BFF34F8F00BF00BF80BD00BFE42B00204E
:10D9A000406001007860010034600100EC2B002031
:10D9B00000F0024080B500AF0B4B5B68002B06D136
:10D9C0000A4B0B4A40F644310A4802F075F90A4BFB
:10D9D0001B68054A5268114608489847BFF34F8FA5
:10D9E00000BF00BF80BD00BFE42B00205C600100D1
:10D9F0009460010034600100F02B002000F0024030
:10DA000080B584B000AF78600023FB7302E0FB7B3D
:10DA10000133FB73FB7B002B03D1094A7B689342E4
:10DA2000F5D1FB7B002B05D0064B074AE4210748C4
:10DA300002F042F9FB7B18461037BD4680BD00BF9F
:10DA400000100B40B0600100D4620100D4600100FE
:10DA500080B586B000AF786039603B68002B06D196
:10DA60002C4B2D4A40F24B112C4802F025F97B68D3
:10DA70001B697B617B685B693B617B689B69FB60C1
:10DA80003B685B7A002B21D03B687A69DA603B689F
:10DA90005B7A032B1AD13B68DB681A023B68DA60B9
:10DAA0003B691A027B691B0E1A433B681A61FB68CB
:10DAB0001A023B691B0E1A433B685A617B68DB699B
:10DAC0001A02FB681B0E1A433B689A613B68DB69CC
:10DAD000002B19D03B685B7A012B0BD03B685B7A3B
:10DAE000022B07D03B685B7A082B03D03B685B7A3C
:10DAF000062B09D13B68DA693B68DB681340002BD1
:10DB000002D040F2A66300E0002318461837BD4655
:10DB100080BD00BFE0600100E8620100D460010048
:10DB200080B586B000AF7860396000237B61002348
:10DB30003B613B685B6803F00303002B06D03B6846
:10DB40005B6823F003031A1D3B685A603B689B68BF
:10DB50003A68526802FB03F39B08FB6026E000BFB3
:10DB6000786806F0ACFD0246184B1340002BF7D046
:10DB7000786806F0A4FD034603F0B873002B08D0C4
:10DB80003B685B7883F00103DBB2002B01D00123FB
:10DB90003B613B69002B05D17A693968786806F0EA
:10DBA0007AFE78610949786806F095FD3B69002B9B
:10DBB00003D17A69FB689A42D1D30549786806F0A7
:10DBC0008AFD3B6918461837BD4680BD20007001AC
:10DBD0000200700180B586B000AF78603960002324
:10DBE0007B6100233B613B685B6803F00303002B10
:10DBF00006D03B685B6823F003031A1D3B685A603C
:10DC00003B689B683A68526802FB03F39B08FB6021
:10DC100026E000BF786806F052FD0246254B13400F
:10DC2000002BF7D0786806F04AFD034603F0B8737E
:10DC3000002B08D03B685B7883F00103DBB2002B3C
:10DC400001D001233B613B69002B05D17A6939681A
:10DC5000786806F072FE78611649786806F03BFD38
:10DC60003B69002B03D17A69FB689A42D1D300BF8C
:10DC7000786806F024FD02460F4B1340002BF7D0C6
:10DC8000786806F01CFD034603F0B873002B08D03B
:10DC90003B685B7883F00103DBB2002B01D00123EA
:10DCA0003B610549786806F016FD3B691846183750
:10DCB000BD4680BD100070010200700180B584B0C7
:10DCC00000AF786039600023FB6000BF786806F021
:10DCD000F6FC02460F4B1340002BF7D0786806F095
:10DCE000EEFC034603F47023002B01D00123FB60FC
:10DCF000FB68002B04D139687868FFF7A9FEF8604B
:10DD00000449786806F0E7FCFB6818461037BD4602
:10DD100080BD00BF01000F0080B584B000AF786007
:10DD200039600023FB6000BF786806F0C8FC02463B
:10DD30000E4B1340002BF7D0786806F0C0FC02466B
:10DD40000B4B1340002B08D03B685B7883F001033A
:10DD5000DBB2002B01D00123FB600649786806F096
:10DD6000BAFCFB6818461037BD4680BD0200701132
:10DD7000000070110A00701180B584B000AF7860A7
:10DD800039603B68002B06D1494B4A4A40F22A31A0
:10DD9000494801F091FF3B689B78012B06D1474B26
:10DDA000444A4FF44B71444801F086FF3B689B683E
:10DDB000002B03D03B689B68802B06D9404B3D4A23
:10DDC00040F22E313C4801F077FF3B685B68002B46
:10DDD00003D03B685B68802B06D93A4B354A40F24A
:10DDE0002F31354801F068FF7868FFF709FE364BA0
:10DDF000184606F04AFC7B68DB6A43F0E0627B6809
:10DE0000DA627B689B6AFB607B685B6CBB60FB686B
:10DE100023F44E73FB603B681B78002B03D0FB6838
:10DE200043F00803FB603B685B781B0103F03002A2
:10DE30003B689B781B0203F440731343FA68134357
:10DE4000FB60BB6803F0FF23BB603B685B68DAB232
:10DE50003B689B681B0403F47F031343BA681343B6
:10DE6000BB607B68BA685A647B68FA689A627B68B0
:10DE7000DB6A43F007027B68DA627B68134A5A6305
:10DE80007B6800229A637B68104A1A637B68DB6AAE
:10DE900043F000627B68DA6200BF7B68DB6A03F0F4
:10DEA0000063002BF9D100BF00BF1037BD4680BD15
:10DEB000B45B010004630100D4600100F060010064
:10DEC00018610100686101001100301037017F11F5
:10DED00080B58AB000AFF860B9607A60BB68002B8B
:10DEE00006D15C4B5C4A40F2B3315C4801F0E4FE81
:10DEF0007B68002B03D07A68BB689A4206D9584BDE
:10DF0000554A4FF46D71554801F0D6FE00237B62EF
:10DF100000233B620023FB6100237B610023BB6184
:10DF2000BA687B68B2FBF3F37B627B6AB3F5805F10
:10DF300001D900238AE07B6A002B49D0BA687B6A4A
:10DF4000B2FBF3F37A689A4202D27B6A01337B62B6
:10DF50007B6A102B32D97B6A1B09FB6102E0FB69EB
:10DF60000133FB614FF48073FA69B3FBF2F2F96994
:10DF700001FB02F29B1A002BF1D1FB69012BEED0C1
:10DF80007A6AFB69B2FBF3F33B6202E03B6A01335E
:10DF90003B623B6AFA6902FB03F37A6A9A42F5D85C
:10DFA0003B6A002B01D03B6A00E00123BA68B2FB58
:10DFB000F3F2FB69B2FBF3F3BB610FE07B6A3B62F8
:10DFC0000023FB61BA683B6AB2FBF3F3BB6105E077
:10DFD00000233B620023FB61BB68BB613B6A002BF3
:10DFE00002D03B6A013B3B62FB69002B02D0FB691C
:10DFF0005B08FB61FB68DB6A23F00802FB68DA62FE
:10E00000FB68DB6A7B617B6923F47F2323F47F63F6
:10E010007B613B6A1B01DAB2FB691B029BB21A43AC
:10E020007B69134343F460237B61FB687A69DA629E
:10E0300000BFFB685B6A03F00803002BF9D0FB68A4
:10E04000DB6A43F00802FB68DA62BB6918462837CE
:10E05000BD4680BDB861010010630100D4600100BD
:10E06000CC61010080B582B000AF786039603B6858
:10E07000002B06D1204B214A40F23F41204801F0BD
:10E080001BFE3B681B68B3F5005F06D31D4B1B4AA4
:10E090004FF488611A4801F00FFE3B685B68B3F5E6
:10E0A000803F06D3184B154A40F24141144801F015
:10E0B00003FE7B685B6803F460423B681B68C3F344
:10E0C0000C013B685B681B040B431A437B685A6076
:10E0D0003B689A687B689A603B68DB681B0603F0C4
:10E0E0007C523B681969094B0B401A437B68DA6024
:10E0F00000BF0837BD4680BDB45B0100206301004E
:10E10000D460010000620100546201003700FB008E
:10E1100080B48BB000AFF8607A603B600B46FB7256
:10E1200000237B623B6B3B627B68002B02D03B6829
:10E13000002B05D1FB7A012B0BD0FB7A022B08D0E8
:10E140003B6B002B05D07B6B002B02D0FB7A012BA5
:10E1500002D104237B627FE0FB7A022B08D13B6A69
:10E1600003F00303002B03D04FF4D5637B6273E00D
:10E17000FB7A022B70D17B6B03F00303002B04D0DE
:10E180007B6B23F0030304337B637B6B364AA2FB78
:10E190000323DB0B0133BB613B689B00DB08BA69DF
:10E1A0009A4202D903237B6256E07B687B6100239D
:10E1B000FB6147E03A6A3B6BD31A9B007A6BD31A38
:10E1C000B3F5803F1ED2FB69DB007A6913443A6ADB
:10E1D0005A603A6A3B6BD31A9B007A6BD21AFB697E
:10E1E000DB0079690B4412041A60FB69DB007A6971
:10E1F00013441A68FB69DB0079690B4442F023027F
:10E200001A601CE0FB69DB007A6913443A6A5A60C1
:10E21000FB69DB007A691344144A1A60FB69DB006E
:10E220007A6913441A68FB69DB0079690B4442F090
:10E2300021021A603B6A03F57F43FC333B62FB69B2
:10E240000133FB61FA69BB699A42B3D3FB680022D0
:10E250001A607A68FB689A657B6A18462C37BD4657
:10E260005DF8047B704700BF018000800000FCFF68
:10E2700080B58AB002AFF860B9607A603B603B68F5
:10E28000002B06D13E4B3F4A40F26E513E4801F012
:10E2900013FD0023BB61FB689B6A1B0A03F00303A9
:10E2A000FB773B685B687B613B681B683B617B6914
:10E2B000002B07D03B69002B06D03B699B68B3F568
:10E2C000803F01D3042356E000BFF86806F011FA3E
:10E2D000034603F00103002BF7D13B69002B07D065
:10E2E000F86806F006FA034603F00203002BF4D1A7
:10E2F0003B69002B1FD0BB68002B1CD03B69DB683F
:10E30000002B02D03B69DB6801E03B691B693A697D
:10E3100092683969496801FB02F2F97F0192009322
:10E320007B68BA68F868FFF7F3FEB861BB69002B39
:10E3300001D00023FB77FB7F3A697969F86806F022
:10E34000FEF97969F868FFF7B9FCB861BB69002B81
:10E3500001D0BB690FE03B69002B0BD0FB7F3A6912
:10E36000F968184606F060FBB861BB69002B01D064
:10E37000BB6900E0002318462037BD4680BD00BFC2
:10E38000A862010038630100D460010080B500AFCD
:10E390000B4B1B68002B06D10A4B0B4A40F24B611A
:10E3A0000A4801F089FC0A4B1B68054A12681146AD
:10E3B00008489847BFF34F8F00BF00BF80BD00BF24
:10E3C000F42B0020BC62010050630100D460010006
:10E3D000F82B002000100B4080B500AF054B1B68E8
:10E3E000054A1268114605489847BFF34F8F00BF92
:10E3F00000BF80BD142C0020FC2B002000A0064094
:10E4000080B500AF054B1B68054A526811460548A8
:10E410009847BFF34F8F00BF00BF80BD142C002072
:10E42000FC2B002000B0064080B500AF054B1B68F8
:10E43000054A9268114605489847BFF34F8F00BFC1
:10E4400000BF80BD142C0020FC2B002000C0064023
:10E4500080B500AF054B1B68054AD26811460548D8
:10E460009847BFF34F8F00BF00BF80BD142C002022
:10E47000FC2B002000D0064080B500AF054B1B6888
:10E48000054A1269114605489847BFF34F8F00BFF0
:10E4900000BF80BD142C0020FC2B002000A00E40EB
:10E4A00080B500AF054B1B68054A52691146054807
:10E4B0009847BFF34F8F00BF00BF80BD142C0020D2
:10E4C000FC2B002000B00E4080B500AF0B4BD3F802
:10E4D00088300A4A43F47003C2F88830084B4CF283
:10E4E0002052DA81064B4DF62812DA81044B4FF4A4
:10E4F000E9721A8006F042FB00BF80BD00ED00E02B
:10E500000020054080B483B000AF78600B4B03F56A
:10E51000805304331B6823F040527B681B0703F0D1
:10E52000405306491A4301F5805304331A6000BF73
:10E530000C37BD465DF8047B704700BF0070044097
:10E5400080B400AF054B03F5825304334FF0927251
:10E550001A6000BFBD465DF8047B70470070044040
:10E5600080B483B000AF7860044A7B68136000BF5A
:10E570000C37BD465DF8047B704700BF582B002068
:10E5800080B483B000AF0346FB710B4B1B78DBB24A
:10E5900023F03803DAB2FB79DB00DBB203F0380397
:10E5A000DBB205491343DBB20B7000BF0C37BD462D
:10E5B0005DF8047B704700BF0040064080B500AFA7
:10E5C000FFF7BEFF1048FDF719FD104B1846FFF787
:10E5D000C7FF00231846FFF7D3FF00230C4A002192
:10E5E0001846FDF7ADFD0B48FDF712FB0A4B0B4A31
:10E5F0001A600B494FF4E020FDF726FB0120FFF7DE
:10E6000081FF00BF80BD00BF7C6301000024F400D7
:10E6100070630100746301000C010020000E2707E5
:10E62000006CDC0280B483B000AF0346FB7197F945
:10E630000730002B0BDBFB7903F01F02074997F92A
:10E6400007305B09012000FA02F241F8232000BFE5
:10E650000C37BD465DF8047B704700BF00E100E069
:10E6600080B483B000AF03463960FB7197F907307F
:10E67000002B0ADB3B68DAB20C4997F9073012012C
:10E68000D2B20B4483F800230AE03B68DAB20849AF
:10E69000FB7903F00F03043B1201D2B20B441A764C
:10E6A00000BF0C37BD465DF8047B704700E100E019
:10E6B00000ED00E080B582B000AF786039603B6863
:10E6C0000F2B06D9084B094A40F28621084801F071
:10E6D000F3FA3B68DBB203F00F03DAB27B68DA7659
:10E6E00000BF0837BD4680BD84630100406601005D
:10E6F000BC63010080B582B000AF786039603B68D0
:10E700000F2B05D90B4B0C4A4D210C4801F0D4FAC4
:10E710007A683B6813441B78DBB263F07F03D9B29D
:10E720007A683B6813440A461A7000BF0837BD4632
:10E7300080BD00BF846301002866010018640100E9
:10E7400080B584B000AFF860B9607A60BB680F2B09
:10E7500005D90F4B0F4A6B210F4801F0ADFAFA684B
:10E76000BB6813441B78DBB223F03F03DAB27B684B
:10E77000DBB203F03F03DBB21343D9B2FA68BB68E4
:10E7800013440A461A7000BF1037BD4680BD00BF53
:10E7900084630100146601001864010080B584B030
:10E7A00000AFF8600B467A60FB72FB7A012B06D94A
:10E7B000164B174A40F2D911164801F07DFA7B68D2
:10E7C000002B06D1144B124A4FF4ED71114801F0A1
:10E7D00073FA7B689B681B0403F47F027B685B68A9
:10E7E0001B029BB242EA03017B681B68DBB2FA7A28
:10E7F0001943F86813469B001344DB0003441033AD
:10E80000196000BF1037BD4680BD00BF78640100AD
:10E810005C660100B46401004458010090B585B005
:10E8200000AFF8607B600B46FB721346BB72FB7A4D
:10E83000012B06D9104B114A4FF4F871104801F022
:10E840003BFABB7A012B06D90E4B0C4A40F2F11170
:10E850000B4801F031FAFA7ABC7A7B6898B2F96811
:10E8600013469B0013445B002344063341F8230006
:10E8700000BF1437BD4690BD786401007866010082
:10E88000B46401001065010080B500AF4FF48072E0
:10E8900000212548FFF754FF00212348FFF72AFFF6
:10E8A00000212248FDF7C2FE214A00211F48FDF742
:10E8B000BBFD4FF4947201211B48FFF741FF01217A
:10E8C0001948FFF717FF01211848FDF7AFFE194A55
:10E8D00001211648FDF7A8FD40F229120221124835
:10E8E000FFF72EFF02211048FFF704FF02210F4817
:10E8F000FDF79CFE02210220FFF7B2FE022006F087
:10E900004AF90D4A02210948FDF78EFD002107480A
:10E91000FFF7D0FE01210548FFF7CCFE0221034896
:10E92000FFF7C8FE00BF80BD00100240008000401D
:10E9300000000020200000204000002080B500AF33
:10E940000F491048FCF7FEFD01210E4806F055F96D
:10E95000032319460B4805F013FB00231946094809
:10E9600005F0F2FA074805F057FA0121054806F0CC
:10E9700028F9054A00210348FCF772FE00BF80BD5C
:10E980006465010000B003401001002080B500AFB5
:10E990000F491048FCF7D6FD01210E4806F02DF96D
:10E9A000032319460B4805F0EBFA002319460948E2
:10E9B00005F0CAFA074805F02FFA0121054806F0CC
:10E9C00000F9054A00210348FCF74AFE00BF80BD5C
:10E9D0007065010000B00B401801002080B582B0C6
:10E9E00002AF0C490C48FEF77DFA0220FDF76CF8E7
:10E9F0000346019343F6381300930023032207498B
:10EA00000548FEF7EFFA0121034806F012F900BFAE
:10EA1000BD4680BD7C650100008003409865010013
:10EA200080B582B002AF0C490C48FEF75BFA0220B9
:10EA3000FDF74AF80346019343F638130093002389
:10EA4000012207490548FEF7CDFA0121034806F0E7
:10EA5000F0F800BFBD4680BDA865010000900340EE
:10EA6000C465010080B582B002AF0C490C48FEF7C6
:10EA700039FA0220FDF728F80346019343F63813CC
:10EA800000930023042207490548FEF7ABFA012151
:10EA9000034806F0CEF800BFBD4680BDCC6501003E
:10EAA00000900B40E865010080B500AF084A0949B5
:10EAB0000948FEF737FD4021074805F053FC0021C7
:10EAC0001920FFF7CDFD192006F065F800BF80BDC5
:10EAD00000879303FC6501000070064080B500AF1D
:10EAE00011491248FEF756FE40F2DC510F4806F07D
:10EAF000CDF80F4A00210D48FFF750FE01230022F8
:10EB000000210A48FFF78AFE0A4A01210748FFF759
:10EB100045FE0123002201210448FFF77FFE034840
:10EB200006F0A4F800BF80BD086601000060034045
:10EB3000200100202C01002080B500AF1C491D4899
:10EB4000FEF7A4FE41F26F7200211A4806F0CAF8DF
:10EB5000194A0121174806F0C5F8184A022115483C
:10EB600006F0C0F802220021124806F09EF80222A8
:10EB70000121104806F099F8022202210D4806F002
:10EB800094F801213020FFF76BFD02213120FFF7BF
:10EB900067FD02213220FFF763FD302005F0FBFF07
:10EBA000312005F0F8FF322005F0F5FF00BF80BDF1
:10EBB0001066010000700340BF270900DF930400C6
:10EBC00080B500AF0248FEF7B3FE00BF80BD00BFB6
:10EBD0000090024080B500AF0E48FDF767FB0E497C
:10EBE0000E48FDF7D1FCFFF74FFEFFF7A7FEFFF73A
:10EBF000CDFEFFF7F3FEFFF713FFFFF733FFFFF73D
:10EC00006DFFFFF799FFFFF7DBFF06F07FF800BF0E
:10EC100080BD00BF00100240606501000080004020
:10EC200080B598B000AFDC4806F087F8DB4806F006
:10EC300084F8DB4806F081F8DA4806F07EF8DA4816
:10EC400006F07BF8002387F85C30002387F85D30FE
:10EC500007F15C031A460D21D448FEF79FFB002301
:10EC600087F85830002387F8593007F158031A46BF
:10EC70000E21CE48FEF792FB002387F85430002384
:10EC800087F8553007F154031A460F21C748FEF79D
:10EC900085FB002387F85030002387F8513007F1B7
:10ECA00050031A461021C148FEF778FB002387F86D
:10ECB0004C30002387F84D3007F14C031A461121E0
:10ECC000BA48FEF76BFB012387F84830002387F82A
:10ECD000493007F148031A460021B548FEF75EFBAC
:10ECE000012387F84430002387F8453007F14403B7
:10ECF0001A460121AE48FEF751FB012387F8403048
:10ED0000002387F8413007F140031A460221A84842
:10ED1000FEF744FB012387F83C30002387F83D30A1
:10ED200007F13C031A460321A148FEF737FBA14B2C
:10ED30001B883B8707F138031A460A219C48FEF7D7
:10ED40002DFB9C4B1B88BB8607F134031A460B2115
:10ED50009748FEF723FB012387F83030002387F81C
:10ED6000313007F130031A4610219148FEF716FBA7
:10ED7000012387F82C30002387F82D3007F12C036E
:10ED80001A4611218A48FEF709FB012387F828302B
:10ED9000002387F8293007F128031A4612218448F6
:10EDA000FEF7FCFA012387F82430002387F825308A
:10EDB00007F124031A4613217D48FEF7EFFA0123D9
:10EDC00087F82030002387F8213007F120031A4606
:10EDD00001217948FEF7E2FA01233B7700237B7794
:10EDE00007F11C031A4602217348FEF7D7FA0123E4
:10EDF0003B7600237B7607F118031A4605216E48FF
:10EE0000FEF7CCFA01233B7500237B7507F1140351
:10EE10001A4606216848FEF7C1FA01233B74002315
:10EE20007B7407F110031A4607216348FEF7B6FA10
:10EE300001233B7300237B7307F10C031A4608215F
:10EE40005D48FEF7ABFA01233B7200237B7207F1AA
:10EE500008031A4605215948FEF7A0FA01233B7121
:10EE600000237B713B1D1A4606215448FEF796FA93
:10EE700000233B7000237B703B461A461A21504802
:10EE8000FEF78CFA03220C214E4805F070FF012298
:10EE90000D214C4805F06BFF0B220D21494805F070
:10EEA00083FF01220E21474805F061FF0B220E214E
:10EEB000444805F079FF01220F21424805F057FF31
:10EEC0000B220F213F4805F06FFF012210213D4822
:10EED00005F04DFF0B2210213A4805F065FF012295
:10EEE0001121384805F043FF0B221121354805F068
:10EEF0005BFF344B5B6C23F0807323F00303314AD8
:10EF000043F003035364012200212F4805F02FFF33
:10EF1000012201212C4805F02AFF01220A212A485A
:10EF200005F025FF01220B21274805F020FF0122D3
:10EF30001021254805F01BFF01221121224805F070
:10EF400016FF01221221204805F011FF0122132192
:10EF50001D4805F00CFF012202211B4805F007FFA8
:10EF600001220321184805F002FF01220121174860
:10EF700005F0FDFE02220A21144805F0F8FE134BAD
:10EF80009B6A23F0807323F06303104A43F061030C
:10EF9000936202220B211BE0090038100A0038108E
:10EFA0000B0038100C0038100D00381000F00F4026
:10EFB00040F00F409866010080F00F40C0F00F4015
:10EFC00000F10F400090044000A0044000B0044055
:10EFD000684805F0CCFE674BDB6A23F0807323F0B2
:10EFE0006303644A43F06103D36201220221614852
:10EFF00005F0BDFE042203215E4805F0B8FE0122A3
:10F0000005215C4805F0B3FE01220621594805F0B0
:10F01000AEFE01220721574805F0A9FE0122082172
:10F02000544805F0A4FE04220021534805F09FFE39
:10F0300004220121504805F09AFE042202214E4884
:10F0400005F095FE042203214B4805F090FE0422B2
:10F050000421494805F08BFE01220521464805F0B0
:10F0600086FE01220621444805F081FE0422072184
:10F07000414805F07CFE04220021404805F077FE5F
:10F080003E4B1B6823F0807323F043033B4A43F05D
:10F090004303136004220121384805F068FE374B12
:10F0A0005B6823F0807323F04303344A43F0430347
:10F0B000536004220221314805F059FE2F4B9B6812
:10F0C00023F0807323F043032C4A43F04103936001
:10F0D00001221921294805F04AFE01221A21274858
:10F0E00005F045FE254B9B6E23F0807323F0030350
:10F0F000224A43F002039366042203211F4805F0CD
:10F1000036FE1E4BDB6823F0807323F043031B4A5B
:10F1100043F04303D36004220421184805F027FE7E
:10F12000164B1B6923F0807323F04303134A43F00B
:10F130004303136104220521104805F018FE0F4B0C
:10F140005B6923F0807323F043030C4A43F04303CD
:10F1500053610B4B03F580530C331B68084923F4B0
:10F16000402201F580530C331A6000BF6037BD4662
:10F1700080BD00BF00B0044000C0044000D0044087
:10F180000070044081F0004102E000BF83F00043C2
:10F1900030B54FEA41044FEA430594EA050F08BF32
:10F1A00090EA020F1FBF54EA000C55EA020C7FEAF6
:10F1B000645C7FEA655C00F0E2804FEA5454D4EB73
:10F1C0005555B8BF6D420CDD2C4480EA020281EA3D
:10F1D000030382EA000083EA010180EA020281EA75
:10F1E0000303362D88BF30BD11F0004F4FEA0131C7
:10F1F0004FF4801C4CEA113102D0404261EB4101D6
:10F2000013F0004F4FEA03334CEA133302D052425B
:10F2100063EB430394EA050F00F0A780A4F1010417
:10F22000D5F1200E0DDB02FA0EFC22FA05F2801851
:10F2300041F1000103FA0EF2801843FA05F3594137
:10F240000EE0A5F120050EF1200E012A03FA0EFCB6
:10F2500028BF4CF0020C43FA05F3C01851EBE371E0
:10F2600001F0004507D54FF0000EDCF1000C7EEBFD
:10F2700000006EEB0101B1F5801F1BD3B1F5001F3B
:10F280000CD349085FEA30004FEA3C0C04F101045A
:10F290004FEA445212F5800F80F09A80BCF1004F83
:10F2A00008BF5FEA500C50F1000041EB045141EA05
:10F2B000050130BD5FEA4C0C404141EB0101013CCE
:10F2C00028BFB1F5801FE9D291F0000F04BF0146BD
:10F2D0000020B1FA81F308BF2033A3F10B03B3F18F
:10F2E00020020CDA0C3208DD02F1140CC2F10C021F
:10F2F00001FA0CF021FA02F10CE002F11402D8BF7D
:10F30000C2F1200C01FA02F120FA0CFCDCBF41EA48
:10F310000C019040E41AA2BF01EB0451294330BD17
:10F320006FEA04041F3C1CDA0C340EDC04F11404F4
:10F33000C4F1200220FA04F001FA02F340EA0300CB
:10F3400021FA04F345EA030130BDC4F10C04C4F111
:10F35000200220FA02F001FA04F340EA03002946F1
:10F3600030BD21FA04F0294630BD94F0000F83F43B
:10F37000801306BF81F480110134013D4EE77FEA1E
:10F38000645C18BF7FEA655C29D094EA050F08BF6A
:10F3900090EA020F05D054EA000C04BF194610464B
:10F3A00030BD91EA030F1EBF0021002030BD5FEA8F
:10F3B000545C05D14000494128BF41F0004130BDB7
:10F3C00014F580043CBF01F5801130BD01F000450B
:10F3D00045F0FE4141F470014FF0000030BD7FEA7E
:10F3E000645C1ABF194610467FEA655C1CBF0B4679
:10F3F000024650EA013406BF52EA033591EA030F90
:10F4000041F4002130BD00BF90F0000F04BF002187
:10F41000704730B54FF4806404F132044FF00005BA
:10F420004FF0000150E700BF90F0000F04BF002133
:10F43000704730B54FF4806404F1320410F0004599
:10F4400048BF40424FF000013EE700BF42004FEA94
:10F45000E2014FEA31014FEA02701FBF12F07F4311
:10F4600093F07F4F81F06051704732F07F4208BFC8
:10F47000704793F07F4F04BF41F40021704730B5CF
:10F480004FF4607401F0004521F000411CE700BF1B
:10F4900050EA010208BF704730B54FF000050AE09E
:10F4A00050EA010208BF704730B511F0004502D59F
:10F4B000404261EB41014FF4806404F132045FEAA1
:10F4C000915C3FF4D8AE4FF003025FEADC0C18BF4A
:10F4D00003325FEADC0C18BF033202EBDC02C2F13C
:10F4E000200300FA03FC20FA02F001FA03FE40EACE
:10F4F0000E0021FA02F11444BDE600BF70B54FF0D2
:10F50000FF0C4CF4E06C1CEA11541DBF1CEA1355AF
:10F5100094EA0C0F95EA0C0F00F0DEF82C4481EA17
:10F52000030621EA4C5123EA4C5350EA013518BF37
:10F5300052EA033541F4801143F4801338D0A0FB24
:10F5400002CE4FF00005E1FB02E506F00042E0FBD1
:10F5500003E54FF00006E1FB03569CF0000F18BFD7
:10F560004EF0010EA4F1FF04B6F5007F64F540747F
:10F5700004D25FEA4E0E6D4146EB060642EAC62112
:10F5800041EA55514FEAC52040EA5E504FEACE2E7F
:10F59000B4F1FD0C88BFBCF5E06F1ED8BEF1004F82
:10F5A00008BF5FEA500E50F1000041EB045170BDFE
:10F5B00006F0004646EA010140EA020081EA030142
:10F5C000B4EB5C04C2BFD4EB0C0541EA045170BD3E
:10F5D00041F480114FF0000E013C00F3AB8014F1B8
:10F5E000360FDEBF002001F0004170BDC4F1000401
:10F5F000203C35DA0C341BDC04F11404C4F1200582
:10F6000000FA05F320FA04F001FA05F240EA0200DC
:10F6100001F0004221F0004110EBD37021FA04F612
:10F6200042EB06015EEA430E08BF20EAD37070BDCC
:10F63000C4F10C04C4F1200500FA04F320FA05F02B
:10F6400001FA04F240EA020001F0004110EBD3702D
:10F6500041F100015EEA430E08BF20EAD37070BD9D
:10F66000C4F1200500FA05F24EEA020E20FA04F376
:10F6700001FA05F243EA020321FA04F001F0004125
:10F6800021FA04F220EA020000EBD3705EEA430E96
:10F6900008BF20EAD37070BD94F0000F0FD101F0C5
:10F6A0000046400041EB010111F4801F08BF013CFE
:10F6B000F7D041EA060195F0000F18BF704703F03C
:10F6C0000046520043EB030313F4801F08BF013DC3
:10F6D000F7D043EA0603704794EA0C0F0CEA13557F
:10F6E00018BF95EA0C0F0CD050EA410618BF52EA39
:10F6F0004306D1D181EA030101F000414FF000003F
:10F7000070BD50EA410606BF1046194652EA43064C
:10F7100019D094EA0C0F02D150EA013613D195EAC0
:10F720000C0F05D152EA03361CBF104619460AD108
:10F7300081EA030101F0004141F0FE4141F4700112
:10F740004FF0000070BD41F0FE4141F4780170BD02
:10F7500070B54FF0FF0C4CF4E06C1CEA11541DBF67
:10F760001CEA135594EA0C0F95EA0C0F00F0A7F869
:10F77000A4EB050481EA030E52EA03354FEA013196
:10F7800000F088804FEA03334FF0805545EA1313A9
:10F7900043EA12634FEA022245EA111545EA106571
:10F7A0004FEA00260EF000419D4208BF964244F108
:10F7B000FD0404F5407402D25B084FEA3202B61A27
:10F7C00065EB03055B084FEA32024FF480104FF4FB
:10F7D000002CB6EB020E75EB030E22BFB61A75466F
:10F7E00040EA0C005B084FEA3202B6EB020E75EB02
:10F7F000030E22BFB61A754640EA5C005B084FEA6A
:10F800003202B6EB020E75EB030E22BFB61A754636
:10F8100040EA9C005B084FEA3202B6EB020E75EB41
:10F82000030E22BFB61A754640EADC0055EA060E02
:10F8300018D04FEA051545EA16754FEA06164FEA45
:10F84000C30343EA52734FEAC2025FEA1C1CC0D1F1
:10F8500011F4801F0BD141EA00014FF000004FF07E
:10F86000004CB6E711F4801F04BF01430020B4F13F
:10F87000FD0C88BFBCF5E06F3FF6AFAEB5EB030CF7
:10F8800004BFB6EB020C5FEA500C50F1000041EBF4
:10F89000045170BD0EF0004E4EEA113114EB5C04C1
:10F8A000C2BFD4EB0C0541EA045170BD41F4801194
:10F8B0004FF0000E013C90E645EA060E8DE60CEA9C
:10F8C000135594EA0C0F08BF95EA0C0F3FF43BAFB9
:10F8D00094EA0C0F0AD150EA01347FF434AF95EA70
:10F8E0000C0F7FF425AF104619462CE795EA0C0F54
:10F8F00006D152EA03353FF4FDAE1046194622E721
:10F9000050EA410618BF52EA43067FF4C5AE50EAFA
:10F9100041047FF40DAF52EA43057FF4EBAE12E7EA
:10F920004FEA4102B2F1E04324BFB3F5001CDCF121
:10F93000FE5C0DD901F0004C4FEAC0024CEA507059
:10F94000B2F1004F40EB830008BF20F00100704788
:10F9500011F0804F21D113F13872BCBF01F000408B
:10F96000704741F480114FEA5252C2F11802C2F1BD
:10F97000200C10FA0CF320FA02F018BF40F001003E
:10F980004FEAC1234FEAD32303FA0CFC40EA0C00F0
:10F9900023FA02F34FEA4303CCE77FEA625307D12D
:10F9A00050EA01331EBF4FF0FE4040F44000704764
:10F9B00001F0004040F0FE4040F40000704700BFFE
:10F9C00053B94AB9002908BF00281CBF4FF0FF31C6
:10F9D0004FF0FF3000F06EB9ADF1080C6DE904CEC8
:10F9E00000F006F8DDF804E0DDE9022304B070471A
:10F9F0002DE9F047089D04468C46002B40F083809B
:10FA00008A42174647D9B2FA82F242B1C2F12000C7
:10FA100024FA00F09140974040EA010C94404FEAEC
:10FA20001748230CBCFBF8F61FFA87FE08FB16C12B
:10FA300043EA014306FB0EF1994209D9FB1806F18E
:10FA4000FF3080F01981994240F21681023E3B441A
:10FA50005B1AA4B2B3FBF8F008FB103344EA03448A
:10FA600000FB0EFEA64509D93C1900F1FF3380F0DA
:10FA70000581A64540F2028102383C4440EA064036
:10FA8000A4EB0E0400261DB1D4400023C5E90043B9
:10FA90003146BDE8F08702B9FFDEB2FA82F2002AF1
:10FAA00050D1CB1B4FEA174E1FFA87F80126B3FB44
:10FAB000FEFC210C0EFB1C3341EA034108FB0CF356
:10FAC0008B4207D979180CF1FF3002D28B4200F239
:10FAD000E9808446C91AA3B2B1FBFEF00EFB1011F7
:10FAE00043EA014408FB00F8A04507D93C1900F19E
:10FAF000FF3302D2A04500F2D9801846A4EB0804D7
:10FB000040EA0C40BFE78B4209D9002D00F0B180DC
:10FB10000026C5E9000130463146BDE8F087B3FA5A
:10FB200083F6002E4AD18B4202D3824200F2B88083
:10FB3000841A61EB030101208C46002DA8D0C5E991
:10FB4000004CA5E7C2F1200320FA03F6974001FA22
:10FB500002F04FEA174ED9403043030CB1FBFEF6DA
:10FB60001FFA87F80EFB161143EA014306FB08F162
:10FB7000994204FA02F409D9FB1806F1FF3C80F01F
:10FB80008D80994240F28A80023E3B445B1A81B2EA
:10FB9000B3FBFEF00EFB103341EA034100FB08F318
:10FBA0008B4207D9791800F1FF3C73D28B4271D98F
:10FBB00002383944CB1A40EA064678E7C6F1200CF1
:10FBC00003FA06F422FA0CF31C4320FA0CF701FAAC
:10FBD00006F34FEA144E21FA0CF11F433B0CB1FB24
:10FBE000FEF91FFA84F80EFB191143EA014109FBE3
:10FBF00008FA8A4502FA06F200FA06F308D96118F3
:10FC000009F1FF3048D28A4546D9A9F102092144B9
:10FC1000A1EB0A01BFB2B1FBFEF00EFB101147EAE7
:10FC2000014700FB08F8B84507D9E71900F1FF3193
:10FC30002ED2B8452CD90238274440EA0940A7EB18
:10FC40000807A0FB02894F45C64649461AD317D07C
:10FC50005DB1B3EB0E0267EB010707FA0CFCF24053
:10FC60004CEA0202F740C5E9002700263146BDE80C
:10FC7000F0872E4628460BE70646E9E61846FDE6DD
:10FC80004345E5D2B8EB020E69EB04010138DFE72A
:10FC90000846D2E760468DE78146B9E7664675E7D4
:10FCA00030464AE7ACF1020C394413E702383C44D1
:10FCB00024E700BF704700BF1FB514461A46094B22
:10FCC0001B680546D8684CB1074B0091CDE901345B
:10FCD00006492B4600F00EF805F047F9044B1C4688
:10FCE000F3E700BF38010020306701003D670100E5
:10FCF0006B6701000EB403B5014603AB054853F82A
:10FD0000042B0068019300F0D5F802B05DF804EB15
:10FD100003B070473801002070B50D4D0D4C641BC9
:10FD2000A4100026A64209D10B4D0C4C06F03CFD58
:10FD3000641BA4100026A64205D170BD55F8043BF3
:10FD400098470136EEE755F8043B98470136F2E74D
:10FD5000B8670100B8670100B8670100C06701001B
:10FD600037B5002948D051F8043C0190002BA1F18F
:10FD70000404B8BFE41800F085FD204A0198136818
:10FD8000154633B96360146003B0BDE8304000F03D
:10FD90007FBDA3420BD921686218934204BF1A6841
:10FDA0005B68636004BF521822602C60ECE71A465F
:10FDB0005B680BB1A342FAD911685518A5420BD163
:10FDC000246821445418A3421160DDD11C685B688B
:10FDD000536021441160D7E702D90C230360D3E7B5
:10FDE000256861198B4204BF19685B68636004BFB2
:10FDF000491921605460C7E703B030BD182C0020BA
:10FE0000F8B5CD1C25F0030508350C2D38BF0C25A1
:10FE1000002D064601DBA94203D90C2333600020E4
:10FE2000F8BD00F02FFD21490A6814469CB9204F07
:10FE30003B6823B92146304600F092FA38602946E3
:10FE4000304600F08DFA431C23D10C23336030463A
:10FE500000F01EFDE3E723685B1B17D40B2B03D9CF
:10FE600023601C44256004E06368A2420CBF0B6061
:10FE70005360304600F00CFD04F10B00231D20F010
:10FE80000700C21ACCD01B1AA350C9E722466468E7
:10FE9000CCE7C41C24F00304A042E3D0211A30466E
:10FEA00000F05EFA0130DDD1CFE700BF182C002052
:10FEB0001C2C00202DE9F04F0D469DB014469846AD
:10FEC000064618B183690BB900F01EFC894B9D42B0
:10FED0001BD175686B6ED90705D4AB899A0502D41E
:10FEE000A86D05F07FF8AB891B0701D52B69EBB92D
:10FEF0002946304600F096FAC0B16B6EDC070ED58D
:10FF00004FF0FF301DB0BDE8F08F7B4B9D4201D11B
:10FF1000B568DFE7794B9D4208BFF568DAE7AB8942
:10FF20009805EDD4A86D05F05EF8E9E70023099384
:10FF300020238DF82930CDF80C803023DFF8C081E4
:10FF40008DF82A304FF0010923469A4613F8012B09
:10FF50000AB1252AF9D1BAEB040B0BD05B46224635
:10FF60002946304604F082FF013000F0AA80099A49
:10FF70005A4409929AF80030002B00F0A280002326
:10FF80004FF0FF32CDE905230AF1010A04930793EC
:10FF90008DF853301A935446052214F8011B584823
:10FFA000F0F736FA049AD8B9D10644BF20238DF869
:10FFB0005330130744BF2B238DF853309AF8003089
:10FFC0002A2B15D0079A544600204FF00A0C2146E0
:10FFD00011F8013B303B092B4ED9B0B1079214E028
:10FFE000A0EB080309FA03F313430493A246D2E7F4
:10FFF000039B191D1B680391002BBBBF5B4242F0A2
:020000021000EC
:10000000020207930793B8BF049223782E2B0CD1DA
:1000100063782A2B35D1039B1A1D1B680392002B92
:10002000B8BF4FF0FF3302340593DFF8E4A0217826
:1000300003225046F0F7ECF940B14023A0EB0A0050
:1000400003FA00F0049B03430134049314F8011BEA
:100050002C488DF828100622F0F7DAF900283FD056
:10006000294B1BBB039B073323F007030833039380
:10007000099B3B44099367E70CFB02320C460120C5
:10008000A5E700230134059319464FF00A0C2046DA
:1000900010F8012B303A092A03D9002BC5D005915D
:1000A000C3E70CFB012104460123F0E703AB0093F7
:1000B0002A46164B04A93046AFF300800746781C49
:1000C000D6D16B6ED90705D4AB899A0502D4A86D39
:1000D00004F089FFAB895B063FF512AF099811E781
:1000E00003AB00932A46094B04A9304600F012F8EE
:1000F000E4E700BFC0660100E0660100A066010001
:100100006C67010076670100000000006D4E010081
:10011000726701002DE9FF470C469146277E0C9936
:10012000782F80469A4604F1430207D8622F0AD8F6
:10013000002F00F0D880582F00F0A38004F1420671
:1001400084F842703AE0A7F16303152BF6D801A0BA
:1001500050F823F0AD010100C10101003D01010093
:100160003D0101003D0101003D010100C10101000F
:100170003D0101003D0101003D0101003D01010083
:10018000CD020100F1010100AF0201003D010100BB
:100190003D010100EF0201003D010100F1010100FC
:1001A0003D0101003D010100B70201000B681A1D6D
:1001B0001B680A6004F1420684F842300123A3E080
:1001C000256808682E0600F104030AD505680B604F
:1001D000002D03DA2D236D4284F843305E480A2354
:1001E00019E015F0400F05680B6018BF2DB2EFE75E
:1001F0000B682568181D0860280601D51D6802E0F7
:100200006906FBD51D8854486F2F0CBF08230A23AD
:10021000002184F843106668A660002EA2BF216802
:1002200021F0040121600DB9002E4DD01646B5FB1A
:10023000F3F103FB1157C75D06F8017D2F46BB4262
:100240000D46F4D9082B0BD12368DF0708D52369A5
:1002500061689942DEBF302306F8013C06F1FF36A3
:10026000921B2261CDF800A04B4603AA21464046CE
:1002700004F00EFE01304CD14FF0FF3004B0BDE869
:10028000F087354884F8457023680E681F0656F8D5
:10029000045B0E6014D5D90744BF43F020032360EC
:1002A0001DB9236823F0200323601023B0E72368DF
:1002B00043F0200323607823284884F84530E3E79F
:1002C0005E0648BFADB2E6E71646BBE70B68266898
:1002D00060691D1D0D6035061B6801D5186002E0C0
:1002E0007106FBD51880002323611646BAE70B6818
:1002F0001A1D0A601E68626800213046F0F788F80F
:1003000008B1801B606063682361002384F8433078
:10031000A8E72369324649464046D0470130ABD072
:1003200023689B0713D4E068039B9842B8BF184624
:10033000A4E70123324649464046D04701309BD0CE
:100340000135E36803995B1AAB42F2DCEBE7002569
:1003500004F11906F5E700BF7D6701008E67010013
:1003600038B5064D0023044608462B6001F06CFAB0
:10037000431C02D12B6803B1236038BD902C0020B0
:10038000F8B50E461446054618B183690BB900F05E
:10039000BBF9214B9C422BD16C68A369A360A38954
:1003A0001A072FD523696BB323692068C01A6369C4
:1003B000F6B28342374604DC2146284600F026F98F
:1003C00030BBA368013BA36023685A1C22601E70E7
:1003D00063690130834204D0A389DB0706D50A2E66
:1003E00004D12146284600F011F988B93846F8BDF5
:1003F0000A4B9C4201D1AC68CFE7094B9C4208BF35
:10040000EC68CAE72146284600F00CF80028CBD05B
:100410004FF0FF37EAE700BFC0660100E066010069
:10042000A0660100324B70B51D6806460C4625B12A
:10043000AB6913B9284600F067F92E4B9C420FD1E7
:100440006C68A389B4F90C2019072CD4DD0611D4EB
:100450000923336042F04003A3814FF0FF303EE0B8
:10046000254B9C4201D1AC68EBE7244B9C4208BF72
:10047000EC68E6E7580712D5616B41B104F144031B
:10048000994202D03046FFF76BFC00236363A389D7
:1004900023F02403A3810023636023692360A389DD
:1004A00043F00803A38123694BB9A38903F42073A4
:1004B000B3F5007F03D02146304600F0A3F9A089B0
:1004C000B4F90C2010F001030AD00023A360636983
:1004D0005B42A361236943B910F08000BAD170BDBB
:1004E000810758BF6369A360F4E70020F7E700BF06
:1004F00038010020C0660100E0660100A06601002E
:100500008A892DE9F041054610070C4658D44B68FE
:10051000002B05DC0B6C002B02DC0020BDE8F08119
:10052000E66A002EF9D0002312F480522F682B6067
:1005300032D0606DA3895A0705D56368C01A636B12
:100540000BB1236CC01A00230246E66A216A2846D2
:10055000B047431CA38906D129681D292CD82A4AF3
:10056000CA40D60728D500226260D90422692260D9
:1005700004D5421C01D12B6803B96065616B2F6003
:100580000029CAD004F14403994202D02846FFF75B
:10059000E7FB00206063C1E7216A01232846B047DA
:1005A000411CC7D12B68002BC4D01D2B01D0162BAA
:1005B00001D12F60B1E7A38943F04003A381ADE7E8
:1005C0000F69002FA9D093070E6808BF4B690F6011
:1005D00018BF0023A6EB07088B60B8F1000F9CDD65
:1005E000216AA66A43463A462846B047002806DCF8
:1005F000A38943F04003A3814FF0FF308EE7074407
:10060000A8EB0008E9E700BF0100402038B50B69FE
:1006100005460C4613B90025284638BD18B1836934
:100620000BB900F071F8144B9C421BD16C68B4F903
:100630000C30002BEFD0626ED00704D4990502D4A1
:10064000A06D04F0CFFC28462146FFF759FF636EEA
:10065000DA070546E0D4A3899B05DDD4A06D04F03C
:10066000C2FCD9E7054B9C4201D1AC68DFE7044BE3
:100670009C4208BFEC68DAE7C0660100E066010052
:10068000A0660100002310B50446C0E90033C0E9AC
:100690000433836081814366C281836119460822E5
:1006A0005C3004F0C4FB054B6362054BA362054B51
:1006B000E362054B2462236310BD00BF8550010037
:1006C000A7500100DF50010003510100014904F06F
:1006D00069BC00BF0D060100014804F083BC00BFE7
:1006E0009C2C0020014804F07EBC00BF9C2C002004
:1006F000014804F077BC00BF972C0020014804F0AB
:1007000072BC00BF972C002010B50446FFF7F0FF25
:10071000A3691BB1BDE81040FFF7F0BFC4E9123375
:100720002365134B134A1B68A262A34204BF012333
:10073000A361204600F020F86060204600F01CF81D
:10074000A060204600F018F80022E06004216068F4
:10075000FFF798FFA06801220921FFF793FFE068E7
:1007600002221221FFF78EFF0123A361D2E700BF0F
:100770009C660100CD060100F8B50746FFF7ACFF07
:100780001E4B1E68B36913B93046FFF7BDFF4836EC
:10079000D6E90134013B03D533680BB33668F7E77C
:1007A000B4F90C50D5B9164BE36004F158006566F6
:1007B00004F017FCFFF796FFC4E90155C4E904559E
:1007C0002560A5610822294604F15C0004F02FFB96
:1007D000C4E90D55C4E912552046F8BD6834D9E77F
:1007E0000421384604F0C8FB044630600028D5D107
:1007F000FFF778FF0C233B60EEE700BF9C6601002B
:100800000100FFFF8B8973B59D0706460C4607D58F
:1008100004F14703236023610123636102B070BDCB
:1008200001AB6A4604F0E0FB009905463046FFF74D
:10083000E7FA48B9B4F90C309A05EFD423F0030372
:1008400043F00203A381E3E70D4BB362A389206069
:1008500043F08003A381009B6361019B20615BB136
:10086000B4F90E10304600F067F828B1A38923F0E0
:10087000030343F00103A381A0890543A581CDE7CC
:10088000CD060100014804F0ADBB00BF982C00204C
:10089000014804F0A8BB00BF982C0020024B014681
:1008A000186804F0C5BB00BF3801002038B5074DFB
:1008B00000230446084611462B6000F0E3FF431C6A
:1008C00002D12B6803B1236038BD00BF902C0020FB
:1008D00038B5074D04460846114600222A601A46DC
:1008E00004F0AEFC431C02D12B6803B1236038BD79
:1008F000902C002038B5064D0023044608462B6096
:1009000001F038F8431C02D12B6803B1236038BDD5
:10091000902C002038B5074D0023044608461146A8
:100920002B6004F0DFFC431C02D12B6803B1236071
:1009300038BD00BF902C002038B5064D002304467A
:1009400008462B6004F0DCFC431C02D12B6803B189
:10095000236038BD902C002038B5074D044608466A
:10096000114600222A601A4604F058FC431C02D1AA
:100970002B6803B1236038BD902C002038B5074D9B
:1009800004460846114600222A601A4604F0EFFB8E
:10099000431C02D12B6803B1236038BD902C00208A
:1009A00008B52DED028BF0EE408AB0EE608A00F0C3
:1009B00015F820B9B0EE480ABDEC028B08BDB0EEC8
:1009C000480A00F00BF820B1F4EEC88AF1EE10FAF4
:1009D000F0D5B0EE680ABDEC028B08BD10EE103AFF
:1009E00033F000400ED0A0F50003B3F1FE4F0DD35D
:1009F000074B421E9A4207D9A0F1FF40B0FA80F09F
:100A00004009704702207047032070470420704758
:100A1000FEFF7F00D0B52DED028B3B4C8AB0F0EE8F
:100A2000408A00F027FA94F900300133B0EE408A92
:100A300012D0B0EE680A00F023FE68B1DFED337A21
:100A4000F4EEE78AF1EE10FA40DCDFED317AF4EEF5
:100A5000E78AF1EE10FA05D4B0EE480A0AB0BDEC10
:100A6000028BD0BD04232B4A009318EE900A00237A
:100A700008930192FEF7EAFC94F900300026002763
:100A8000022BCDE90401CDE90201CDE9066718D0BA
:100A9000684600F0EBFDA0B1089B002B2ED1DDE9EC
:100AA0000601FEF73DFF08EE100AB0EE480A0AB054
:100AB000BDEC028BD0BD18490020022BCDE9060108
:100AC000E6D100F0A9FF22230360E5E70323114AE2
:100AD000009318EE900A002308930192FEF7B6FCEB
:100AE00094F90030CDE90401CDE90201002BE2D1F7
:100AF0000A4B4FF06042CDE90623C9E700F08CFFB6
:100B0000089B0360CBE700BF9C0100208071B142CD
:100B1000B5F1CFC2006701000000F07FFFFFEF4793
:100B2000F0B52DED048BB84D8BB0F0EE408AB0EEF1
:100B3000608A00F097FA95F90040631CB0EE409A85
:100B400033D0B4EE488AF1EE10FA2ED6F4EE688A6D
:100B5000F1EE10FA80F19C80DFEDAC9AF4EE698A38
:100B6000F1EE10FA27D1B4EE698AF1EE10FA5FD1F6
:100B70000123A74A009318EE900A002301920893DC
:100B8000FEF764FC02460B4618EE100ACDE902237C
:100B9000FEF75CFC00220023CDE90401CDE9062329
:100BA000002C00F09580B7EE009AB0EE490A0BB029
:100BB000BDEC048BF0BD00F063FD0446002800F09E
:100BC0009E80B5EE409AF1EE10FAEED1B0EE680AD2
:100BD00000F056FD0028E8D0B0EE480A00F050FDC5
:100BE0000028E2D004238A4A009318EE900A0023DA
:100BF00001920893FEF72AFC02460B4618EE100AF3
:100C0000CDE90223FEF722FC95F9003000260027EB
:100C1000022BCDE90401CDE9066704D0684600F057
:100C200025FD002859D100F0F7FE2223036054E08F
:100C3000B0EE480A00F024FD0028B6D0B5EEC08A18
:100C4000F1EE10FAB1D50123714A009318EE900A23
:100C5000002301920893FEF7F9FB02460B4618EEBB
:100C6000100ACDE90223FEF7F1FB95F90030CDE93A
:100C70000401002B40F0818000220023CDE90623EF
:100C8000684600F0F3FC00287ED0089B5BB326E0AA
:100C9000B5EE408AF1EE10FA87D101235C4A009349
:100CA00018EE900A002301920893FEF7CFFB02464C
:100CB0000B4618EE100ACDE90223FEF7C7FB554B91
:100CC0000022022CCDE90401CDE906233FF46BAFED
:100CD000684600F0CBFC00285BD0089B1BB100F0FD
:100CE0009BFE089B0360DDE90601FEF719FE09EE95
:100CF000100AB0EE490A0BB0BDEC048BF0BDB0EEAB
:100D0000680A00F0BDFC00283FF45BAFB0EE480A73
:100D100000F0B6FC00283FF454AFB4EE499AF1EE6F
:100D200010FA80F181803A4B0894032218EE900A61
:100D3000CDE90023FEF78AFB02460B4618EE100AA7
:100D4000CDE90223FEF782FB95F90030CDE90401DD
:100D500023BB314BF5EEC08A4FF06042F1EE10FA42
:100D6000CDE9062326D4684600F080FC00288CD10B
:100D700000F052FE2223036087E728490020022B5F
:100D8000CDE906017FF47CAF00F046FE212303602D
:100D90007BE700F041FE212303609EE72049F5EE4A
:100DA000C08A0020F1EE10FACDE9060117D4022B1B
:100DB000DED0D8E7F6EE007A28EE278AB0EE480AB1
:100DC00000F072FCB4EE480AF1EE10FA18D01549A2
:100DD00095F900304FF06040CDE90601E7E7F6EE07
:100DE000007A28EE278AB0EE480A00F05DFCB4EEE7
:100DF000480AF1EE10FA03D0084B0022CDE9062391
:100E000095F90030D3E700BF9C01002000000000EE
:100E1000086701000000F03FFFFFEF470000F0FF10
:100E20000000F07FFFFFEFC7114B0894012218EE7E
:100E3000900ACDE90023FEF709FB02460B4618EEA7
:100E4000100ACDE90223FEF701FB95F90040CDE938
:100E50000401002C3FF410AFC9EEA97A17EE900AF6
:100E6000FEF7F4FA022CCDE906018DD008E700BFA9
:100E70000867010010EE103A23F00042B2F1FF4F74
:100E800057D84FEAD37100F098806448834253DC0E
:100E9000002BC0F28B80624B9A4252D9614B9A422E
:100EA00000F29E80604B614A03EB810393ED004AA0
:100EB00002EB8102C1F1010330EE444A92ED007A67
:100EC0005B1A34EE470ADFED5A7ADFED5A4A9FED9E
:100ED0005A5ADFED5A5A9FED5A6A60EE006AE6EE02
:100EE000A74AF0EE407AA4EEA65AE5EE265AA5EE01
:100EF000A66AE6EE667AF0EE676A002B47D0B0EE9F
:100F0000006A60EE275A76EE676A13F17D0F85EE70
:100F1000A60AF7EE007A37EE400A30EE440A37EEC2
:100F2000C00A51DB10EE102A02EBC35300EE103A58
:100F3000704730EE000A70479FED420A20EE000A2B
:100F40007047B2F1465F0AD2DFED3E7A70EE277A43
:100F5000B7EE007AF4EEC77AF1EE10FA5ADC60EEE2
:100F6000007A9FED335ADFED335A9FED336ADFEDA0
:100F7000336A9FED337AE7EE855AA7EEA56AE7EE6E
:100F8000866AA7EEA67AF0EE406AE7EEC76AB0EE90
:100F9000007A36EEC77A60EE266AB7EE006AC6EED1
:100FA000877A37EEC00A36EE400A7047264B9A42DF
:100FB0007FF671AF9FED250A7047DFED247A002997
:100FC00018BFB0EE670A704710EE102A643302EBC8
:100FD000C353DFED1F7A00EE103A20EE270A704768
:100FE0001C4B9FED1D7A9FED1D6ADFED1D6A03EB23
:100FF0008103D3ED007AE0EE077AB0EE404AFDEED1
:10100000E77AB8EEE77A17EE903AA7EE464A27EE6F
:10101000267A56E730EE070A704700BF1772B142D2
:101020001872B13E9115853F1867010020670100D5
:101030004CBB31330EEADDB555B38A38610B36BB94
:10104000ABAA2A3ECAF24971B5F1CF4200000000B6
:101050000000800D106701003BAAB83F8071313F4E
:10106000D1F717372DE9F04710EE904A34F00048D9
:101070002DED028B15D010EE105A25F00047B7F178
:10108000FF4F10EE109A06DDBDEC028BBA48BDE8AA
:10109000F04700F003BBB8F1FF4F08DDB7F17E5F0A
:1010A000F2D1B7EE000ABDEC028BBDE8F087002D4F
:1010B00010EE906AC0F2F6804FF0000AB8F1FF4FD0
:1010C00000F00481B8F17E5F00F02A81B6F1804F14
:1010D00000F03F81B6F17C5F00EE105A40F00381D2
:1010E000B9F1000F80F23A8100F0C2FAB7F1FF4F78
:1010F00000F00B81002F00F00481B7F17E5F00F05B
:10110000FA804FEAD972013A5AEA020300F02C81C0
:10111000B8F19A4F40F35281984B9F4240F35F825F
:10112000974B9F4200F30181F7EE007A30EE670A99
:10113000DFED946ADFED947ADFED945A9FED946AC7
:10114000B5EE007AE0EE476AB6EE007AA6EEC07A17
:10115000F0EE476A20EE007A27EE267A67EEC77A2D
:10116000E0EE257AF0EE676AE0EE066A16EE903A57
:1011700023F47F6323F00F0307EE103AA0EE467AC4
:1011800006EE903A77EEC77A26F47F6626F00F06D1
:1011900007EE104A06EE106A67EE877A37EE466A67
:1011A00007EE106AE6EE267A0AF1FF3A5AEA0203DF
:1011B00026EE877AB7EE000A77EE876ABFEE006AFE
:1011C00016EE903A0CBFB0EE468AB0EE408A002B85
:1011D00023F0004240F3B981B2F1864F00F3F88169
:1011E00000F0EB81B2F17C5F00F3BB81002210467E
:1011F00023F47F6323F00F0306EE103ADFED656AF8
:10120000DFED655A9FED653ADFED653A9FED652AA2
:101210009FED654ADFED654A9FED655A36EE477AE8
:10122000F0EE002A77EEC77A26EE267AA7EEA57AA8
:10123000F7EE005AF0EE477AA6EE037A67EE076AF9
:10124000F0EE471AE6EE431AB0EE636AA6EE826A43
:1012500077EEE17AA6EE264AE7EE277AE4EE264A12
:10126000A4EEA65AB0EE456AB0EE475AA6EE665A0C
:10127000F0EE456A36EEE26A27EE055AC5EE066ADA
:1012800076EEE77A37EEC77A35EEC70A10EE103AF7
:101290001344B3F5000FC0F2BA8100EE103A20EE0D
:1012A000080A00E7B8F1974F1ADAB8F17E5F0ADB57
:1012B0004FEAE853C3F1960348FA03F202FA03F344
:1012C000434500F03D814FF0000AFBE6B7F17E5F39
:1012D0003FF4E7AE2FDD002E2ADB00EE104AE2E6F7
:1012E0004FF0020AEAE600F0C3F9B7F1FF4F02D06F
:1012F000002F7FF402AF002EBCBFF7EE007A87EE1E
:10130000800AB9F1000FBFF6CEAEA7F17E5757EABB
:101310000A0340F00E8170EE407A87EEA70AC2E61B
:10132000002E0FDB00EE105ABDE6002E00F35A81AE
:101330009FED200AB7E6002EFADA07EE904AB1EEEA
:10134000670AB0E607EE105AF7EE007A87EE870AD2
:10135000A9E607EE905A27EEA70AA4E6BDEC028B99
:10136000BDE8F04700F07EB907EE905A77EEE77AD5
:1013700087EEA70A97E600BFB4610100F7FF7F3F41
:101380000700803FABAAAA3E3BAAB83F70A5EC3647
:1013900000AAB83F8CBEBF351872313F0072313F92
:1013A0000EEADDB54CBB313355B38A38610B36BB21
:1013B000ABAA2A3E000000000000804B19F0FF4F4E
:1013C00040F0F9805FED047A60EE277A6FF0170144
:1013D00017EE907A8F48FB15C7F316077F3B8742BD
:1013E0000B4447F07E5140F3DE808B48874240F348
:1013F000FE80DFED8A4A0133A1F50001F0EE643A88
:101400000020B7EE006A06EE901A76EE867AB7EE06
:10141000007A87EE278A491041F0005101F58021BA
:10142000014436EEC67A07EE901A27EE082A77EEC8
:10143000C65A9FED7B4A7B49DFED7B8A9FED7B0A95
:10144000DFED7B0A9FED7B1ADFED7B1ADFED7B2A58
:101450009FED7B3A9FED7B5A22EE026A12EE100A54
:1014600076EEE56AF0EE445AE6EE285A084004EEBD
:10147000100AA4EE677AF0EE407AE5EE867AA4EEE2
:10148000667AE7EE860A67EE086AB0EE417AA0EE69
:10149000867A72EE047AE7EE061A67EEA67A26EEF0
:1014A000066AF0EE085AE6EE217AB0EE656AA4EE1E
:1014B000046A07EE103A36EE276AB8EEC77A16EEDF
:1014C000103A0B4006EE103A76EE655AE4EE445AB6
:1014D00077EEE57A67EE827AE6EE867AF0EE675A84
:1014E000E4EE065A15EE903A0B4006EE903AE4EE22
:1014F000466A05EE903A77EEE67A67EEA27AE5EE76
:10150000837A77EEA37AF0EE676AE5EE856A76EE87
:10151000A46A76EE876A16EE903A0B4006EE903A91
:1015200036EEC77A37EE647AA5EEC57A77EEC77ADB
:101530002AE6BAF1010F7FF4B6ADB1EE400AB2E58A
:1015400002F00102C2F1020ABCE53F498A4257DCBF
:101550007FF448AE76EEC76AF4EEE76AF1EE10FA71
:101560004EDAD2154FF400017E3A41FA02F21A44E3
:10157000C2F3C751354C7F390C41C2F3160022EA41
:10158000040206EE902A37EE667AC1F1170140F4A4
:1015900000000841002B77EE876AB8BF404216EE84
:1015A000903AC20524E6DFED1D4A0020F0EE643AD1
:1015B000B7EE006A27E700210CE79FED256A76EE7B
:1015C000C76A37EE866AB4EEE66AF1EE10FAC8DD55
:1015D000DFED207A28EE270A20EE270A63E5002EA9
:1015E000BFF6A6AE9FED1B0A20EE000A5BE5DFED1D
:1015F0001A4ADFED1A3A4FF40010B7EE086A02E714
:10160000DFED177A28EE270A20EE270A4BE500F0D7
:10161000A9F844E671C41C00D6B35D0000000000C8
:1016200055326C3E00F0FFFF42F1533E05A38B3E66
:10163000ABAAAA3EB76DDB3E9A99193F4F38763F69
:10164000A0C39D360038763F00001643FFFF7F00A1
:101650003CAA3833CAF2497100C0153FDCCFD135FE
:101660006042A20DB1EEC00A704700BF0020704773
:1016700010EE103A23F0004300EE103A704700BF1E
:1016800082B08DED010A019820F00040B0F1FF4FCB
:10169000ACBF0020012002B0704700BF9FED010ADF
:1016A000704700BF0000C07F10EE101AC1F3C7538F
:1016B000A3F17F02162A21F0004328DC33B310B4D3
:1016C000002A83B04FEAD17027DB244B1341194223
:1016D00018D05C0811EA530307D04FF4001321EA35
:1016E000040113410B4300EE103A1D4B03EB800045
:1016F000D0ED007A37EE800A8DED010A9DED010AEA
:1017000030EE670A03B05DF8044B70477047B3F1E1
:10171000FF4FFBD330EE000A7047C1F316035B4264
:101720000F4A5B0A090D03F480030905194302EB14
:101730008002D2ED006A07EE901A36EEA77A8DEDA0
:10174000017ADDED017A77EEE67A17EE903A23F032
:10175000004343EAC07300EE103AD3E7FFFF7F0077
:101760002867010082B08DED010A019B33F0004231
:101770002AD0B2F1FF4F23D213F0FF4F28D19DEDB5
:10178000017ADFED2A7A2A4B67EE277A9842CDED6F
:10179000017A37DB019BC3F3C752193A0244FE2A90
:1017A0001ADD9FED240A9FED247A019B002BF0EEB9
:1017B000407AB8BFB0EE470A20EE270A02B0704761
:1017C00030EE000A02B070479DED010A02B070478A
:1017D000D20D0244FE2AE4DC002A0BDC12F1160FC3
:1017E00017DA4CF250339842DBDC9FED140A9FED80
:1017F000147ADAE723F0FF4343EAC25300EE103ACB
:1018000002B070479FED0D0ADDED017A27EE800AE8
:10181000D8E7193223F0FF4343EAC253DFED097AD8
:1018200007EE103A27EE270ACCE700BF0000004C75
:10183000B03CFFFFCAF24971CAF249F16042A20D01
:101840006042A28D0000003370B50C4D2B680BB9BF
:101850000B4B2B6003302E6820F0030434442046E9
:1018600000F0AEF810B92C60304670BD00F0D4F82E
:101870000C2303604FF0FF36F6E700BF202C00205A
:10188000A02C0020062930B50CBF044D044D1824AF
:1018900020462946ABBE0446204630BD2300020048
:1018A000260002002DE9F04F234E336885B0002B4F
:1018B0003FD1DFF898A0CDF804A04FF00309CDF890
:1018C0000C90012402930DF1040820464146ABBE62
:1018D00005461A4FCDF804A00423CDF80C903D60C6
:1018E000029320464146ABBE8346154DCDF804A079
:1018F0000823CDF80C90C5F800B00293204641466D
:10190000ABBE04460F4A28681460013404BF2B683C
:1019100013600D4B12684FF0FF31996119623968FD
:1019200019600021C3E90201C3E9042159600123C0
:10193000336005B0BDE8F08F242C00202C2C002053
:10194000302C0020282C0020342C00209F67010020
:10195000042810B5044601D9002010BDFFF7A2FFEE
:10196000034850F834200132F6D000EBC400F4E70D
:10197000342C002038B50546FFF7EAFF044630B99D
:1019800000F04AF8092303604FF0FF3038BD013DF5
:10199000012D09D8094B9A681B699A4204D14FF06E
:1019A000FF3303600020F1E7206803F06BFC0028A0
:1019B000ECD14FF0FF332360E8E700BF342C002068
:1019C000044B23B1984234BF0020012070471846D1
:1019D000704700BFA03C002010B5054C237833B9F8
:1019E000044B13B10448AFF300800123237010BDF2
:1019F0005C2C002000000000D867010008B5034BF4
:101A00001BB103490348AFF3008008BD000000008C
:101A1000602C0020D8670100014B1868704700BF98
:101A20003801002008B5FAF799FF08BD08B5FAF7A4
:101A3000A3FF08BD08B5FAF7ADFF08BD08B5FAF772
:101A4000B7FF08BD08B5FAF7C1FF08BD08B5FAF73A
:101A5000CBFF08BD08B5FAF7D5FF08BD08B5FAF702
:101A6000DFFF08BD08B5FAF7E9FF08BD08B5FAF7CA
:101A7000F3FF08BD08B5FAF7FDFF08BD08B5FBF791
:101A800007F808BD08B5FBF711F808BD08B5FBF766
:101A90001BF808BD08B5FBF725F808BD08B5EEF73B
:101AA000E2FB08BD08B5EEF7DEFB08BD08B5EEF7B2
:101AB000DAFB08BD08B5EEF7D6FB08BD08B5EEF7B2
:101AC000D2FB08BD08B5EEF7CEFB08BD08B5EEF7B2
:101AD000CAFB08BD08B5EEF7C6FB08BD08B5FBF7A5
:101AE00013FE08BD08B5FAF715FC08BD08B5FAF7EE
:101AF00031FC08BD08B5FBF737FF08BD08B5FBF79B
:101B000059FF08BD08B5EEF7AEFB08BD08B502F0F9
:101B1000FFFF08BD08B5EEF7A6FB08BD08B503F04A
:101B200000F808BD08B5EEF79EFB08BD08B503F048
:101B300001F808BD08B5EEF796FB08BD08B503F03F
:101B400002F808BD08B5EEF78EFB08BD08B5EEF744
:101B50008AFB08BD08B5EEF786FB08BD08B5EEF7B1
:101B600082FB08BD08B5EEF77EFB08BD08B5EEF7B1
:101B70007AFB08BD08B5EEF776FB08BD08B5EEF7B1
:101B800072FB08BD08B5EEF76EFB08BD08B5EEF7B1
:101B90006AFB08BD08B5EEF766FB08BD08B5EEF7B1
:101BA00062FB08BD08B5EEF75EFB08BD08B5EEF7B1
:101BB0005AFB08BD08B5EEF756FB08BD08B5EEF7B1
:101BC00052FB08BD08B5EEF74EFB08BD08B5EEF7B1
:101BD0004AFB08BD08B5EEF746FB08BD08B5EEF7B1
:101BE00042FB08BD08B5EEF73EFB08BD08B5EEF7B1
:101BF0003AFB08BD08B5EEF736FB08BD08B5FAF7A5
:101C0000C9FB08BD08B502F0A7FF08BD08B5EEF78F
